:020000040800F2
:1000000000100020813B0008F13C000841B60108C7
:10001000F13C000821B6010801B60108F13C0008D6
:10002000F13C0008F13C0008F13C0008213D0008CB
:10003000E1B50108F13C0008F13C0008213E000850
:10004000F13C0008518E0008F13C0008918F000837
:10005000F13C0008F13C0008118C0008418C0008BC
:10006000718C0008A18C0008D18C0008B1800008B8
:10007000F18000083181000871810008B181000819
:10008000F181000831820008218A0008619300088C
:1000900081930008A1930008C1930008018D000816
:1000A000A1B1000821B10008F13C000841B10008ED
:1000B00061B1000881B10008B1B40008F19A0008EC
:1000C000319C0008F13C0008F13C0008F13C0008BC
:1000D000F13C000831B9000851B9000871B90008B5
:1000E000A18D0008918E0008D18E0008F13C000817
:1000F00041B50008F13C000871B5000871820008A4
:10010000F13C0008F13C000881AF0008F13C000818
:10011000F13C0008F13C0008F13C0008F13C00080B
:10012000B1820008F1820008318300087183000861
:10013000B1830008F13C0008118F0008E19300082A
:10014000019400082194000841940008D1A70008F8
:10015000F18300083184000871840008F13C000834
:10016000F13C0008F13C0008F13C0008F13C0008BB
:10017000518F0008F13C0008F13C0008F13C0008F8
:10018000F13C0008F13C0008F13C0008F13C00089B
:10019000F13C0008F13C0008F13C0008F13C00088B
:0C01A000F13C0008F13C0008F13C0008B4
:1001AC0051020008D1020008F102000811030008F6
:1001BC005103000891030008C1030008E103000883
:1001CC00010400082104000861040008A1040008CF
:1001DC00C1040008610500087105000891050008BC
:1001EC00B1050008F10500081106000831060008E9
:1001FC0081060008E1060008110700083107000815
:10020C00B1070008D107000891080008B1080008E0
:10021C00D1080008210900084109000881090008DB
:10022C00D1090008710C0008C10C0008A10E0008CF
:0C023C007110000891100008F11000087B
:1002500070B542F68054C2F2000442F610212046E6
:10026000C2F2000125F0ACF942F68441201DC2F231
:10027000000125F0A5F942F6703104F10800C2F240
:10028000000125F09DF942F67443C2F2000326688E
:100290006568A4681E6042F6103042F220611A467A
:1002A0005D609C60C2F20001C2F2000014F018FE12
:1002B00042F66C40C2F2000025F05AF942F6704353
:1002C000C2F2000300221A705A709A7070BD00BF0B
:1002D00010B542F69854C2F20004204614F028FFEC
:1002E00004F11800BDE8104014F022BFAFF3008005
:1002F00008B543F64850C2F2000011F0D1FB42F6B7
:10030000D050C2F20000BDE808400EF0F9B800BFBE
:1003100038B543F6C05044F6E834C2F20004002574
:10032000C2F2000025F024F9204629464FF48072DD
:10033000C4F8005102F0FCFE4023C4F80451C4F894
:100340000831C4F8045138BDAFF30080AFF300802A
:1003500038B544F6F44044F60854C2F200040025CF
:10036000C2F2000014F0D4FF204629464FF48072F8
:10037000C4F8005102F0DCFE4023C4F80451C4F874
:100380000831C4F8045138BDAFF30080AFF30080EA
:1003900010B544F61464C2F20004204614F0B8FF0D
:1003A00004F1100014F0B4FF04F12000BDE8104087
:1003B00014F0AEBFAFF30080AFF30080AFF3008066
:1003C00044F688604AF2742144F6C462C2F2000026
:1003D000C0F60201C2F2000241F2883324F018B9DB
:1003E00046F264204AF25031C2F20000C0F6020127
:1003F00024F026B9AFF30080AFF30080AFF30080A4
:10040000044B002103F5DC7243F8581C5833934227
:10041000FAD17047C8630020AFF30080AFF30080CB
:10042000F8B546F660060024C2F20006402746F6FC
:100430001405C2F2000521463A463046B46402F083
:1004400077FE3A462846214634647464AC6402F070
:100450006FFE2C646C64F8BDAFF30080AFF30080D6
:10046000F8B546F6F8060024C2F20006402746F624
:10047000AC05C2F2000521463A463046B46402F0AB
:1004800057FE3A462846214634647464AC6402F050
:100490004FFE2C646C64F8BDAFF30080AFF30080B6
:1004A00046F64C1040F68031C2F20000C0F603015F
:1004B00024F0C6B8AFF30080AFF30080AFF3008044
:1004C00046F65C20C2F2000046F69C4110B40022C1
:1004D000C2F200014FF0FF3481608161816281636B
:1004E000816481650260426002614261026242622F
:1004F000026342630264426402654265C460C4618F
:10050000C462C463C464C46500F1740300F5B270CE
:1005100043F80C1C43F8142C43F8102C43F8084CF7
:1005200043F8042C14338342F2D10A4B002203F126
:10053000F0044FF0FF3043F80C1C43F8142C43F840
:10054000102C03E905001433A342F4D15DF8044BE9
:10055000704700BFC06B0020AFF30080AFF3008096
:1005600046F6A040C2F2000014F022BFAFF30080B4
:1005700046F6DC704DF63841C2F20000C0F60201CA
:1005800024F05EB8AFF30080AFF30080AFF30080DB
:1005900047F280104DF66061C2F20000C0F6020121
:1005A00024F04EB8AFF30080AFF30080AFF30080CB
:1005B00038B50D4C04F50065204624F0E9F804F147
:1005C0007C0004F5807424F0E3F8AC42F4D147F2E7
:1005D0006874C2F20004201D00214FF4006202F092
:1005E000A7FD0023236038BD74770020AFF300809F
:1005F00048F2F0204EF29001C2F20000C0F6020173
:1006000024F01EB8AFF30080AFF30080AFF300809A
:1006100048F668404EF28C21C2F20000C0F602019A
:1006200024F00EB8AFF30080AFF30080AFF300808A
:1006300008B549F294104EF2E84148F6AC624FF426
:10064000FA73C0F60201C2F20002C2F2000023F007
:10065000DFFF49F2A40041F2C471C2F20001C2F20C
:10066000000019F0A5F848F6BC5041F26871C2F2DA
:100670000000C2F20001BDE8084019F099B800BFBF
:1006800049F2CC404EF6400138B5C0F60201C2F244
:10069000000014F02DFE49F2E04549F24850C2F244
:1006A0000005C2F2000014F033FE49F2105428464F
:1006B00014F03EFDC2F2000405F1180014F038FDFC
:1006C000204614F035FD04F11800BDE8384014F060
:1006D0002FBD00BFAFF30080AFF30080AFF3008009
:1006E00008B549F660104EF60421C2F20000C0F6CB
:1006F000020123F0A5FF49F64C10C2F20000BDE84C
:10070000084014F005BE00BFAFF30080AFF30080D7
:1007100049F670404FF28811C2F20000C0F60201A3
:1007200023F08EBFAFF30080AFF30080AFF3008003
:100730004EF64C204FF284414EF2A04208B5C2F270
:1007400000024FF4AF63C0F60201C2F2000023F0D2
:100750005FFF4EF68C204FF29041C0F60201C2F2CC
:10076000000023F06DFF4EF2A8004FF29C41C0F64E
:100770000201C2F2000023F063FF4EF29800C2F2C1
:10078000000014F0C5FD4EF61820C2F2000014F06F
:10079000BFFD4EF62820C2F2000014F0B9FD4EF65F
:1007A0003820C2F20000BDE8084014F0B1BD00BF1F
:1007B00040F698404FF2CC71C2F20100C0F602013F
:1007C00023F03EBFAFF30080AFF30080AFF30080B3
:1007D00010B540F6B45082B0C2F2010025F0A8FB7B
:1007E0004CF2AE73C4F236330024009340F6CC5082
:1007F00047F6E12200232146CCF2D402C4F2A00342
:10080000C2F2010025F09CFB40F6A4504DF6100208
:10081000002300944FF07C51C4F2B622C4F240038E
:10082000C2F2010025F08CFB0023C4F24833009390
:1008300040F6BC50002321462246C4F2A003C2F277
:10084000010025F07DFB0023C4F28233009340F6C3
:10085000AC50002321464FF08242C4F2A003C2F202
:10086000010025F06DFB0023C4F2C823009340F67D
:10087000C450002322464FF07C51C4F29003C2F2D0
:10088000010025F05DFB02B010BD00BFAFF300809A
:1008900041F2802040F6905140F69862C2F2010089
:1008A000C0F60301C2F201024FF47A7323F0B0BE26
:1008B00041F2E02040F6D051C2F20100C0F603013F
:1008C00023F0BEBEAFF30080AFF30080AFF3008033
:1008D00038B541F2B84040F6E02141F24045C0F65B
:1008E0000301C2F20105C2F2010014F001FD41F260
:1008F0007844284614F01CFCC2F2010405F11800EB
:1009000014F016FC204614F013FC04F11800BDE8A6
:10091000384014F00DBC00BFAFF30080AFF300808F
:1009200041F6000041F2C011C2F20100C0F603011D
:1009300023F086BEAFF30080AFF30080AFF30080FA
:1009400041F6707008B5C2F2010014F0E1FC41F606
:100950002040C2F2010014F0A3FA41F61810C2F2CE
:1009600001001AF0FDFB41F68470C2F20100BDE8FF
:10097000084011F0CDBD00BFAFF30080AFF30080A1
:1009800010B542F2A82082B0C2F2010014F088FA39
:1009900042F29420C2F2010014F0BAFC00244FF09D
:1009A0007E5100220091C4F2B42442F2782000214A
:1009B00013460194C4F22011C2F2010026F068FF30
:1009C00002B010BDAFF30080AFF30080AFF3008042
:1009D0002DE9F04142F60824C2F20104002142F25E
:1009E0006C67C2F201070A46204642F6502814F00E
:1009F000BFF8C2F201082146384614F041F842F22D
:100A00002475396840460722C2F2010514F0C0F887
:100A100041F2DC4239682846C0F6030242F69C14D3
:100A2000C2F2010414F0A4F841F2E442396820460D
:100A3000C0F6030242F2B476C2F2010614F098F84E
:100A400041F2F04239683046C0F6030214F090F8E3
:100A500042F6E80041460822C2F2010014F098F87C
:100A600042F6E41041460922C2F2010014F090F867
:100A700042F6C01029460A22C2F2010014F088F89A
:100A800042F27C6029460B22C2F2010014F080F889
:100A900042F2FC7029460D22C2F2010014F078F8EF
:100AA00042F2006029460E22C2F2010014F070F8F2
:100AB00042F67C0029461022C2F2010014F068F8C8
:100AC00042F6DC2029460C22C2F2010014F060F844
:100AD00042F6A00029461422C2F2010014F058F890
:100AE00042F6B82029461122C2F2010014F050F853
:100AF00042F6942029461222C2F2010014F048F86E
:100B000042F6541041F2F8424FF251532146C0F6DA
:100B10000302C0F60103C2F2010014F019F842F218
:100B2000907041F2045242F241232146C0F6030282
:100B3000C0F60203C2F2010014F00AF842F678107F
:100B400041F2105242F2D123C0F602032146C0F610
:100B50000302C2F2010013F0FBFF42F2DC6041F23B
:100B60001C522146C0F60302C2F2010014F000F844
:100B700042F2007041F228522146C0F60302C2F24E
:100B8000010013F0F5FF42F2B86041F23452214601
:100B9000C0F60302C2F2010013F0EAFF42F248700D
:100BA00041F240522146C0F60302C2F2010013F0A6
:100BB000DFFF42F2D87041F24C522146C0F60302E8
:100BC000C2F2010013F0D4FF42F2486041F25C52DD
:100BD0002146C0F60302C2F2010013F0C9FF42F63B
:100BE000200041F26C522146C0F60302C2F201001D
:100BF00013F0BEFF42F6440041F27C522146C0F69B
:100C00000302C2F2010013F0B3FF42F6C400314602
:100C10000122C2F2010013F0BBFF42F22460314610
:100C20000222C2F2010013F0B3FF42F62C2031463B
:100C30000322C2F2010013F0ABFF42F6301031463E
:100C40000422C2F2010013F0A3FF42F26C7031469D
:100C50000522C2F2010013F09BFF42F60C10314650
:100C6000C2F201000622BDE8F04113F091BF00BFBF
:100C700042F61C6041F2447108B5C0F60301C2F2AD
:100C8000010023F0DDFC41F67810C1F2000013F002
:100C9000EFFA42F620700949C2F2010013F0D8FCC5
:100CA00042F62830C2F2010024F022FC42F618601D
:100CB000C2F20100BDE8084024F05ABC586400109C
:100CC0002DE9F00F47F6AC30C2F2010082B047F6D2
:100CD0000032C2F201020168019047F6D02347F6C4
:100CE000DC20C2F201031160C2F201004EF65C6129
:100CF0000090C0F60201062047F6E82AC2F2010A77
:100D0000916050601A6041F68422C0F6030247F6F3
:100D10009439C2F2010958609A60CAF800304EF264
:100D200040230720C0F6020347F65838C2F20108F4
:100D3000CAF80830CAF80400C9F800A041F6882AA9
:100D4000C0F6030AC9F80400C9F808A0C8F8009062
:100D500047F6A03C4FF00809C2F2010CC8F8049015
:100D600041F68C29C0F60309C8F80890CCF8008039
:100D700047F6C4274FF00908C2F20107CCF80480F7
:100D800041F69028C0F6030847F60C36C2F2010679
:100D9000CCF80880C7F800C047F664354FF00A0C5D
:100DA00041F69428C2F20105C7F804C0C0F6030852
:100DB00047F6883441F6982CC2F20104C7F808803F
:100DC0003760C0F6030C0B2741F69C287760C6F805
:100DD00008C02E60C0F603080C2641F6D8376E60B6
:100DE000C5F808802560C0F603070325656041F655
:100DF000A02CA7600098C0F6030C0527046047608C
:100E0000C0F808C047F67C3B0198C2F2010B47F6D8
:100E1000B821C2F20101C0F800B047F6B032009824
:100E200047F6703347F6F42A41F6A426C2F20103CE
:100E3000C2F2010AC2F20102C0F60306022441F620
:100E4000A82841F6AC2541F6B02741F6B42CC0F6EF
:100E50000308C0F60305C0F60307C0F6030C4FF005
:100E6000040908604C600D200E248E600F2682E875
:100E70000202C2F808801A6058609D60CAF800300B
:100E8000CBF800A0CAF80440CAF80870CBF8046098
:100E9000CBF808C002B0BDE8F00F7047AFF3008098
:100EA00048F6845049F6781238B5C0F6020264213B
:100EB000C2F2010024F04CFC48F654604FF66C522C
:100EC000C0F602026A21C2F2010024F041FC49F29C
:100ED00084004FF20032C0F602026B21C2F2010020
:100EE00024F036FC48F63C604FF24432C0F6020271
:100EF0006D21C2F2010024F02BFC48F69C5040F614
:100F00008042C0F603026621C2F2010024F020FCF8
:100F100048F6745041F6A462C0F603026521C2F29D
:100F2000010024F015FC49F26C0041F6B452C0F601
:100F300003026E21C2F2010024F00AFC48F6A85018
:100F400041F6AC62C0F603026821C2F2010024F04F
:100F5000FFFB47F64C5041F6BC62C0F60302692124
:100F6000C2F2010024F0F4FB48F2685041F6CC6272
:100F7000C0F603026721C2F2010024F0E9FB48F247
:100F80005C5041F66C62C0F603026F21C2F20100B0
:100F900024F0DEFB47F6C030C2F2010048F6606480
:100FA00024F0F6FBC2F2010404F50075204610346B
:100FB00024F0DEFBAC42F9D149F2600048F66061F2
:100FC000C2F20100C2F20101202247F65C5424F073
:100FD00077FEC2F2010404F500652046103424F0C7
:100FE000C7FBAC42F9D148F6905047F65C51C2F2CB
:100FF0000100C2F20101802248F2745424F060FE24
:10100000C2F2010404F500652046103424F0B0FB60
:10101000AC42F9D148F6486048F27451C2F201007E
:10102000C2F2010180220F4C24F04AFE04F5E06573
:101030002046703413F034FFAC42F9D148F6B45076
:10104000C2F2010047F64C4424F0A2FBC2F20104B4
:1010500004F580752046103414F05AF9AC42F9D1E9
:1010600038BD00BF90C10010AFF30080AFF3008027
:1010700008B5054826F0E4FB4CF69000C1F20000EC
:1010800026F0DEFB08BD00BFE0DA0010AFF3008001
:101090002DE9F04149F2DC070024C2F201074FF0CC
:1010A000400849F29006C2F20106214642463846FF
:1010B00049F22815C2F20105BC6402F039F8214654
:1010C000424630463C647C64B46402F031F84246E7
:1010D0002846214634647464AC6402F029F82C6418
:1010E0006C64BDE8F08100BFAFF30080AFF3008017
:1010F00049F2741042F2E811C2F20100C0F6030195
:1011000023F09EBAAFF30080AFF30080AFF300800E
:1011100008B504F0CDFA02F033FF1AF059FA26F0C0
:10112000BFFD002008BD00BFAFF30080AFF300801B
:1011300050EA010301D102207047D0F1010338BF0A
:101140000023B1F1004F08BF0028F4D021F0004186
:101150004FF6FF72A1F58010C7F6DF72904201D8FA
:1011600004207047B1F5801F01D203207047002092
:10117000C7F6F070814214BF002003F001007047F1
:10118000C1F30A5C2DE9F843ACF2FF33132B06469A
:101190000F4613DC002B40DB4FF6FF7CC0F20F0C38
:1011A0004CFA03F303EA010C5CEA000C1CD107F0D3
:1011B0000041C2E900676046BDE8F883332B1EDCBE
:1011C0004FF0FF33ACF2134C23FA0CFC1CEA000383
:1011D0001CD020EA0C060F460B46C2E900673246D7
:1011E00000F09AFABDE8F88321EA030700263B469F
:1011F000C2E90067324600F08FFABDE8F88307F0D5
:101200000041C2E900670020BDE8F88307F0004113
:10121000C2E900671846BDE8F88307F000494FF0BF
:101220000008C2E90089BDE8F88300BF00000000A3
:10123000F8B5C1F30A57A7F2FF360246132E0B4644
:101240000D468C4616DC002E31DB4FF6FF7CC0F2DB
:101250000F0C4CFA06FC0CEA010101430FD04FF4CD
:101260000023002143FA06F62E4426EA0C0C084619
:101270006146F8BD332E05DDB6F5806F23D01046EC
:101280001946F8BD4FF0FF30A7F21341C840104295
:10129000F5D0C7F5866701210237B940891828BF04
:1012A00003F1010C21EA000108466146F8BD01F096
:1012B000004C013602BF4CF07F5C00214CF4401C16
:1012C000D5D00021D3E700F029FAF8BD00000000D6
:1012D00070B58AB0054600F06BF841F20064C2F2C6
:1012E000000494F900300133064609D0284600F086
:1012F000EFF928B12846002101F0A6F9034610B104
:1013000030460AB070BD42F2F0122846C0F6030221
:101310000893019200F060FB2478CDE90401CDE947
:10132000020174BB4FF6FF734FF06042CCF2EF73D3
:10133000CDE906232846002101F05EF978B10223A9
:1013400000939C4229D0684600F0B2F928B3089B6C
:1013500043BBDDE9060100F05BFE0AB070BD022C64
:101360004FF00103009313D0684600F0A1F978B163
:1013700041F64810C0F6030000F0A2F9CDE90601DD
:10138000E5E700230022CFF6F073CDE90623D1E78D
:1013900001F06EFE21230360EAE701F069FE2223DB
:1013A0000360D4E701F064FE089B0360D1E700BF4F
:1013B00020F0004201462DE9F84F0346002A00F0D4
:1013C000B0800028C0F2D380B0F1FF4F80F2CB8014
:1013D000B0F5000FA8BF002706DA4FF098416FF074
:1013E000180700F075FF03464FF62030C3F31604CC
:1013F000C0F24A00DB1520447F3B00F400021F448A
:1014000082F07E504FF07E51204307EBD25700F020
:1014100053FE04F10F03C3F316030F2B054640F3ED
:1014200087804FF0804145F6304800F047FECFF608
:10143000CF78A044C4F5571404F5227444EA080890
:101440000146284600F0F8FF8146384600F0EAFEE3
:1014500049468346484600F03BFF0146824600F07D
:1014600037FF48F69701C3F61761064600F030FFD4
:1014700043F22531C3F63A6100F020FE314600F018
:1014800027FF44F62511C3F6926100F017FE31469E
:1014900000F01EFF4AF6AB21C3F62A7100F00EFEE3
:1014A000514600F015FF4DF24F01C3F61C61824614
:1014B000304600F00DFF48F62961C3F6636100F085
:1014C000FDFD314600F004FF4CF6CD41C3F6CC6182
:1014D00000F0F4FD314600F0FBFE0146504600F0FE
:1014E000EDFDB8F1000F064640F3AF804FF07C51A0
:1014F000284600F0EDFE294600F0EAFE0446002FE3
:1015000059D1314600F0DAFD494600F0E1FE0146CE
:10151000204600F0D1FD0146284600F0CDFDBDE893
:10152000F88F00214FF04C4000F086FFBDE8F88FA7
:10153000002101F061F808B3002F00F083803846E5
:1015400000F070FE4FF4E341C3F63171054600F040
:10155000BFFE4FF2D171C3F217710446284600F066
:10156000B7FE0146204600F0A9FDBDE8F88F00F067
:10157000A3FD002100F060FFBDE8F88F2946284652
:1015800000F0A6FE4AF6AB21C3F6AA61044628463F
:1015900000F09EFE01464FF07C5000F08DFD0146AC
:1015A000204600F095FE04466FBB2846214600F019
:1015B00083FDBDE8F88F4FF4E3415846C3F631711F
:1015C00000F086FE31460746204600F077FD49468A
:1015D00000F07EFE4FF2D171C3F2177106465846F5
:1015E00000F076FE0146304600F068FD01462046D8
:1015F00000F062FD294600F05FFD0146384600F02C
:101600005BFDBDE8F88F384600F00CFE4FF4E34177
:10161000C3F63171074600F05BFE4FF2D171C3F2A1
:1016200017710646384600F053FE0146204600F08A
:1016300043FD294600F040FD0146304600F03CFDE8
:10164000BDE8F88F0020BDE8F88F1FB34FF4E341E9
:101650005846C3F6317100F03BFE31460446284639
:1016600000F02AFD494600F033FE4FF2D171C3F27B
:1016700017710646584600F02BFE0146304600F032
:101680001BFD294600F018FD0146204600F014FD20
:10169000BDE8F88F0146284600F00EFD494600F0EF
:1016A00017FE0146284600F007FDBDE8F88F00BF91
:1016B0000020704700000000000000000000000053
:1016C00000210020C7F6F871704700BF000000003D
:1016D00030F0004001D102207047A0F50003B3F1C3
:1016E000FE4F01D2042070474FF6FE73421EC0F237
:1016F0007F039A4201D803207047B0F1FF4358425C
:101700005841704700000000000000000000000089
:1017100081F0004102E000BF83F0004330B54FEAA2
:1017200041044FEA430594EA050F08BF90EA020F0F
:101730001FBF54EA000C55EA020C7FEA645C7FEAA2
:10174000655C00F0E2804FEA5454D4EB5555B8BFC5
:101750006D420CDD2C4480EA020281EA030382EA36
:10176000000083EA010180EA020281EA0303362DC8
:1017700088BF30BD11F0004F4FEA01314FF4801C9B
:101780004CEA113102D0404261EB410113F0004FAD
:101790004FEA03334CEA133302D0524263EB430364
:1017A00094EA050F00F0A780A4F10104D5F1200E02
:1017B0000DDB02FA0EFC22FA05F2801841F100015D
:1017C00003FA0EF2801843FA05F359410EE0A5F131
:1017D00020050EF1200E012A03FA0EFC28BF4CF062
:1017E000020C43FA05F3C01851EBE37101F0004518
:1017F00007D54FF0000EDCF1000C7EEB00006EEB25
:101800000101B1F5801F1BD3B1F5001F0CD34908AE
:101810005FEA30004FEA3C0C04F101044FEA445205
:1018200012F5800F80F09A80BCF1004F08BF5FEA8C
:10183000500C50F1000041EB045141EA050130BD6C
:101840005FEA4C0C404141EB010111F4801FA4F10F
:101850000104E9D191F0000F04BF01460020B1FA64
:1018600081F308BF2033A3F10B03B3F120020CDA9C
:101870000C3208DD02F1140CC2F10C0201FA0CF07A
:1018800021FA02F10CE002F11402D8BFC2F1200CDF
:1018900001FA02F120FA0CFCDCBF41EA0C01904095
:1018A000E41AA2BF01EB0451294330BD6FEA0404DE
:1018B0001F3C1CDA0C340EDC04F11404C4F12002C9
:1018C00020FA04F001FA02F340EA030021FA04F3DB
:1018D00045EA030130BDC4F10C04C4F1200220FA32
:1018E00002F001FA04F340EA0300294630BD21FA70
:1018F00004F0294630BD94F0000F83F4801306BF36
:1019000081F480110134013D4EE77FEA645C18BF29
:101910007FEA655C29D094EA050F08BF90EA020FC0
:1019200005D054EA000C04BF1946104630BD91EAB8
:10193000030F1EBF0021002030BD5FEA545C05D1BB
:101940004000494128BF41F0004130BD14F58004FA
:101950003CBF01F5801130BD01F0004545F0FE416E
:1019600041F470014FF0000030BD7FEA645C1ABFA3
:10197000194610467FEA655C1CBF0B46024650EADA
:10198000013406BF52EA033591EA030F41F4002106
:1019900030BD00BF90F0000F04BF0021704730B58C
:1019A0004FF4806404F132044FF000054FF0000161
:1019B00050E700BF90F0000F04BF0021704730B522
:1019C0004FF4806404F1320410F0004548BF4042F7
:1019D0004FF000013EE700BF42004FEAE2014FEA4C
:1019E00031014FEA02701FBF12F07F4393F07F4F27
:1019F00081F06051704792F0000F14BF93F07F4F59
:101A0000704730B54FF4607401F0004521F000419B
:101A100020E700BF50EA010208BF704730B54FF021
:101A200000050AE050EA010208BF704730B511F026
:101A3000004502D5404261EB41014FF4806404F15E
:101A400032045FEA915C3FF4DCAE4FF003025FEAE0
:101A5000DC0C18BF03325FEADC0C18BF033202EB68
:101A6000DC02C2F1200300FA03FC20FA02F001FAC2
:101A700003FE40EA0E0021FA02F11444C1E600BF61
:101A800070B54FF0FF0C4CF4E06C1CEA11541DBF14
:101A90001CEA135594EA0C0F95EA0C0F00F0DEF8DF
:101AA0002C4481EA030621EA4C5123EA4C5350EAC4
:101AB000013518BF52EA033541F4801143F4801315
:101AC00038D0A0FB02CE4FF00005E1FB02E506F0A6
:101AD0000042E0FB03E54FF00006E1FB03569CF0FB
:101AE000000F18BF4EF0010EA4F1FF04B6F5007F01
:101AF00064F5407404D25FEA4E0E6D4146EB060673
:101B000042EAC62141EA55514FEAC52040EA5E50FB
:101B10004FEACE2EB4F1FD0C88BFBCF5E06F1ED8A5
:101B2000BEF1004F08BF5FEA500E50F1000041EBDC
:101B3000045170BD06F0004646EA010140EA020089
:101B400081EA0301B4EB5C04C2BFD4EB0C0541EAAB
:101B5000045170BD41F480114FF0000E013C00F3C0
:101B6000AB8014F1360FDEBF002001F0004170BDE4
:101B7000C4F10004203C35DA0C341BDC04F11404FD
:101B8000C4F1200500FA05F320FA04F001FA05F289
:101B900040EA020001F0004221F0004110EBD37056
:101BA00021FA04F642EB06015EEA430E08BF20EA82
:101BB000D37070BDC4F10C04C4F1200500FA04F325
:101BC00020FA05F001FA04F240EA020001F00041B7
:101BD00010EBD37041F100015EEA430E08BF20EA2A
:101BE000D37070BDC4F1200500FA05F24EEA020E72
:101BF00020FA04F301FA05F243EA020321FA04F0A1
:101C000001F0004121FA04F220EA020000EBD37057
:101C10005EEA430E08BF20EAD37070BD94F0000F57
:101C20000FD101F00046400041EB010111F4801F8B
:101C300008BF013CF7D041EA060195F0000F18BF3C
:101C4000704703F00046520043EB030313F4801F78
:101C500008BF013DF7D043EA0603704794EA0C0F32
:101C60000CEA135518BF95EA0C0F0CD050EA410648
:101C700018BF52EA4306D1D181EA030101F00041C5
:101C80004FF0000070BD50EA410606BF10461946ED
:101C900052EA430619D094EA0C0F02D150EA0136F9
:101CA00013D195EA0C0F05D152EA03361CBF10463A
:101CB00019460AD181EA030101F0004141F0FE41D9
:101CC00041F470014FF0000070BD41F0FE4141F45D
:101CD000780170BD70B54FF0FF0C4CF4E06C1CEA5D
:101CE00011541DBF1CEA135594EA0C0F95EA0C0F12
:101CF00000F0A7F8A4EB050481EA030E52EA0335CD
:101D00004FEA013100F088804FEA03334FF08055ED
:101D100045EA131343EA12634FEA022245EA11151A
:101D200045EA10654FEA00260EF000419D4208BFCB
:101D3000964244F1FD0404F5407402D25B084FEA78
:101D40003202B61A65EB03055B084FEA32024FF424
:101D500080104FF4002CB6EB020E75EB030E22BF81
:101D6000B61A754640EA0C005B084FEA3202B6EB41
:101D7000020E75EB030E22BFB61A754640EA5C00F0
:101D80005B084FEA3202B6EB020E75EB030E22BF80
:101D9000B61A754640EA9C005B084FEA3202B6EB81
:101DA000020E75EB030E22BFB61A754640EADC0040
:101DB00055EA060E18D04FEA051545EA16754FEAA2
:101DC00006164FEAC30343EA52734FEAC2025FEAC0
:101DD0001C1CC0D111F4801F0BD141EA00014FF04F
:101DE00000004FF0004CB6E711F4801F04BF014320
:101DF0000020B4F1FD0C88BFBCF5E06F3FF6AFAE3C
:101E0000B5EB030C04BFB6EB020C5FEA500C50F1CB
:101E1000000041EB045170BD0EF0004E4EEA11314E
:101E200014EB5C04C2BFD4EB0C0541EA045170BD55
:101E300041F480114FF0000E013C90E645EA060E99
:101E40008DE60CEA135594EA0C0F08BF95EA0C0FC7
:101E50003FF43BAF94EA0C0F0AD150EA01347FF40F
:101E600034AF95EA0C0F7FF425AF104619462CE7E6
:101E700095EA0C0F06D152EA03353FF4FDAE104649
:101E8000194622E750EA410618BF52EA43067FF49A
:101E9000C5AE50EA41047FF40DAF52EA43057FF42A
:101EA000EBAE12E7000000000000000000000000A0
:101EB0004FF0FF3C06E000BF4FF0010C02E000BF16
:101EC0004FF0010C4DF804CD4FEA410C7FEA6C5CF9
:101ED0004FEA430C18BF7FEA6C5C1BD001B050EA9C
:101EE000410C0CBF52EA430C91EA030F02BF90EA87
:101EF000020F0020704710F1000F91EA030F58BF46
:101F0000994208BF90422CBFD8176FEAE37040F0A7
:101F1000010070474FEA410C7FEA6C5C02D150EA45
:101F2000013C07D14FEA430C7FEA6C5CD6D152EA00
:101F3000033CD3D05DF8040B704700BF84461046C5
:101F400062468C461946634600E000BF01B5FFF7C4
:101F5000B7FF002848BF10F1000F01BD4DF808ED94
:101F6000FFF7F4FF0CBF012000205DF808FB00BF65
:101F70004DF808EDFFF7EAFF34BF012000205DF8BF
:101F800008FB00BF4DF808EDFFF7E0FF94BF01200C
:101F900000205DF808FB00BF4DF808EDFFF7CEFF0D
:101FA00094BF012000205DF808FB00BF4DF808ED4C
:101FB000FFF7C4FF34BF012000205DF808FB00BF1D
:101FC0004FEA410212F5001215D211D56FF4787361
:101FD000B3EB625212D94FEAC12343F0004343EA04
:101FE000505311F0004F23FA02F018BF40427047DF
:101FF0004FF00000704750EA013005D111F0004069
:1020000008BF6FF0004070474FF00000704700BFFE
:102010004FEA4102B2F1E04324BFB3F5001CDCF10A
:10202000FE5C0DD901F0004C4FEAC0024CEA507042
:10203000B2F1004F40EB830008BF20F00100704771
:1020400011F0804F21D113F13872BCBF01F0004074
:10205000704741F480114FEA5252C2F11802C2F1A6
:10206000200C10FA0CF320FA02F018BF40F0010027
:102070004FEAC1234FEAD32303FA0CFC40EA0C00D9
:1020800023FA02F34FEA4303CCE77FEA625307D116
:1020900050EA01331EBF4FF0FE4040F4400070474D
:1020A00001F0004040F0FE4040F40000704700BFE7
:1020B00080F0004002E000BF81F0004142001FBFFD
:1020C0005FEA410392EA030F7FEA226C7FEA236C06
:1020D0006AD04FEA1262D2EB1363C1BFD2184140FB
:1020E00048404140B8BF5B42192B88BF704710F091
:1020F000004F40F4000020F07F4018BF404211F034
:10210000004F41F4000121F07F4118BF494292EA9B
:10211000030F3FD0A2F1010241FA03FC10EB0C00C7
:10212000C3F1200301FA03F100F0004302D5494254
:1021300060EB4000B0F5000F13D3B0F1807F06D301
:1021400040084FEA310102F10102FE2A51D2B1F1F9
:10215000004F40EBC25008BF20F0010040EA0300EE
:102160007047490040EB000010F4000FA2F101029B
:10217000EDD1B0FA80FCACF1080CB2EB0C0200FA25
:102180000CF0AABF00EBC25052421843BCBFD04073
:102190001843704792F0000F81F4000106BF80F4ED
:1021A00000000132013BB5E74FEA41037FEA226CB0
:1021B00018BF7FEA236C21D092EA030F04D092F07B
:1021C000000F08BF0846704790EA010F1CBF0020AF
:1021D000704712F07F4F04D1400028BF40F000400C
:1021E000704712F100723CBF00F50000704700F02C
:1021F000004343F0FE4040F4000070477FEA226253
:1022000016BF08467FEA23630146420206BF5FEA23
:10221000412390EA010F40F4800070474FF0000323
:1022200004E000BF10F0004348BF40425FEA000CEA
:1022300008BF704743F0964301464FF000001CE092
:1022400050EA010208BF70474FF000030AE000BFE8
:1022500050EA010208BF704711F0004302D5404226
:1022600061EB41015FEA010C02BF84460146002098
:1022700043F0B64308BFA3F18053A3F50003BCFAB3
:102280008CF2083AA3EBC25310DB01FA02FC634460
:1022900000FA02FCC2F12002BCF1004F20FA02F267
:1022A00043EB020008BF20F00100704702F120025A
:1022B00001FA02FCC2F1200250EA4C0021FA02F2BB
:1022C00043EB020008BF20EADC707047000000000A
:1022D0004FF0FF0C1CEAD0521EBF1CEAD15392EA09
:1022E0000C0F93EA0C0F6FD01A4480EA010C4002E5
:1022F00018BF5FEA41211ED04FF0006343EA50103F
:1023000043EA5111A0FB01310CF00040B1F5000F80
:102310003EBF490041EAD3715B0040EA010062F12F
:102320007F02FD2A1DD8B3F1004F40EBC25008BF19
:1023300020F00100704790F0000F0CF0004C08BF37
:1023400049024CEA502040EA51207F3AC2BFD2F104
:10235000FF0340EAC250704740F400004FF0000312
:10236000013A5DDC12F1190FDCBF00F0004070474C
:10237000C2F10002410021FA02F1C2F1200200FA8A
:1023800002FC5FEA310040F1000053EA4C0308BF51
:1023900020EADC70704792F0000F00F0004C02BFA2
:1023A000400010F4000F013AF9D040EA0C0093F01D
:1023B000000F01F0004C02BF490011F4000F013B77
:1023C000F9D041EA0C018FE70CEAD15392EA0C0FE5
:1023D00018BF93EA0C0F0AD030F0004C18BF31F050
:1023E000004CD8D180EA010000F00040704790F026
:1023F000000F17BF90F0004F084691F0000F91F0CA
:10240000004F14D092EA0C0F01D142020FD193EA8F
:102410000C0F03D14B0218BF084608D180EA010017
:1024200000F0004040F0FE4040F40000704740F0F3
:10243000FE4040F4400070474FF0FF0C1CEAD052C1
:102440001EBF1CEAD15392EA0C0F93EA0C0F69D01D
:10245000A2EB030280EA010C49024FEA402037D088
:102460004FF0805343EA111143EA10130CF000407F
:102470008B4238BF5B0042F17D024FF4000C8B426F
:1024800024BF5B1A40EA0C00B3EB510F24BFA3EB4F
:10249000510340EA5C00B3EB910F24BFA3EB91031F
:1024A00040EA9C00B3EBD10F24BFA3EBD10340EA79
:1024B000DC001B0118BF5FEA1C1CE0D1FD2A3FF6BF
:1024C00050AF8B4240EBC25008BF20F00100704774
:1024D0000CF0004C4CEA50207F32C2BFD2F1FF0317
:1024E00040EAC250704740F400004FF00003013A48
:1024F00037E792F0000F00F0004C02BF400010F4EC
:10250000000F013AF9D040EA0C0093F0000F01F0FF
:10251000004C02BF490011F4000F013BF9D041EA21
:102520000C0195E70CEAD15392EA0C0F08D1420254
:102530007FF47DAF93EA0C0F7FF470AF084676E727
:1025400093EA0C0F04D14B023FF44CAF08466EE700
:1025500030F0004C18BF31F0004CCAD130F00042CE
:102560007FF45CAF31F000437FF43CAF5FE700BF26
:102570004FF0FF3C06E000BF4FF0010C02E000BF4F
:102580004FF0010C4DF804CD4FEA40024FEA4103F1
:102590007FEA226C18BF7FEA236C11D001B052EAA7
:1025A000530C18BF90EA010F58BFB2EB030088BF6D
:1025B000C81738BF6FEAE17018BF40F001007047DC
:1025C0007FEA226C02D15FEA402C05D17FEA236CBE
:1025D000E4D15FEA412CE1D05DF8040B704700BF05
:1025E000844608466146FFE70FB5FFF7C9FF00289C
:1025F00048BF10F1000F0FBD4DF808EDFFF7F4FFD5
:102600000CBF012000205DF808FB00BF4DF808ED6D
:10261000FFF7EAFF34BF012000205DF808FB00BF90
:102620004DF808EDFFF7E0FF94BF012000205DF8B2
:1026300008FB00BF4DF808EDFFF7D2FF94BF012063
:1026400000205DF808FB00BF4DF808EDFFF7C8FF5C
:1026500034BF012000205DF808FB00BF000000002F
:102660004BB942B9002908BF002802D04FF0FF3112
:10267000084600F065B882B0EC462DE9005000F045
:1026800047F8DDF804E002B00CBC70470000000021
:1026900070B5FFF7A1F900230022C3F6F0530446FA
:1026A0000D46FFF7EDF900F053F80646FFF772F913
:1026B00000230022C4F2F013FFF7E2F902460B46B2
:1026C00020462946FFF728F800F042F8002231465C
:1026D00042EA0004204670BD000000000000000037
:1026E0002DE9F0471746804689469A46089E00F035
:1026F0004FF8A7FB004507FB01F700FB0A721544E2
:10270000B8EB040469EB0505C6E90045BDE8F087B0
:102710002DE9F8431746804689461D46089E00F07D
:10272000E7F900FB05F3A0FB074507FB01373D4434
:10273000B8EB040469EB0505C6E90045BDE8F8837C
:10274000704700BF00000000000000000000000013
:102750004A0011D212F5001211D20DD56FF4787320
:10276000B3EB62520ED44FEAC12343F0004343EA75
:10277000505323FA02F070474FF00000704750EAC0
:10278000013002D14FF0FF3070474FF0000070472A
:102790002DE9F04F444261EB410500294FF0FF362F
:1027A000A2BF04460D460026002B85B0C0F2C780AC
:1027B0002046AA469446194690462746A946002B2D
:1027C00058D1AA426CD9B2FA82F35BB1C3F12002AC
:1027D00005FA03F924FA02F20CFA03F842EA0909AD
:1027E00004FA03F74FEA1844484621461FFA88FACC
:1027F00000F0FEFA21468346484600F027FC3A0CDA
:102800000AFB0BF042EA014188420BD911EB0801A7
:102810000BF1FF3305D2884284BFABF1020B414478
:1028200000D89B46C0EB010921464846BFB200F0E4
:10283000DFFA21460546484600F008FC0AFB05FA87
:1028400047EA01418A4509D911EB080805F1FF3330
:1028500003D2C24588BF023D00D81D4645EA0B435E
:1028600000241846214616B1404261EB410105B0F3
:10287000BDE8F08FAB4284BF00242346F1D8B1FA03
:1028800081F5002D40F0B580514528BF82428CBFB4
:10289000002401249CBF01232C46E2D92346E0E713
:1028A00022B91146012000F0A3FA8046B8FA88F355
:1028B000002B49D1C8EB09094FEA18451FFA88FADD
:1028C00001242946484600F093FA294683464846A3
:1028D00000F0BCFB3A0C0AFB0BF042EA01418842D3
:1028E0000CD911EB08010BF1FF3380F0F280884224
:1028F00084BFABF1020B414440F2EB800A1A294637
:102900001046019200F074FA019A2946BFB281463E
:10291000104600F09BFB0AFB09FA47EA01418A4591
:102920000AD911EB080809F1FF3304D2C24588BF68
:10293000A9F1020900D8994649EA0B4391E7F64309
:10294000524263EB430333E708FA03F8C3F1200B69
:1029500029FA0BF409FA03F94FEA184520462946EB
:1029600027FA0BFB9F4000F043FA29461FFA88FA2A
:102970004BEA090B02462046019200F067FB019AE0
:102980004FEA1B430AFB02F043EA014188420BD99C
:1029900011EB080102F1FF3380F0A180884284BF6F
:1029A000023A414440F29B80C0EB01092946484667
:1029B000019200F01DFA29461FFA8BFB0446484697
:1029C00000F044FB019A0AFB04F94BEA01418945F6
:1029D0000AD911EB080104F1FF3304D2894584BF01
:1029E000023C414400D81C46C9EB010944EA0244B8
:1029F00067E7C5F12003A94022FA03F82AFA03FB8E
:102A000048EA010820FA03F30AFA05FA58464FEAA1
:102A1000184902FA05FC494643EA0A0ACDF80CC0F7
:102A200000F0E6F949460446584600F00FFB1FFA4D
:102A300088F24FEA1A4E02FB04F04EEA014E70454E
:102A400009D91EEB080E04F1FF3146D2704584BF50
:102A5000023CC64441D9C0EB0E0C49466046019287
:102A6000CDF808C000F0C4F9DDF808C049461FFAE7
:102A70008AFA8346604600F0E9FA019A02FB0BF2FB
:102A80004AEA01418A420AD911EB08010BF1FF30F1
:102A900021D28A4284BFABF1020B41441BD9039877
:102AA0004BEA044B891AABFB002399420DD314BFA8
:102AB0000023012307FA05F494422CBF002403F0FD
:102AC00001045B46002C3FF4CCAE0BF1FF33002435
:102AD000C7E69B4612E78346E1E70C46BBE71A468A
:102AE00062E700BF000000000000000000000000DE
:102AF0002DE9F04F064683B00D461446074688463A
:102B0000002B51D18A4264D9B2FA82F35BB1C3F18E
:102B1000200801FA03F520FA08F802FA03F448EA5B
:102B2000050800FA03F7250C404629461FFA84FAE7
:102B300000F05EF929468146404600F087FA3B0CDA
:102B40000AFB09F043EA014188420AD9091909F14F
:102B5000FF3205D2884284BFA9F10209091900D8C1
:102B60009146C0EB010829464046BFB200F040F94B
:102B700029460646404600F069FA0AFB06FA47EA8B
:102B800001418A4509D90C1906F1FF3380F01981FA
:102B9000A24588BF023E40F2148146EA0940002661
:102BA000314603B0BDE8F08F8B4284BF002630462B
:102BB000F6D8B3FA83F4002C5AD18B4228BFB24224
:102BC0008CBF002601269CBF01202646E8D930464E
:102BD000E6E722B91146012000F00AF90446B4FAEA
:102BE00084F3002B40F0A2802D1B4FEA14481FFAFB
:102BF00084FA01264146284600F0FAF8414681460B
:102C0000284600F023FA3B0C0AFB09F043EA014195
:102C100088420BD9091909F1FF3280F0D48088422B
:102C200084BFA9F10209091940F2CD80C0EB010B64
:102C300041465846BFB200F0DBF8414605465846CB
:102C400000F004FA0AFB05FA47EA01418A4509D96E
:102C50000C1905F1FF3380F0B880A24588BF023D12
:102C600040F2B38045EA0940314603B0BDE8F08F39
:102C7000C4F12001A34022FA01F825FA01F748EA3D
:102C80000308384626FA01F3A5404FEA1849A24046
:102C9000494601921D4300F0ABF849468346384649
:102CA00000F0D4F91FFA88F22F0C02FB0BF047EA70
:102CB0000147B84206D917EB08070BF1FF31C0F006
:102CC0008D808B463F1A49463846009200F090F8B6
:102CD0004946ADB28246384600F0B8F9009A02FB88
:102CE0000AF245EA01418A4205D911EB08010AF1CD
:102CF000FF306CD38246019D4AEA0B40891AA0FB43
:102D0000052399420CD306FA04F614BF00210121D1
:102D100096422CBF002601F00106002E3FF440AF82
:102D200000260138314603B0BDE8F08F9C40C3F166
:102D3000200925FA09FA06FA03F74FEA1448504623
:102D400041469D4000F054F8414626FA09F949EA07
:102D500005098346504600F079F91FFA84FA4FEAD4
:102D600019430AFB0BF043EA0141884209D90919CA
:102D70000BF1FF333AD2884284BFABF1020B091941
:102D800034D90D1A414628461FFA89F900F030F867
:102D900041460646284600F059F90AFB06F549EA7D
:102DA00001418D4209D9091906F1FF3304D28D4240
:102DB00084BF023E091900D81E464D1B46EA0B4649
:102DC00018E71E46E9E6914630E71D464AE78A4283
:102DD00084BFAAF1020A41448DD88BE7B84284BF70
:102DE000ABF1020B47443FF66DAF6AE79B46C8E77D
:102DF0004A1E08BF7047C0F02481884240F2168105
:102E0000114200F01781B0FA80F3B1FA81F2A2EB1F
:102E10000303C3F11F0304A202EB03134FF00002EC
:102E20009F4600BFAFF30080B0EBC17F00BF42EB15
:102E3000020228BFA0EBC170B0EB817F00BF42EB64
:102E4000020228BFA0EB8170B0EB417F00BF42EBD4
:102E5000020228BFA0EB4170B0EB017F00BF42EB44
:102E6000020228BFA0EB0170B0EBC16F00BF42EBC4
:102E7000020228BFA0EBC160B0EB816F00BF42EB44
:102E8000020228BFA0EB8160B0EB416F00BF42EBB4
:102E9000020228BFA0EB4160B0EB016F00BF42EB24
:102EA000020228BFA0EB0160B0EBC15F00BF42EBA4
:102EB000020228BFA0EBC150B0EB815F00BF42EB24
:102EC000020228BFA0EB8150B0EB415F00BF42EB94
:102ED000020228BFA0EB4150B0EB015F00BF42EB04
:102EE000020228BFA0EB0150B0EBC14F00BF42EB84
:102EF000020228BFA0EBC140B0EB814F00BF42EB04
:102F0000020228BFA0EB8140B0EB414F00BF42EB73
:102F1000020228BFA0EB4140B0EB014F00BF42EBE3
:102F2000020228BFA0EB0140B0EBC13F00BF42EB63
:102F3000020228BFA0EBC130B0EB813F00BF42EBE3
:102F4000020228BFA0EB8130B0EB413F00BF42EB53
:102F5000020228BFA0EB4130B0EB013F00BF42EBC3
:102F6000020228BFA0EB0130B0EBC12F00BF42EB43
:102F7000020228BFA0EBC120B0EB812F00BF42EBC3
:102F8000020228BFA0EB8120B0EB412F00BF42EB33
:102F9000020228BFA0EB4120B0EB012F00BF42EBA3
:102FA000020228BFA0EB0120B0EBC11F00BF42EB23
:102FB000020228BFA0EBC110B0EB811F00BF42EBA3
:102FC000020228BFA0EB8110B0EB411F00BF42EB13
:102FD000020228BFA0EB4110B0EB011F00BF42EB83
:102FE000020228BFA0EB0110B0EBC10F00BF42EB03
:102FF000020228BFA0EBC100B0EB810F00BF42EB83
:10300000020228BFA0EB8100B0EB410F00BF42EBF2
:10301000020228BFA0EB4100B0EB010F00BF42EB62
:10302000020228BFA0EB0100104670470CBF012030
:1030300000207047B1FA81F2C2F11F0220FA02F0BB
:10304000704708B14FF0FF30FFF77ABB0029F8D086
:103050002DE90340FFF7CCFEBDE8064002FB00F37C
:10306000A1EB0301704700BF00000000000000005A
:1030700041F20463C2F200031868704700000000C8
:103080000F2AF0B445D940EA01039B0745D1A2F1CC
:1030900010070C4603463F0900EB0716103625685B
:1030A0001033103443F8105C54F80C5C43F80C5C9B
:1030B00054F8085C43F8085C54F8045C43F8045C7A
:1030C000B342ECD17B1C02F00F0CBCF1030F4FEAB2
:1030D00003131944034422D90E461D46644656F88C
:1030E000047B043C032C45F8047BF8D8ACF10404C1
:1030F00002F0030224F0030404342344214432B1D7
:103100000A4411F8014B914203F8014BF9D1F0BC8C
:1031100070470346002AF3D1F9E70346F0E7624619
:10312000002AEDD1F3E700BF00000000000000001E
:103130008307F0B448D0541E002A43D0CDB20346D2
:1031400002E0002C3ED0144603F8015B13F0030F9D
:1031500004F1FF32F5D1032C2DD9CDB20F2C45EA65
:10316000052545EA054518D9A4F1100703F1100615
:103170001A463F0906EB07161560103242F80C5C40
:1031800042F8085C42F8045CB242F5D104F00F0446
:103190000137032C03EB07130DD91E462246043AD0
:1031A00046F8045B032AFAD8221F04F0030422F035
:1031B0000302043213442CB1C9B21C4403F8011BAE
:1031C000A342FBD1F0BC704714460346C3E700BFDF
:1031D000C9B2F0B4002947D084070FD00278002A82
:1031E0003FD091423ED0431C05E013F8012B002A4A
:1031F00037D0914236D09A071846F6D141EA0127D6
:10320000036847EA0747A3F1013483EA070224EA87
:103210000303A2F1013424EA0202134313F0803FB6
:1032200011D1021D104652F8043B83EA0704A3F1B2
:103230000136A4F1013526EA030325EA04042343F9
:1032400013F0803FEED00378002B3BD0994209D099
:10325000431C01E0914205D0184613F8012B002AC7
:10326000F8D11046F0BC704781070DD00378002BD1
:10327000F8D0431C02E00278002AF3D013F0030FC9
:10328000184603F10103F6D10368A3F1013222EAE3
:10329000030313F0803F0AD1031D184653F8042B93
:1032A000A2F1013121EA020212F0803FF5D0037849
:1032B000002BD7D0431C184601330278002AFAD1DC
:1032C000F0BC70471846CDE7000000000000000089
:1032D00080EA0102844612F0030F4FD111F0030F70
:1032E00032D14DF8044D11F0040F51F8043B0BD0CE
:1032F000A3F101329A4312F0803F04BF4CF8043B23
:1033000051F8043B16D100BF51F8044BA3F1013230
:103310009A4312F0803FA4F101320BD14CF8043BE8
:10332000A24312F0803F04BF51F8043B4CF8044B19
:10333000EAD023460CF8013B13F0FF0F4FEA33238A
:10334000F8D15DF8044B704711F0010F06D011F869
:10335000012B0CF8012B002A08BF704711F0020F57
:10336000BFD031F8022B12F0FF0F16BF2CF8022B42
:103370008CF8002012F47F4FB3D1704711F8012B65
:103380000CF8012B002AF9D1704700BF00000000A3
:1033900020F0030110F00300C0F1000051F8043BDD
:1033A00000F1040C4FEACC0C6FF000021CBF22FAB3
:1033B0000CF213434FF0010C4CEA0C2C4CEA0C4C71
:1033C000A3EB0C0222EA030212EACC1204BF51F86A
:1033D000043B0430F4D013F0FF0F1FBF013013F48F
:1033E0007F4F013013F47F0F18BF0130704700BFCB
:1033F000F0B4002A4BD040EA010313F003032DD1AF
:10340000032A2BD904680D68AC4227D1043A3ED078
:10341000A4F1013525EA040414F0803F3DD10C46A7
:1034200005460EE06B68054666680C46A3F1013759
:10343000B34227EA030711D1043A28D017F0803F9E
:1034400028D1032A00F1040001F10401EAD8561E34
:103450002AB928792279801AF0BC7047561E037861
:103460000A7893421BD1E6B1BBB101368B1C0446EE
:10347000314405E08B4203F101030BD00028EBD06F
:1034800014F8010F13F8012C9042F3D0E3E7104633
:10349000F0BC70470020F0BC70471846DCE71846C7
:1034A000D9E73046D8E700BF000000000000000068
:1034B00040EA01039B0770B42BD1032A84BF0B465B
:1034C000054626D9194653F8044BA4F1013626EADD
:1034D000040616F0803F05D1043A45F8044B032A50
:1034E0001946EFD89AB10C78013A6B1C2C703CB19C
:1034F0006AB111F8014F013A03F8014B002CF7D1E2
:103500002AB11A44002103F8011B9342FBD170BC7D
:1035100070470546E6E700BF00000000000000001D
:1035200038B502460C46002511B909E0421C054693
:1035300010462146FFF74CFE0028F7D1284638BD3B
:10354000BDE83840FFF744BE000000000000000066
:103550004FF0010C2DE9F003644600254FF0FF36D3
:10356000631987198B420DD23F5D10F80380B8456F
:103570002FD21D460124C6EB030C63198B4200EBCE
:103580000607F1D34FF0010900254C464FF0FF37F5
:10359000C2F800C0631900EB070C99420ED91CF861
:1035A00004C010F80380E0451AD91D460124C7EB7A
:1035B00003096319994200EB070CF0D80137013673
:1035C000B74226BFC2F8009038463046BDE8F00347
:1035D00070470CD04FF0010C2E4664466544BFE79F
:1035E0000CD04FF001092F464C464D44D2E76445BC
:1035F00004F10104B4D11D460124B1E74C4504F1A6
:103600000104C7D11D460124C4E700BF2DE9F04FD6
:10361000ADF2244D164680460D461046194607AABF
:103620001C46FFF795FF07AB0DF21C42039043F8D1
:10363000044F9342FBD1671E002308A834B1F25C0B
:10364000F91A0133A34240F82210F8D10799304605
:10365000039A314400F04CFA002840F08180DDF8F4
:103660000CC02A468246671E0CF1FF3CCDF808C00C
:10367000B444CDF810C0DDF80CC005460196CCF17D
:10368000010CCDF814C008E025B1079A934238BF69
:10369000C2EB04039A44002532460AEB040608EB09
:1036A00002000021B21A00F0DBF9002853D1002EED
:1036B00051D008EB060308A913F8013C51F8233058
:1036C000002BE1D1039A954228BF2A46BA4212D272
:1036D000019908EB0A03985C11F802C01144844573
:1036E00006D032E011F8010F13F802C084452CD146
:1036F0000132BA42F6D3039B02989D4228BF184676
:103700001CD2DDF810C008EB0A039CF80010DDF8AD
:1037100008C013F80C20914240F08680DDF804B018
:10372000049AAB4406E012F8019D13F801C0E1458C
:1037300004D108465A4500F1FF31F4D101358542E4
:1037400074D8079DAA44651BA6E7DDF814C00025C0
:10375000E2449244A0E700200DF2244DBDE8F08F32
:10376000DDF80CC02A46DDF80CA04FF0000BCCEBC6
:1037700004030DF12009634538BF6346671E01331A
:10378000254607930CF1FF33B444CDF808C0DDF8AB
:103790000CC00193CCF1010CCDF810C00BEB05046B
:1037A00008EB02000021A21A00F05AF90028D2D139
:1037B000002CD0D008EB040313F8013C59F8233057
:1037C00053BBBA4508EB0B0013D2029B1A7810F8D2
:1037D0000A309A4218BF534621D1029A534605E057
:1037E00012F8011F10F803C08C4518D10133BB42F9
:1037F000F6D3019B5A1CAFD0DDF804C016F80C10AC
:1038000010F80C20914206D113F1FF33A4D3F15CE0
:10381000C25C9142F8D0079B9B442246BEE7DDF88C
:1038200010C0E3449B44F8E7039887E708EB0A00DD
:1038300092E700BF2DE9F04F8046037887B00E462F
:10384000002B00F001810A789AB1844601310124ED
:1038500002E011F8012B5AB1934214BF002404F086
:1038600001041CF8013F0D46002BF2D12B7813BB4D
:103870001CB1404607B0BDE8F08F08F10100317877
:10388000FFF7A6FCAD1B012D18BF0028074608BF97
:103890000046EFD0A844474594BFC7EB0804012475
:1038A0001F2D0CD93846214632462B46FFF7AEFE77
:1038B00007B0BDE8F08F002007B0BDE8F08F2946C3
:1038C00005AA3046FFF744FE0599314400900246B0
:1038D000304600F00DF9002857D1009B8346804602
:1038E0002246013B019333440293009BC3F1010341
:1038F000039308EB0504B8180021A21A00F0B0F8F1
:103900000028D8D1002CD6D0009B9B4528BF5B4611
:103910009D4214D9F918F05CF21811F80810884289
:1039200040F08C8007EB080C06E012F8011F1CF831
:103930000300884240F0828001339D42F5D8009B0D
:1039400001995B4540F28380029B07EB08091A78D6
:1039500019F801309A427AD1029B06EB0B0A06E075
:1039600013F801CD19F80200844504D111465345DE
:1039700001F1FF32F4D10BF1010B8B4569D8059BA6
:103980009844C3EB050B2246B3E700984FF0000BB9
:1039900022462B1A8146834238BF0346B144013385
:1039A0000593009B38440190C3F101030293009BEF
:1039B00003F1FF389A460BEB0504B8180021A21A50
:1039C00000F04EF800287FF476AF002C3FF473AF80
:1039D000554598BF07EB0B0014D9019899F80020C2
:1039E00010F80B309A4224D14A46534607EB0B009D
:1039F00005E012F8011F10F803C08C451AD10133FD
:103A00009D42F6D8B8F1FF3F43463FF433AF16F876
:103A1000081010F80820914207D113F1FF33FFF48A
:103A200029AFF15CC25C9142F7D0059B9B442246D2
:103A3000C1E75346029A93449B44F8E703994FF039
:103A4000000B884498449EE70D4601240EE7009938
:103A500091E707EB08000DE7000000000000000000
:103A60008307C9B270B43FD0541E2AB303788B4287
:103A700023D0431C04E0FCB1057814468D421CD0D1
:103A800013F0030F184604F1FF3203F10103F2D1E2
:103A9000032C14D8651E4CB303788B420DD0421C06
:103AA000002302E004788C4207D0AB42104603F1B9
:103AB000010302F10102F5D1002070BC704741EA18
:103AC0000126034646EA0646184604330268724059
:103AD000A2F1013525EA020212F0803FDAD1043C5E
:103AE0001846032CF0D8D5E71446D1E72046E4E782
:103AF000032A70B412D940EA01039B070FD10C4688
:103B0000034621461846043404330D680668AE4265
:103B100004D1043A1846032A2146F2D8C2B10578E6
:103B20000C78A54204BF02F1FF32002306D00CE05E
:103B300010F8015F11F8014FA54206D1934203F13D
:103B40000103F5D1002070BC7047281B70BC704782
:103B50001046F8E700000000000000000000000030
:103B6000704700BFAFF30080AFF30080AFF3008079
:103B7000FEE700BFAFF30080AFF30080AFF300803B
:103B800072B641F20060C2F2000080F309884EF67E
:103B90003472CEF200024EF68853CEF200034FF09C
:103BA000404111601A6842F470021A600023E1EE8D
:103BB000103A4EF63C73CEF2000300221A60062340
:103BC00083F31488BFF36F8F40F2000341F20002C9
:103BD000C2F20003C2F2000293420BD2D943114455
:103BE00021F0030119444FF05532043B43F8042FF0
:103BF0008B42FBD141F20003C2F2000383420CD29C
:103C000037491A1D891A21F0030119444FF0553222
:103C1000043B43F8042F8B42FBD107F069FF41F2CC
:103C2000006141F63C13C2F20001C2F20003994266
:103C30000ED2CC431C4424F0030442F2002004348E
:103C4000C0F603000023C258CA500433A342FAD17D
:103C500041F6401349F61842C2F20003C2F20102D3
:103C600093420AD2D943114421F00301194400229E
:103C7000043B43F8042F8B42FBD1FFF771FF40F266
:103C8000AC1540F24823C0F60005C0F600039D4283
:103C90000BD2EE431E44B6080136043D0024013425
:103CA00055F8043F9847B442F9D1FDF731FA40F294
:103CB000482540F24823C0F60005C0F600039D42A7
:103CC0000BD2EE431E44B6080136043D00240134F5
:103CD00055F8043F9847B442F9D1FFF749FF00BFB8
:103CE00003160020AFF30080AFF30080AFF3008035
:103CF000FEE700BFAFF30080AFF30080AFF30080BA
:103D000072B6FEE7AFF30080AFF30080AFF3008040
:103D100000F0CEF900F06CFC00F0EAF900DF00BF23
:103D20004EF63073CEF200035A6822F001025A6058
:103D3000EFF30983683383F30988002383F3118841
:103D4000704700BFAFF30080AFF30080AFF3008097
:103D500008B54FF46D43CEF200034FF44072C0F249
:103D6000FA52002199600720DA60102100F0E0F893
:103D70000A20202100F0DCF80B206021BDE808407B
:103D800000F0D6B8AFF30080AFF30080AFF300804F
:103D9000202383F311884FF46D43CEF200035B6858
:103DA00013F4006328D0F1EE10FAEFF309834EF616
:103DB0003072CEF200024FF08071D26843F84C1C92
:103DC00043F8082CA3F1680282F3098840F2985264
:103DD000C1F200029169887F88B110688A688168A1
:103DE000914294BF0022012292B143F61152C0F6D3
:103DF000000243F8502C704783F311887047106815
:103E00008A688168914234BF00220122002AECD1E5
:103E100043F61C52C0F6000243F8502C704700BF16
:103E200008B500F0CDF9202383F3118800F080F964
:103E300000F0E6F800F09CF9002383F3118800F00D
:103E4000EFF9BDE80840FFF7A3BF00BFAFF3008064
:103E50002DE9F04F2DED108AC1F80CD0D0F80CD020
:103E6000BDEC108ABDE8F08FAFF30080AFF30080A7
:103E700008B500F03DF9002383F311882846A047D8
:103E800000F09EFC08BD00BFAFF30080AFF30080E0
:103E900020F0030303F1604303F56143F0B400F045
:103EA00003024409D3F80053D200FF26A400964031
:103EB00004F1604404F5614425EA060501279140B8
:103EC00000F01F0007FA00F045EA0102C3F80023E2
:103ED000C4F880012060F0BC704700BFAFF30080E1
:103EE00041094FF4614230B4203100F01F04012534
:103EF000CEF2000220F0030305FA04F403F160435C
:103F000042F8214003F5614300F00300D3F8002399
:103F1000C000FF2101FA00F022EA0000C3F800030C
:103F200030BC7047AFF30080AFF30080AFF3008088
:103F300020F0030303F1604303F56D4300F0030039
:103F400010B4C0009A69FF24844022EA0402814030
:103F50000A439A615DF8044B704700BFAFF30080DD
:103F600040F29852C1F2000247F640639269C0F6EF
:103F700002039361FEE700BFAFF30080AFF3008060
:103F800010B582B0FFF7E4FE00F022FA00F0B0F9BD
:103F900000F0CEFF01F01CF840F200004021C1F219
:103FA000000000F035FB40F298530122C1F20003FB
:103FB0000277986100F05CF8002383F3118862B601
:103FC00040F29853C1F2000347F6B0729C69C0F604
:103FD0000202002140F2480043F66173A261C0F67C
:103FE0000003009101224FF4AA61C1F2000000F029
:103FF00087FB02B010BD00BFAFF30080AFF30080BD
:10400000F8B500F035F940F29853C1F200039B690E
:104010009A7F0AB1013A9A7740F2B453C1F2000391
:10402000DA681C6801329C42DA601DD0A768013F43
:10403000A760CFB91E462268E568E76053601A6042
:1040400000F096F8002383F311882069A847202305
:1040500083F3118800F06CF83468A26840F2B4531E
:10406000C1F20003002AE6D0F8BD00BFAFF3008024
:1040700041F64013C2F200031B682BB941F644130A
:10408000C2F200031B685BB147F6806047F65861D7
:10409000C0F60200C0F602014FF48C721DF028BC7D
:1040A000704700BFAFF30080AFF30080AFF3008034
:1040B00041F64013C2F2000310B51B6841F64414E8
:1040C000C2F200040BB923685BB147F6886047F67B
:1040D0005861C0F60200C0F602014FF48C721DF068
:1040E00007FC0123236010BDAFF30080AFF3008015
:1040F00041F64013C2F2000310B51B6841F64414A8
:10410000C2F200042BB92368002B02DD00232360D8
:1041100010BD47F6A46047F65861C0F60200C0F62D
:1041200002014FF48C721DF0E3FB0023236010BDED
:1041300041F64013C2F2000310B51B6841F6441467
:10414000002BC2F2000401DD23685BB147F6AC60CE
:1041500047F65861C0F60200C0F602014FF48C72B7
:104160001DF0C6FB0123236010BD00BFAFF300802C
:1041700041F64013C2F2000310B51B6841F6441427
:10418000002BC2F2000405DD2368002B02DD0023B2
:10419000236010BD47F6CC6047F65861C0F60200B8
:1041A000C0F602014FF48C721DF0A2FB00232360C5
:1041B00010BD00BFAFF30080AFF30080AFF300800D
:1041C00010B5202383F3118841F64014C2F2000495
:1041D0002268002A05DB41F64413C2F200031B6883
:1041E00063B147F6D46047F658614FF48C72C0F65D
:1041F0000200C0F602011DF07BFB226847F68473C3
:10420000C2F200030132196822608A42C8BF1A60F4
:10421000002383F3118810BDAFF30080AFF300805B
:1042200010B5202383F3118841F64014C2F2000434
:104230002268002A05DD41F64413C2F200031B6820
:1042400063B147F6DC6047F658614FF48C72C0F6F4
:104250000200C0F602011DF04BFB2268013A226009
:10426000002383F3118810BDAFF30080AFF300800B
:1042700041F64013C2F200031B68002B07DB41F636
:104280004413C2F200031B68002B00DD704747F6A1
:10429000E46047F65861C0F60200C0F602014FF430
:1042A0008C721DF025BB00BFAFF30080AFF3008020
:1042B00041F64013C2F200031B683BB941F64413B8
:1042C000C2F200031B68002B00DD704747F6087040
:1042D00047F65861C0F60200C0F602014FF48C7236
:1042E0001DF006BBAFF30080AFF30080AFF300809A
:1042F00040F2B453C1F200034FF0FF3100225B6083
:104300001B609960DA607047AFF30080AFF3008004
:10431000F8B5054616460C461F46FFF7A9FF002EC6
:1043200018BF002D1CD0DCB140F2B451C1F2000125
:104330002F610B68EE609A68944204D91B68A41A36
:104340009A68A242FAD35A682B606A608B425D6019
:104350001560AC601EBF9A68C4EB02049C60F8BD97
:1043600047F6107047F62071C0F60200C0F6020151
:1043700051221DF0BDFAD7E7AFF30080AFF3008004
:1043800010B50446FFF774FF8CB1236840F2B452B5
:10439000C1F2000293421FBF9968A26852189A6046
:1043A00062681360236800215A60E16010BD47F61F
:1043B000407047F62071C0F60200C0F602016D227F
:1043C0001DF096FAE1E700BFAFF30080AFF3008085
:1043D00040F29853C1F2000300225B601B605B61F6
:1043E0001B619A60704700BFAFF30080AFF300809D
:1043F00010B50446FFF73CFF00232377A16840F285
:104400009853C1F200031B689A688A42FBD25A682B
:104410002360626020465C60146010BDAFF30080D2
:1044200038B50446202383F31188FFF781FE257FEA
:10443000032D0ED00D2D10D0ADB14FF0FF33236200
:104440002046FFF7D5FFFFF793FE002383F3118883
:1044500038BD236A9A6801329A6094E80C001A60A9
:1044600022685360E9E7FFF783FE2B4683F3118848
:1044700038BD00BFAFF30080AFF30080AFF3008022
:1044800070B50546FFF714FF40F29853C1F20003E0
:1044900014261A68996914680D7701258E77636070
:1044A00015771C601046BDE870409A61FFF7D0BCDC
:1044B00070B50D4686B00646FFF7FAFE6B1C18D0A5
:1044C00040F29854C1F2000444F22142A369294603
:1044D00001A8C0F60002FFF71BFF3046FFF7D0FF30
:1044E000049B13B101A8FFF74BFFA369186A06B03C
:1044F00070BD40F29854C1F200043046FFF7C0FF8F
:10450000A369186A06B070BDAFF30080AFF30080F6
:1045100070B540F29855C1F2000504460E46FFF70B
:10452000C7FEA869A3688268266293420AD9FFF78A
:104530005FFF012323770146AC612046BDE8704050
:10454000FFF786BC2046BDE87040FFF751BF00BFB3
:1045500070B540F29854C1F2000414212368A56993
:104560001A680126546028461E77A9772260A36145
:10457000FFF73EFF2946A069BDE87040FFF768BC21
:1045800040F29852C1F2000270B410689569036855
:10459000AC681360012600215A60067703469061DB
:1045A000297700E01B689A68A242FBD85A682B6002
:1045B0006A6029465D60156070BCFFF749BC00BFAA
:1045C00008B5FFF775FE40F29853C1F200031A6870
:1045D0009B6992689B689A4200D808BDBDE8084074
:1045E000FFF7CEBFAFF30080AFF30080AFF30080E2
:1045F00040F29853C1F200039B699B7F0BB1FFF718
:10460000BFBFFFF7A5BF00BFAFF30080AFF30080CF
:10461000F0B440F29852C1F2000200245569447788
:1046200000F1240614274FF0020C456102618160FD
:1046300087774463046384618163506180F81CC0A0
:10464000286186624662F0BC704700BFAFF300800D
:104650002DE9F04799460E4604461746FFF708FE37
:10466000B6F5A87F2CBF00230123002C08BF43F020
:10467000010343B9D9F1010338BF00237F2F88BF5D
:1046800043F0010353B147F6507047F66471C0F62A
:104690000200C0F60201A6221DF02AF940F2985548
:1046A000C1F20005A6F164012144089B6A69E1603A
:1046B00043F671600026C0F600004FF0020A4FF08A
:1046C000140C0866C1F840904B6404F1240884F887
:1046D0001CA0667784F81EC0A76025616261A7638D
:1046E0006C6166632663A66120461461C4F8288065
:1046F000C4F82480BDE8F087AFF30080AFF30080FA
:104700002DE9F04182B01D4680460F461646089CB2
:10471000202383F31188FFF7CBFC2B46324600940D
:1047200039464046FFF794FF00210446FFF7F0FEAC
:10473000FFF7DEFC002383F31188204602B0BDE8BA
:10474000F08100BFAFF30080AFF30080AFF30080D3
:1047500010B5044658B947F6A07047F66471C0F624
:104760000200C0F602014FF493721DF0C1F820233D
:1047700083F31188FFF79CFC21460620FFF798FE83
:10478000FFF7B6FC002383F3118810BDAFF3008060
:1047900040F29853C1F200039B695A7F1862920756
:1047A00001BF5A69196911611B694FF00E0008BFFA
:1047B0005A61FFF765BE00BFAFF30080AFF3008022
:1047C00010B52023044683F31188FFF771FC2046BF
:1047D000BDE81040FFF7DCBFAFF30080AFF300800F
:1047E00038B5D0F1010338BF002353EAD173044632
:1047F0000D460AD047F6D07047F6E071C0F60200C9
:10480000C0F6020158221DF073F864602460A560B0
:1048100038BD00BFAFF30080AFF30080AFF300807E
:1048200038B504460D46FFF743FDC4B1A268531ED8
:10483000002BA36001DB002038BDE5B140F29853A6
:10484000C1F2000329469B691C6262681C605A60C1
:10485000032063601360BDE83840FFF729BE48F2CB
:10486000200047F6E071C0F60200C0F60201FD220A
:104870001DF03EF8DAE7A2604FF0FF3038BD00BF10
:1048800010B50446FFF7F4FC84B1A3680133002B94
:10489000A36000DD10BD23681A6800212260546007
:1048A00019621846BDE81040FFF7A2BD48F2480063
:1048B00047F6E071C0F60200C0F602014FF49972AB
:1048C0001DF016F8E1E700BFAFF30080AFF3008002
:1048D00010B5044620B1002364602460A36010BDBD
:1048E00048F2800048F29001C0F60200C0F60201D2
:1048F00058221CF0FDFFEEE7AFF30080AFF300801D
:10490000F8B540F29853C1F2000305469C69FFF7E1
:10491000CFFC002D45D0A86800283DD0A168836851
:1049200099421DD9037F8160002B2DD0042B17D114
:1049300003684268066A1360076833467A6002E0DB
:104940009A688A4202D31B689E42F9D15A68036072
:10495000426058601060B068A16883688B42E1D300
:104960002B4603E09968A268914202D31B689D42DE
:10497000F8D15A68236062605C601460256204208C
:10498000BDE8F840FFF77CBD90E80C001A600268B3
:104990005360FFF72DFDE3E7636BAC60EB6065638D
:1049A000F8BD48F2B00048F29001C0F60200C0F62F
:1049B00002017D221CF09CFFADE700BFAFF3008039
:1049C00010B52023044683F31188FFF771FB2046BE
:1049D000FFF796FFFFF78CFB002383F3118810BDD0
:1049E00040F29852C1F2000270B52023966983F319
:1049F0001188FFF75DFB746B2568E368A54273635C
:104A00001ED0B16B4BB11A689A4203D092689142A2
:104A100038BF1146DB68002BF5D16A6B2B68B1609B
:104A20002846236000215C60A560E2606C63FFF7AC
:104A30006FFDFFF75DFB002383F31188204670BDF7
:104A40000023A360F5E700BFAFF30080AFF3008061
:104A5000002918BF0028F8B505460C4617460AD1AC
:104A600048F2E00048F2F801C0F60200C0F6020188
:104A700057221CF03DFF202383F31188FFF718FB1A
:104A800040F29853C1F200032A689B692260002615
:104A90002C606360A760E660FFF72AFB334683F370
:104AA0001188F8BDAFF30080AFF30080AFF3008052
:104AB00038B504460D46FFF7DBFBBCB1226B237F04
:104AC00045EA0201082B21630CD0092B00D038BD28
:104AD000236A19408B42FAD12046FFF789FC002354
:104AE000036238BD236A1942F6D138BD48F230104E
:104AF00048F2F801C0F60200C0F60201FE221CF0E6
:104B0000F7FEDBE7AFF30080AFF30080AFF3008088
:104B100070B505460E46FFF7ABFB65B12C68A542A4
:104B200008D0201D0BC83343E360FFF7C1FF2468A2
:104B3000A542F6D170BD48F2441048F2F801C0F623
:104B40000200C0F60201BC221CF0D2FEE6E700BF64
:104B500003460022C068DA60704700BFAFF30080F0
:104B600010B4024679B140F29853C1F200030D200F
:104B70009B691A62546883E81400536023605DF8EF
:104B8000044BFFF795BC4FF0FF305DF8044B7047C6
:104B900030B4029C406000250A44856004620261D2
:104BA000006041618161C160C36130BC704700BF7A
:104BB00038B50446FFF75CFB2068E3680022A0429A
:104BC0006361A260A3610AD06FF0010503682360EE
:104BD0005C60FFF70DFC05622068A042F6D138BD8D
:104BE00038B504460D46FFF743FB6369A269A16827
:104BF00093421BD05A1C01316261A1601D70626931
:104C000023699A420BD22068A0420DD0036823602A
:104C10005C60FFF7EDFB00230362184638BD206897
:104C2000E368A0426361F1D1002038BD0029E1D0E2
:104C30006FF0030038BD00BFAFF30080AFF300801A
:104C4000F8B504460E46202383F31188FFF730FAA7
:104C5000E36933B12046984703E0FFF781FF071E61
:104C600018DBA56820463146002DF6D0A2692169DF
:104C7000531C8B42A36105F1FF3528BFE368A56093
:104C8000177828BFA361FFF733FA002383F3118855
:104C90003846F8BDFFF72CFA2B4683F311883846C7
:104CA000F8BD00BFAFF30080AFF30080AFF300802A
:104CB0002DE9F047044615460F461E46D0F81C80E5
:104CC000002A3DD0202383F31188FFF7F1F907EB89
:104CD000050A4FF000090137B8F1000F05D0204652
:104CE000C04702E0FFF73CFF10BBA56820463146F5
:104CF000002DF7D0A369013D5A1CA261A5601B7865
:104D000007F8013C2369A2699A4224BFE368A361C2
:104D1000FFF7EEF9002383F31188574509F10109E4
:104D20000BD0202383F31188FFF7C2F90137D3E7B3
:104D3000FFF7DEF92B4683F311884846BDE8F0877C
:104D400048F2801048F29411C0F60200C0F6020149
:104D5000E7221CF0CDFDB5E7AFF30080AFF3008094
:104D600030B4029C40608D1805610462006082606E
:104D700041618161C160C36130BC7047AFF30080A5
:104D800038B50446FFF774FAE36822692068636166
:104D9000D21AA042A361A2600AD06FF00105036895
:104DA00023605C60FFF724FB05622068A042F6D117
:104DB00038BD00BFAFF30080AFF30080AFF30080D9
:104DC0002DE9F041202304468846164683F31188D6
:104DD000FFF76EF903E0FFF7C3FE071E1DDBA568B2
:104DE00020463146002DF6D06369013D5A1C6261B0
:104DF000A56083F80080236962699A4224BFE36852
:104E00006361E3690BB120469847FFF771F900230E
:104E100083F311880020BDE8F081FFF769F92B4684
:104E200083F311883846BDE8F08100BFAFF30080FE
:104E300038B50446FFF71CFAA3696269A0689A4274
:104E400016D021695A1C0130A060A2618A421D78E7
:104E50000BD22068A04206D0036823605C60FFF795
:104E6000C7FA00230362284638BDE368A361F0E770
:104E70000028E6D06FF0020038BD00BFAFF300801D
:104E80002DE9F84F044617460E469B46D0F81CA065
:104E9000002A3AD0202383F31188FFF709F94FF055
:104EA0000009A56806F1010820466A1EFDB1636984
:104EB000A2605A1C626132781A70236962699A4250
:104EC00024BFE3686361BAF1000F00D0D047FFF759
:104ED0000FF9002383F31188013F09F1010911D073
:104EE000202383F31188FFF7E3F84646D9E72046ED
:104EF0005946FFF735FE0028D3D0FFF7F9F82B46C7
:104F000083F311884846BDE8F88F48F2B81048F29C
:104F10009411C0F60200C0F6020140F29B121CF090
:104F2000E7FCB7E7AFF30080AFF30080AFF300809A
:104F30004CF2000140F2C45240F2C8530648C2F29B
:104F40000101C1F20002C1F2000321F0070120F0CB
:104F500007001160186070471F9C0120AFF30080AC
:104F600010B50446FFF784F940F2C85340F2C4522A
:104F7000C1F20003C1F2000219681268E01D20F0BE
:104F80000700521A90429DBF401818600846002042
:104F900010BD00BFAFF30080AFF30080AFF300801F
:104FA00010B52023044683F31188FFF781F82046CB
:104FB000FFF7D6FF0446FFF79BF8002383F3118821
:104FC000204610BDAFF30080AFF30080AFF3008048
:104FD00040F2D053C1F2000344F6A1720021C0F6A2
:104FE000000203F110001A609960D960FFF770BCED
:104FF000F8B540F2D056C1F20006002818BF0646A8
:10500000073106F1100021F0070506F10804FFF74B
:10501000D7FC03E05A68954211D91C462368002B3F
:10502000F8D1FFF7DDFC33681BB305F108009847A2
:10503000F8B10660456000F108042046F8BD05F1AE
:105040000801914208D91A6822601C4644F8086B8E
:10505000FFF7C6FC2046F8BD4FF6F870CFF6FF709C
:10506000401B5F180244186858507A6027605D60E2
:10507000EBE70024E1E700BFAFF30080AFF300806F
:1050800070B50546002846D055F8080C00F1080414
:105090001030FFF795FCA5F108012346A34204D088
:1050A0008B4202D31B68A342FAD11A681AB191420B
:1050B00001D31346F2E755F8040C45F8082C1960A3
:1050C00000F1080255F8086C8C18B44209D05A68EF
:1050D00002F108001844814211D0BDE87040FFF78A
:1050E0007FBC64688A582044083045F8040C45F8B1
:1050F000082C5A6802F1080018448142EDD155F895
:10510000040C55F8081C0244083283E80600BDE888
:105110007040FFF765BC48F2002048F2E011C0F68D
:105120000200C0F60201C6221CF0E2FBACE700BFA1
:10513000F0B4002B08BF0B4600F10B0700F10A0585
:10514000B1FBF2F602FB161101F13004392CC8BF95
:1051500001F13704E4B2B3FBF2F331462E4605F811
:105160000149002BECD1BA1B3346024401E013F88D
:10517000014F00F8014B9042F9D1F0BC704700BFDD
:105180002DE9F04717469846064600220023384688
:105190004146DDF82090FCF7EBFE60B12D2408F1CC
:1051A00000483846414606F8014B00220023FCF730
:1051B000DFFE0028F3D138464146FBF7B9FF00284F
:1051C0003CD0B9F1000F34D04CF6CD4ACCF6CC4AE5
:1051D000AAFB093A4FEADA0A41463846FCF7F0FEE4
:1051E000044621460A2230460023FFF7A1FF064667
:1051F0002E2306F8013B2046FCF7DCFB02460B465B
:1052000038464146FCF788FA044648460D46FCF706
:10521000C1FB02460B4620462946FCF731FCFCF751
:10522000CFFE534601460A223046BDE8F047FFF75D
:105230007FBF4FF00A0A4FF06409CDE74E23612289
:105240003370B3707270F01CBDE8F087AFF300806C
:105250002DE9F04F8DB00DF1190303930746039824
:105260000DF1180B48F21023CBEB0000C0F602033F
:105270000C461646059004932178631C51B12529EC
:105280000BD03A681C469268384690472178631CD8
:105290000029F4D10DB0BDE8F08F62782D2A03BF4C
:1052A000A278A31C4FF0010C4FF0000C2E2A18BF5F
:1052B000302A03BF5A7801334FF030084FF02008EE
:1052C0001C46002506E03378043605EB8505227878
:1052D00003EB4505A2F13003DBB2092B04F1010415
:1052E000F3D92A2AEFD02E2A4FF0000949D002F034
:1052F000DF034C2B03D123780BB101341A46A2F102
:105300004403342B00F2EE80DFE813F07A00EC0067
:10531000EC00EC00EC007A00EC00EC00EC00EC009F
:10532000EC007800EC00EC00EC00EC00EC00450038
:10533000EC00EC00EA00EC00EC00EC00EC00EC000F
:10534000EC00EC00EC00EC00EC00E0007A00EC007B
:10535000B100EC00EC007A00EC00EC00EC00EC009A
:10536000EC007800EC00EC00EC008E00EC00450056
:10537000EC00EC00EA003378043609EB890903EB12
:10538000490914F8012BA2F13003DBB2092BF4D93F
:105390002A2AF0D0ABE70A22316858460023FFF7EB
:1053A000C7FE0436DA46CBEB0009C9EB050525EA52
:1053B000E575BCF1000F0DD16D425DB19AF800109A
:1053C0002D2900F095803B6838469B6841469847F8
:1053D0000135F8D1B9F1000F05DD3B6851464A4669
:1053E0001B6838469847002D3FF446AF3B68384667
:1053F0009B6841469847013DF8D13DE70822CBE73D
:1054000031680029BFBF2D208DF8180049420DF1E9
:105410001900A8BF58460A220023FFF789FE043668
:10542000DA46CBEB0009C0E7D6F800A0049BBAF13E
:10543000000F08BF9A4647F6FF729AF8003004360C
:10544000B9F1000F08BF9146002B63D00AEB0902A7
:10545000D14601E0914558D099F8013009F1010990
:10546000002BF7D1CAEB09094FF020089DE707365A
:1054700026F00706D6E90001CDF808C0FCF7C8FD04
:1054800007EE900AF5EEC07AF1EE10FADDF808C0EA
:1054900044BFF1EE677A2D2317EE900A4ABF0DF153
:1054A000190ADA468DF81830CDF808C0FCF794FADE
:1054B000CDF8009002460B465046FFF761FE0836D5
:1054C000DA46CBEB0009DDF808C06EE73368DDF89B
:1054D00014908DF8183004364FF02008DA4664E74F
:1054E000102259E78DF81820DDF81490DA465CE7B1
:1054F000B8F1300F7FF467AF3B6838469B68984738
:105500000AF1010A09F1FF395DE7CAEB02094FF020
:1055100020084AE799464FF0200846E7AFF300809D
:10552000C36882689A421FBF4268D154C36801337E
:105530001ABFC36000206FF001007047AFF3008016
:105540000269C168914218BF416803461DBF885C6B
:1055500001321A616FF00100704700BFAFF30080A5
:1055600038B5044608462369E5686168ED1AAA4221
:1055700038BF154619442A46FDF782FD23692B449E
:105580002361284638BD00BFAFF30080AFF3008031
:1055900038B5C36885680446ED1A4068AA4238BF2A
:1055A000154618442A46FDF76BFDE3682B44E3607B
:1055B000284638BDAFF30080AFF30080AFF3008022
:1055C00030B448F22024C0F60204002504600561CE
:1055D00041608260C36030BC704700BFAFF30080A1
:1055E000002910B41CDD02464418002012F8011BEB
:1055F0000823484010F0800F4FEA40001CBF80F0A5
:105600002700C04303F1FF3314BF00F0FE00C0B217
:1056100013F0FF03EED1A242E8D15DF8044B7047CE
:105620000020FAE7AFF30080AFF30080AFF3008013
:1056300010B4A1B148F230240144C0F602044FF086
:10564000FF3310F8012B5A40D2B2884254F822207E
:1056500082EA1323F5D1D8435DF8044B704708461E
:10566000FAE700BFAFF30080AFF30080AFF3008034
:105670002DE9F04104461E468846174618F050FBB7
:10568000E368054613B12046FEF77AFE2046414600
:105690003A463346FEF73CFE0DB1BDE8F081BDE869
:1056A000F04118F065BB00BFAFF30080AFF300809E
:1056B00008B502F0CDFF49F2A020C0F6020004F0C8
:1056C000D7F800F045F800F0ABF800F099F900F0D9
:1056D000CFF900F03DFA00F04BFA00F071FF01F055
:1056E00007F801F085FA01F0FBFB00F019FD01F06D
:1056F0003FF900F09DFFBDE8084006F011BA00BF79
:105700004FF48053CEF2000310B45A681C46104484
:10571000824263680BD2984294BF002101219A42D1
:1057200088BF00210029F3D15DF8044B70479A42ED
:105730008CBF00210121984288BF41F0010100295E
:10574000E6D1F1E7AFF30080AFF30080AFF3008064
:1057500003F06EB8AFF30080AFF30080AFF30080CA
:1057600000230122027043608360C36003614361D0
:105770001830FFF7ADB800BFAFF30080AFF3008083
:1057800038B504460D4680B1202383F31188FEF717
:105790008FFC2046656003F07BF802232370FEF740
:1057A000A7FC002383F3118838BD48F2306048F22B
:1057B0004061C0F60200C0F6020171221CF098F8A8
:1057C000E2E700BFAFF30080AFF30080AFF30080EB
:1057D000F8B504460E4617461D46FEF749FD002E55
:1057E00018BF002C04D01FB1012D0CD0EB070AD537
:1057F00048F2686048F24061C0F60200C0F602015B
:10580000C3221CF075F80323A760E56026612370AE
:105810002046BDE8F84003F093B800BFAFF3008026
:1058200003F01EBEAFF30080AFF30080AFF3008043
:1058300038B5012300250446037045602946083029
:10584000FEF7CEFF294604F11400FEF7C9FF04F16C
:10585000200504F1240004F1280104F12C0204F1D4
:10586000300325626062A162E262236338BD00BF3B
:1058700038B504460D4610B3202383F31188FEF794
:1058800017FC2378022B06D106200121FEF710FE1B
:105890002378022BF8D0012B05D0FEF729FC00233A
:1058A00083F3118838BD2046656003F0F9FD0323BA
:1058B0002370FEF71DFC002383F3118838BD48F2E6
:1058C000E06048F2F061C0F60200C0F602016D220D
:1058D0001CF00EF8D0E700BFAFF30080AFF30080FC
:1058E0002DE9F043002A18BF002883B004469146F2
:1058F0000E46984620D003291ED8202383F3118812
:10590000FEF7D6FB04F108072578042D3146204622
:1059100002D003F025FED8B938464146FEF780FF95
:105920000028F1D00190FEF7E3FB002383F31188F8
:10593000019803B0BDE8F08348F2187048F2F061B6
:10594000C0F60200C0F60201AF221BF0D1FFD4E77F
:10595000204631464A4603F023FEFEF7C9FB0023EA
:1059600083F31188002003B0BDE8F083AFF300801B
:105970002DE9F043002A18BF002883B00446914661
:105980000E46984601D001290AD948F2287048F2FB
:10599000F061C0F60200C0F60201DC221BF0A8FF95
:1059A000202383F31188FEF783FB04F11407257885
:1059B000042D3146204602D003F032FE78B9384635
:1059C0004146FEF72DFF0028F1D00190FEF790FB35
:1059D000002383F31188019803B0BDE8F0832046CB
:1059E00031464A4603F03CFEFEF782FB002383F378
:1059F0001188002003B0BDE8F08300BFAFF3008042
:105A000003F096BEAFF30080AFF30080AFF30080E9
:105A10000122002302704360704700BFAFF3008093
:105A2000002918BF002838B504460D460AD148F2AF
:105A3000607048F27071C0F60200C0F60201622286
:105A40001BF056FF202383F31188FEF731FB20461D
:105A5000656003F0EDFE02232370FEF749FB00238F
:105A600083F3118838BD00BFAFF30080AFF300802F
:105A700005F0AEBAAFF30080AFF30080AFF3008063
:105A80000122002302704360704700BFAFF3008023
:105A9000002918BF002838B504460D460AD148F23F
:105AA000E07048F2F071C0F60200C0F60201602218
:105AB0001BF01EFF202383F31188FEF7F9FA20461E
:105AC000656005F095FA02232370FEF711FB0023B1
:105AD00083F3118838BD00BFAFF30080AFF30080BF
:105AE00038B504460D46FEF7C3FB3CB104232946F6
:105AF00023702046BDE8384005F0B2BA48F64800A9
:105B000048F2F071C0F60200C0F60201D2221BF08A
:105B1000EFFEEBE7AFF30080AFF30080AFF3008060
:105B200010B50446FEF7A4FB34B1022323702046CF
:105B3000BDE8104005F0A4BA48F6600048F2F071E4
:105B4000C0F60200C0F60201F2221BF0D1FEECE723
:105B500004F0F6B8AFF30080AFF30080AFF300803D
:105B600001220023027043600C30FEF7B1BE00BF7B
:105B700005F026BBAFF30080AFF30080AFF30080E9
:105B80000122002302704360704700BFAFF3008022
:105B9000002918BF002838B504460D460AD148F63A
:105BA000800048F69001C0F60200C0F602016022B3
:105BB0001BF09EFE202383F31188FEF779FA20461E
:105BC000656005F02DFB02232370FEF791FA002398
:105BD00083F3118838BD00BFAFF30080AFF30080BE
:105BE00010B5044678B1202383F31188FEF760FADC
:105BF000204605F0C5FB01232370FEF779FA002348
:105C000083F3118810BD48F6AC0048F69001C0F649
:105C10000200C0F6020174221BF06AFEE3E700BF37
:105C200010B5044678B1202383F31188FEF740FABB
:105C3000204605F0FDFB03232370FEF759FA0023ED
:105C400083F3118810BD48F6B80048F69001C0F6FD
:105C50000200C0F6020187221BF04AFEE3E700BF04
:105C600010B5044678B1202383F31188FEF720FA9B
:105C7000204605F00DFC02232370FEF739FA0023BD
:105C800083F3118810BD48F6C80048F69001C0F6AD
:105C90000200C0F6020199221BF02AFEE3E700BFD2
:105CA000002918BF002838B504460D460BD02379CB
:105CB000052B01BFA36A4FF40072002085E80C0099
:105CC00018BF012038BD48F6102048F62021C0F644
:105CD0000200C0F602014FF44F721BF009FEE6E726
:105CE00030B5054683B010242B680121186801AA3D
:105CF00001F0BEF89DF80430FF2B0FD0013CF3D12A
:105D000002E00120FEF724FD2B680121186801AA9A
:105D100001F0AEF89DF80430FF2BF2D103B030BD96
:105D200070B5154682B00C4606462C30FFF7D8FFFA
:105D30002A0C2B0A44F04001280E48F6F0048DF896
:105D400004508DF802208DF803308DF800108DF886
:105D500001006B46C0F6020401AD002201E013F819
:105D6000011F81EA4202AB42A25CF8D15200F36A01
:105D700042F001028DF8052018686A46062101F0FC
:105D80003FF802B070BD00BFAFF30080AFF30080FA
:105D900030B5054683B009242B680121186801AA93
:105DA00001F066F89DF80400FF2801D1013CF3D111
:105DB00003B030BDAFF30080AFF30080AFF30080DD
:105DC000F8B50446C06A0F46154600681E4600F046
:105DD0006FFF39462A462046FFF7A2FF04F12C0048
:105DE000FFF7D6FFE16A054632460868042101F054
:105DF0003FF8E36A186800F07BFF2846F8BD00BF53
:105E0000C36A70B504460E461868154600F050FF88
:105E10002A4631462046FFF783FF04F12C00FFF7A6
:105E2000B7FFE36A0546186800F062FF284670BDB8
:105E3000F0B5C36A85B005460C461868164600F0F2
:105E400037FF214628460022FFF76AFF05F12C00A4
:105E5000FFF79EFF42F2107410B131E0013C36D0E2
:105E6000EB6A012118686A4601F002F89DF80030DB
:105E7000FE2BF3D1EB6A102118686A4600F0F8FF98
:105E80006B4606F10C01321F58781F78DE789C783B
:105E9000000440EA0760304340EA042041F8040966
:105EA000914203F10403EFD1EB6A0221186800F07C
:105EB0003FFFEB6A186800F01BFF002005B0F0BD43
:105EC000EB6A186800F014FF012005B0F0BD012056
:105ED00005B0F0BDAFF30080AFF30080AFF30080FA
:105EE00070B5054682B0002800F08D80EB6A002274
:105EF000032493E803002C7185F8302000F088FE1D
:105F0000EB6A1021186800F013FF0A2402E00A204F
:105F1000FEF71EFC00210A462846FFF771FF012804
:105F20000AD0013CF3D1EB6A186800F099FE022315
:105F30002B71012002B070BD01AB284608214FF43F
:105F4000D572FFF73DFF052825D0642404E0013C0D
:105F5000E9D00A20FEF7FCFB284637210022FFF794
:105F60004FFF01280646F2D14FF4D572C4F2000269
:105F70002846292101ABFFF723FF0028E7D102467D
:105F800001AB28463A21FFF71BFF9DF804305B0662
:105F900048BF85F83060642405E0012BC3D1013C83
:105FA000C1D0FEF7D5FB284601210022FFF728FFCC
:105FB00003460A20002BF0D1EB6A1868996800F0BC
:105FC00027FE284610214FF40072FFF719FF002822
:105FD000A9D105F11804224628460921FFF728FF18
:105FE0000028A0D1204600F0C3FAA86200289AD069
:105FF00028460A2105F10802FFF71AFF002892D16E
:1060000005232B7196E748F6402048F62021C0F67C
:106010000200C0F6020140F2C3121BF069FC65E702
:1060200010B50368044682B0186800F041FE02E033
:106030000120FEF78DFB23680121186801AA00F0FA
:1060400017FF9DF80430FF2BF2D12368186800F089
:106050004FFE02B010BD00BFAFF30080AFF3008071
:1060600070B5044698B12579052D01D0012070BD89
:106070002646082256F82C3F22711868996800F0CD
:10608000C7FD3046FFF7CCFF2571002070BD48F6F4
:10609000502048F62021C0F60200C0F6020140F26E
:1060A0001E321BF025FCDEE7AFF30080AFF300806B
:1060B00038B5044638B3202383F31188FDF7F8FF81
:1060C0002379022B18D004232371FEF711F8002343
:1060D00083F31188254655F82C3F9968186800F01D
:1060E00097FD2846FFF79CFFE36A186800F0B8FDAB
:1060F00002232371002038BDFDF7FAFF002383F34C
:106100001188002038BD48F65C2048F62021C0F6F2
:106110000200C0F6020140F22D221BF0E9FBCAE7A3
:10612000704700BFAFF30080AFF30080AFF3008093
:1061300048F6F0130022C0F602030121036001714A
:10614000C26280F830207047AFF30080AFF3008068
:10615000002918BF002838B504460D460BD148F673
:10616000702048F62021C0F60200C0F6020140F27D
:1061700095121BF0BDFB0223E562237138BD00BF01
:1061800010B5044630B1E36A186800F069FD0123D8
:10619000237110BD48F6802048F62021C0F6020089
:1061A000C0F602014FF4D3721BF0A2FBEBE700BF75
:1061B00038B504460D4628B3E36A06221868996884
:1061C000227100F025FDE36A186800F071FD94F873
:1061D00030308BB12A4620461221FFF7A1FD04F191
:1061E0002C00FFF7D5FD30B1E36A186800F038FDE8
:1061F00005232371012038BD6A0220461221FFF7D2
:106200008FFDECE748F68C2048F62021C0F602000E
:10621000C0F602014FF414721BF06AFBCCE700BF1A
:10622000002918BF002870B506460D4620D03379E6
:10623000062B01D0012070BD42F2107401E0013C38
:1062400023D0F36A012118682A4600F011FE2B784A
:10625000FE2BF4D1F36A2A4618684FF4007100F05F
:1062600007FEF36A0221186800F062FD002070BD8D
:1062700048F6A82048F62021C0F60200C0F6020128
:106280004FF41E721BF034FBD1E7F36A186800F07C
:106290002FFDF36A186800F0E3FC05233371012039
:1062A00070BD00BFAFF30080AFF30080AFF300809C
:1062B00038B50446D0B12379062B01D0012038BD72
:1062C000254648F6503255F82C3FC0F602021868B1
:1062D000072100F095FD2846FFF75AFDE36A18688C
:1062E00000F006FD05232371002038BD48F6C020CC
:1062F00048F62021C0F60200C0F602014FF42772D2
:106300001BF0F6FAD7E700BFAFF30080AFF30080D1
:1063100070B514461D460646FFF74AFF58B915B931
:106320000BE0013D09D021463046FFF779FF04F527
:1063300000740028F5D0012070BD3046BDE87040E3
:10634000FFF7B6BFAFF30080AFF30080AFF300807C
:1063500038B504460D4628B3E36A072218689968E1
:10636000227100F055FCE36A186800F0A1FC94F873
:1063700030308BB12A4620461921FFF7D1FC04F1B9
:106380002C00FFF705FD30B1E36A186800F068FCE7
:1063900005232371012038BD6A0220461921FFF729
:1063A000BFFCECE748F6DC2048F62021C0F60200EE
:1063B000C0F6020140F2BA221BF09AFACCE700BF05
:1063C00030B5002918BF002883B004460D4606D01A
:1063D0002379072B18BF012012D003B030BD48F637
:1063E000F82048F62021C0F60200C0F6020140F273
:1063F000E1221BF07DFA2379072B18BF0120ECD195
:10640000E36A48F640321868C0F60202022100F042
:10641000F7FCE36A2A4618684FF4007100F0F0FCBC
:10642000E36A0221186800F083FCE36A012118681E
:1064300001AA00F01DFD9DF8043003F01F03052B99
:106440000CD0E36A186800F053FCE36A186800F0A7
:1064500007FC05230120237103B030BD04F12C009B
:10646000FFF73EFC0020B8E7AFF30080AFF30080F9
:1064700010B50446A8B12379072B01D0012010BD27
:10648000E36A48F6E0021868C0F60202022100F052
:10649000B7FCE36A186800F02BFC05232371002089
:1064A00010BD48F6103048F62021C0F60200C0F6B4
:1064B00002014FF441721BF01BFADCE7AFF30080DE
:1064C00070B514461D460646FFF742FF58B915B988
:1064D0000BE0013D09D021463046FFF771FF04F57E
:1064E00000740028F5D0012070BD3046BDE8704032
:1064F000FFF7BEBFAFF30080AFF30080AFF30080C3
:10650000914270B50D461446064615D38B1A1F2BC3
:1065100012D805F01F026309013201206D0900FA4B
:1065200002F2AB4202F1FF3204F01F0410D356F81E
:1065300023001040E04070BD48F6603048F67431EA
:10654000C0F60200C0F6020149221BF0D1F9E0E7D3
:1065500056F8250056F823101040C4F12003984047
:1065600021FA04F4204370BDAFF30080AFF3008044
:10657000C3689B0F70B504460AD0012B06D1452194
:106580003022FFF7BDFF0130800270BD002070BDDA
:1065900049213E22FFF7B4FF312106462F22204633
:1065A000FFF7AEFF5321054650222046FFF7A8FF14
:1065B0000136023506FA05F5093805FA00F070BD16
:1065C00005F016B8AFF30080AFF30080AFF30080A2
:1065D0000122002302704360704700BFAFF30080C8
:1065E000002918BF002838B504460D460AD148F6E0
:1065F000903048F6A031C0F60200C0F602016522D4
:106600001BF076F9202383F31188FDF751FDAB8849
:1066100065602381204605F00BF802232370FDF707
:1066200067FD002383F3118838BD00BFAFF30080FE
:1066300004F0E6B9AFF30080AFF30080AFF3008061
:1066400010B5044620B12046BDE8104004F020BA41
:1066500048F6004048F61041C0F60200C0F60201BC
:10666000BB221BF045F92046BDE8104004F010BAEB
:106670000C30FEF71DBB00BFAFF30080AFF300800E
:106680000C304FF0FF33FEF713BB00BFAFF30080B9
:106690003030FEF7F5BB00BFAFF30080AFF30080F2
:1066A00030304FF0FF33FEF7EBBB00BFAFF300809D
:1066B0000C30FEF7C5BA00BFAFF30080AFF3008027
:1066C0000C304FF0FF31FEF7BBBA00BFAFF30080D4
:1066D0003030FEF775BB00BFAFF30080AFF3008032
:1066E00030304FF0FF32FEF76BBB00BFAFF30080DE
:1066F00005F04EB9AFF30080AFF30080AFF3008038
:1067000070B548F6C043C0F60203044682B040F8B4
:10671000043B012600940B461546606004F15401C9
:1067200004F10C0026721022FEF732FA00942B4678
:1067300004F1300004F164011022FEF711FB02B0F5
:1067400070BD00BFAFF30080AFF30080AFF30080F7
:1067500038B504460D4680B1202383F31188FDF738
:10676000A7FC2046294605F04BF902232372FDF7CA
:10677000BFFC002383F3118838BD48F6604048F61B
:106780006C41C0F60200C0F60201A1221BF0B0F875
:10679000E2E700BFAFF30080AFF30080AFF300800B
:1067A00038B504460D46FDF763FDD4B163693BB1CE
:1067B000294604F10C00FEF713FA00280BDB38BD64
:1067C000201D0421FEF7A4F9294604F10C00FEF770
:1067D00007FA0028F3DA201D8021BDE83840FEF7D3
:1067E00097B948F6944048F66C41C0F60200C0F6EE
:1067F0000201D8221BF07CF8D8E700BFAFF300807D
:1068000070B5046AD4F854321A681178042900D09B
:1068100070BD217A0229FBD112891B7942FA03F358
:1068200013F00105F4D1216CE36BA26BC91A8E1A27
:10683000EED0FDF75DFC2B4683F31188D4F854228B
:1068400033461068117904F1300200F0D1FB2023A7
:1068500083F31188FDF72CFCD4F85432BDE8704066
:106860001868197900F0FCBBAFF30080AFF300802B
:10687000F8B5046AD4F8542213681978042900D0B2
:10688000F8BD217A0229FBD15279598903EB8203A1
:1068900041FA02F2DB6812F001075D8AF0D1E66985
:1068A000A2696369B61AF61AB542E9D8FDF720FC69
:1068B0003B4683F31188D4F85422B6FBF5F305FB6D
:1068C00003F31068517904F10C0200F081FB2023DE
:1068D00083F31188FDF7ECFBD4F85432186859792A
:1068E000BDE8F84000F094BBAFF30080AFF3008048
:1068F0000C30FEF7DDB900BFAFF30080AFF30080CE
:106900000C304FF0FF33FEF7D3B900BFAFF3008078
:106910003030FEF7B5BA00BFAFF30080AFF30080B0
:1069200030304FF0FF33FEF7ABBA00BFAFF300805B
:106930000C30FEF785B900BFAFF30080AFF30080E5
:106940000C304FF0FF31FEF77BB900BFAFF3008092
:106950003030FEF735BA00BFAFF30080AFF30080F0
:1069600030304FF0FF32FEF72BBA00BFAFF300809C
:10697000704700BFAFF30080AFF30080AFF300803B
:1069800010B5024648F61053C0F6020342F8043B25
:1069900082B00446012146F671030090C0F6000360
:1069A000426001724FF4807204F154010C30FEF722
:1069B000EFF846F60103009404F1300004F5AA71E3
:1069C000C0F600034FF48072FEF7CAF902B010BDA2
:1069D00070B50D4604460E68D0B1202383F31188AC
:1069E000FDF766FB2A7906EB8202022394616A793D
:1069F000093246F82240AA7906EB8206B461237276
:106A0000C4F85452FDF774FB002383F3118870BD62
:106A100048F6E04048F6F041C0F60200C0F6020138
:106A2000DA221AF065FFD8E7AFF30080AFF30080F9
:106A300070B5D0F8543200F10C06044630461D689B
:106A4000FEF7B6F804F13000FEF79AF9201D012197
:106A5000FEF75EF8D4F85432597905EB81032846E5
:106A6000DB6832465B8A00F0B3FAD4F85432284629
:106A70005979BDE8704000F0CBBA00BFAFF3008099
:106A800090F8443003F06003202B01D000207047C1
:106A900090F84530212B03D0222B0CD0202BF5D1A0
:106AA00041F2F863C2F20003072100228363C1634D
:106AB00002640120704700238363C36303640120E1
:106AC000704700BFAFF30080AFF30080AFF30080EA
:106AD000F8B500EB810306469C690D46CCB1202336
:106AE00083F31188FDF724FB0821201DFEF710F821
:106AF000216CE26BA36B8A1AD71A19D106EB8503B6
:106B0000DA6853695B682BB9FDF732FB002383F326
:106B10001188F8BD128A013A12EA0307F4D1FDF791
:106B200027FB3B4683F31188002304F1300207E082
:106B3000FDF71EFB002383F3118804F130023B466E
:106B40003046294600F054FA202383F31188FDF7DC
:106B5000EFFA3046294600F083FAD5E7AFF300801C
:106B600001F109032DE9F04150F823400D46064696
:106B7000CCB1202383F31188FDF7DAFA201D04211C
:106B8000FDF7C6FF06EB8503E169D868A269636972
:106B9000478A8A1AC3EB0208474506D9FDF7E8FA87
:106BA000002383F31188BDE8F081FDF7E1FA0023AB
:106BB00083F31188B8FBF7F307FB03F304F10C022E
:106BC0003046294600F004FA202383F31188FDF7AC
:106BD000AFFA3046294600F01BFADFE7AFF300803A
:106BE000704700BFAFF30080AFF30080AFF30080C9
:106BF00003F0F6BFAFF30080AFF30080AFF3008087
:106C0000002301220270436083600C30FDF760BEF8
:106C1000002918BF002838B504460D460AD148F6A9
:106C2000305048F64051C0F60200C0F602016D2215
:106C30001AF05EFE202383F31188FDF739FA20460F
:106C4000656004F025F802232370FDF751FA002354
:106C500083F3118838BD00BFAFF30080AFF300802D
:106C600010B5044690B1202383F31188FDF720FA74
:106C7000204604F0F5F8204604F0A2F80123237022
:106C8000FDF736FA002383F3118810BD48F65C50F7
:106C900048F64051C0F60200C0F6020183221AF005
:106CA00027FEE0E7AFF30080AFF30080AFF3008092
:106CB00010B5044668B1202383F31188FDF7F8F975
:106CC000204604F0BDF8FDF713FA002383F3118882
:106CD00010BD48F6685048F64051C0F60200C0F6B4
:106CE000020197221AF004FEE5E700BFAFF300802F
:106CF00010B5044668B1202383F31188FDF7D8F955
:106D0000204604F0ADF8FDF7F3F9002383F3118872
:106D100010BD48F6785048F64051C0F60200C0F663
:106D20000201A9221AF0E4FDE5E700BFAFF30080FD
:106D3000002918BF002838B504460D460BD148F687
:106D4000DC5048F64051C0F60200C0F602014FF494
:106D500095721AF0CDFD202383F31188FDF7A8F971
:106D6000032329462370204604F08AF840F2985302
:106D7000C1F2000302209B69A360FDF781FBFDF7D0
:106D8000B7F9002383F3118838BD00BFAFF300804B
:106D9000002918BF0028F8B504460D4617461E46C0
:106DA00003D0002A18BF002B0BD148F6F05048F64C
:106DB0004051C0F60200C0F602014FF4A5721AF06D
:106DC00097FD202383F31188FDF772F903202946EC
:106DD0003A4633462070204604F072F840F2985349
:106DE000C1F2000302209B69A360FDF749FBFDF798
:106DF0007FF9002383F31188F8BD00BFAFF3008053
:106E0000002918BF002870B504460D4616461BD051
:106E1000D2B1202383F31188FDF74AF903232946D1
:106E200032462370204604F06BF840F29853C1F2CA
:106E3000000302209B69A360FDF722FBFDF758F9D0
:106E4000002383F3118870BD48F6006048F6405176
:106E5000C0F60200C0F6020140F267121AF048FDC7
:106E6000D7E700BFAFF30080AFF30080AFF300803F
:106E7000002918BF002870B504460D4616461BD0E1
:106E8000D2B1202383F31188FDF712F90323294699
:106E900032462370204604F053F840F29853C1F272
:106EA000000302209B69A360FDF7EAFAFDF720F9D1
:106EB000002383F3118870BD48F60C6048F64051FA
:106EC000C0F60200C0F602014FF4C2721AF010FDC3
:106ED000D7E700BFAFF30080AFF30080AFF30080CF
:106EE00003F076B9AFF30080AFF30080AFF300801A
:106EF0000023012202704360C36183620362C362A4
:106F00004362036303814381704700BFAFF3008096
:106F1000002918BF002870B504460E4615D020235E
:106F200083F311880025FDF7C3F820466660E5600D
:106F300025616561A56103F063F902232370FDF704
:106F4000D7F82B4683F3118870BD48F6706048F679
:106F50008061C0F60200C0F6020140F20F121AF082
:106F6000C7FCDCE7AFF30080AFF30080AFF3008035
:106F700070B5054614460E46FDF77AF9002C18BF89
:106F8000002D14D0606918B100211422FCF7D0F84C
:106F9000A06918B100211422FCF7CAF805EB86039A
:106FA0002846DC603146BDE8704003F011BA48F66F
:106FB000A86048F68061C0F60200C0F6020140F207
:106FC00041121AF095FCDDE7AFF30080AFF30080CB
:106FD00070B400EB81040126E468A4690025E26036
:106FE00063602670A56070BC03F0E2BAAFF3008066
:106FF00070B400EB81040126E46864690025E26056
:1070000063602670A56070BC03F04ABBAFF30080DC
:1070100070B504460D46FDF72BF98CB1638943FA30
:1070200005F010F0010601D0012070BD0122AA4038
:10703000134320466381294603F07AFC304670BD35
:1070400048F6DC6048F68061C0F60200C0F6020136
:107050004FF4F4721AF04CFCE0E700BFAFF300808D
:1070600070B504460D46FDF703F98CB1238943FA48
:1070700005F010F0010601D0012070BD0122AA40E8
:10708000134320462381294603F062FC304670BD3D
:1070900048F6F46048F68061C0F60200C0F60201CE
:1070A00040F203221AF024FCE0E700BFAFF30080B7
:1070B000002202210170A0F84C2080F84E2080F8B8
:1070C0004F2002814281C26002614261826180F888
:1070D000342003F00DB900BFAFF30080AFF30080A0
:1070E00070B50023044680F8343000F1440203F008
:1070F0004FFA63689B68002B31D02046984770B3E5
:10710000E06B94F8443094F84B1094F84A2042EA2B
:10711000012282423CBFE263104613F0800FE36815
:1071200040F09180002871D15B69052284F83420F9
:1071300001461870D86058609860204603F0B0FA95
:10714000202383F31188FCF7F3FF00212046FFF78B
:1071500087FFFDF70DF8002383F3118870BD94F8C5
:10716000443013F0600611D02046002103F018FCD3
:107170002046002103F004FC63681B6813B120461D
:1071800005219847062384F8343070BD94F84550A3
:1071900003F07F0242EA0525B5F5407F00F0ED805F
:1071A00016DDB5F5C06F00F0D08063DDB5F5106F6A
:1071B00073D040F60242954200F0F280B5F5006FC0
:1071C000D2D104F14F0201202664A263E0639AE762
:1071D000022D00F0A18040F39680B5F5807F00F08D
:1071E0008280B5F5817FBFD194F84620002ABBD1BB
:1071F00094F8482012F00F014AD01206204600F100
:10720000FD8003F0DDFB94F8443041E09B69A56B01
:107210000022042184F834101146DD6058601A7091
:107220009A60204603F0C4F9202383F31188FCF709
:107230007FFF00212046FFF7EBFEFCF799FF0023BC
:1072400083F3118870BD58B15B69A56B00220121E1
:1072500084F834101146DD6058601A709A606CE74B
:107260009B69032284F8342001461870D860586066
:107270009860D6E740F20232954221D0B5F5A06F72
:107280007FF472AFB4F84420B2F5A06F00F0A48090
:107290000020A063E063206435E794F8462084F87A
:1072A0004F20002A40F08680032222706268126814
:1072B000002AEDD020460221904794F84430E7E7B9
:1072C00094F84620002A7FF44FAF94F8482012F03B
:1072D0000F01DDD01306204600F1958003F050FB2E
:1072E00094F84430D4E794F84620012A7FF43CAF68
:1072F000B4F84C20A66322F00202E663266430460E
:10730000A4F84C20FFE6002D47D104F14C020220E6
:107310002564A263E063F6E694F8481011F0800F4C
:10732000204601F00F0148D103F012F9012848D09E
:1073300002287FF419AF48F66063C0F60203A36326
:10734000E063266494F84430DDE6626894F849000E
:1073500094F84830556894F8471094F8462043EA6A
:1073600000232046A84700283FF4FEAE09C8266443
:10737000A363E06394F84430C5E694F84620012AFC
:107380007FF4F2AEB4F84C20A66342F00202E6634A
:1073900026643046A4F84C20B5E6012D7FF4E4AE17
:1073A00048F65062C0F6020202200021A263E063A8
:1073B0002164A8E60422227078E703F0D9F80128B6
:1073C000B6D148F64073C0F60203A363E5632664B2
:1073D000284694F8443096E694F84630204684F8DF
:1073E0004E3002F0E5FF63681B6813B120460121AF
:1073F00098470323237094F8443049E703F0F0FAE8
:1074000094F8443044E703F0CBFA94F844303FE773
:1074100038B590F83430022B044647D0052B3ED0C7
:10742000012B10D0002103F0BBFA2046002103F00D
:10743000A7FA63681B6813B1204605219847062305
:1074400084F8343038BD90F84B1090F84A30C26B55
:1074500043EA01239342C36805D9198AB2FBF1F5C7
:1074600001FB152222B39A690321002384F834100A
:10747000204619461370D3605360936003F098F868
:10748000202383F31188FCF753FE00212046FFF7E9
:10749000BFFDFCF76DFE002383F3118838BD036C3C
:1074A00003B19847002384F8343038BDC368DAE765
:1074B0005B6911461A70DA605A609A6003F0F0F85E
:1074C000202383F31188FCF733FE00212046FFF7C9
:1074D000C7FDFCF74DFE002383F31188022384F8D7
:1074E000343038BDAFF30080AFF30080AFF30080DD
:1074F00090F83430032B10B504462FD0042B11D054
:107500002046002103F04CFA2046002103F038FA0F
:1075100063681B6813B1204605219847062384F849
:10752000343010BDC3685A690521002380F8341037
:1075300019461370D3605360936003F0B1F82023B1
:1075400083F31188FCF7F4FD00212046FFF788FD46
:10755000FCF70EFE002383F3118810BDC3689B69FE
:107560009B68002BCCD1036C03B19847002384F8AF
:10757000343010BDAFF30080AFF30080AFF3008074
:10758000022909D003290CD049F20010C0F60200EC
:10759000012918BF0020704748F68070C0F602002D
:1075A0007047032A06D849F2D000C0F6020000EB6B
:1075B000C200704700207047AFF30080AFF3008037
:1075C000022910B504461FD1202383F31188FCF74C
:1075D000AFFD48F650722046C0F602020121FFF7C7
:1075E000C7FC48F69072C0F6020202212046FFF75F
:1075F000BFFC41F66010C2F20000FFF719FAFCF779
:10760000B7FD002383F3118810BD00BFAFF30080E6
:1076100038B541F66015C2F2000549F2F00428467B
:10762000C0F60204FFF7ACF921462846FFF7D0F96F
:107630002468236D9A6B22F400229A6340F2DC5096
:10764000FDF786F848F6C0712046C0F60201FFF744
:107650005FFC236D9A6B42F2285042F400229A6339
:10766000C2F200000021BDE83840FFF771B800BF4A
:1076700041F66013C2F20003D3F854321B68187845
:10768000031F584258417047AFF30080AFF30080AA
:1076900002464FF00060CAB1531EDBB2032B11D972
:1076A000042B08BF4FF4803206D0063AD2B2062A25
:1076B00094BF4FF40032002210441A46531EDBB22E
:1076C000032BEDD800F58040002BF6D1704700BFAA
:1076D0004FF47053C4F2020370B51A69002A0646CB
:1076E000C0F28D804FF47051C4F20201CA684FF4A9
:1076F0007053D403C4F20203F8D41A6922F48072DE
:107700001A611A6942F400721A611A6922F0780249
:107710001A61F00742BF1A6942F008021A61B10704
:1077200041BF4FF47053C4F202031A6942F01002D1
:1077300048BF1A61720741BF4FF47053C4F202038D
:107740001A6942F0200248BF1A61330741BF4FF463
:107750007053C4F202031A6942F0400248BF1A6132
:107760004FF47053C4F202031C461A6942F002023D
:107770001A611A6942F480321A61E3684FF4705159
:1077800013F48035C4F20201F7D10B6923F0020330
:107790000B610B6943F000430B613046FFF778FF44
:1077A000032E15D9042E27D0053EF6B2062E98BF1B
:1077B0004FF4003206D9002070BD043A032A00F1CC
:1077C000040008D901680131F7D06FF00A0070BDDC
:1077D0004FF48042F6E7002AEDD00178FF29F4D17A
:1077E0000244013A034603E013F8011FFF29ECD1DC
:1077F0009342F9D1002070BD4FF48032E2E740F2AD
:10780000231148F6AB12C4F26751CCF6EF5259601F
:107810005A601B69002BBFF665AF4FF0FF3070BD9B
:10782000F8B58C46074639B3002500E025466C1CA8
:10783000E4B22046FFF72CFFB8420646F6D92846A8
:10784000FFF746FFB8B9032D98BF4FF480430BD91B
:10785000042D08BF4FF4803306D06B1FDBB2062B1C
:1078600094BF4FF400330023634505D2BCEB030CF7
:1078700002D03746D8E7F8BD0020F8BDAFF300804E
:1078800008B5034608461946FBF7FAFB002008BD79
:107890004FF470532DE9F043C4F202030546186912
:1078A000002883B00F461646C0F297804FF47052FE
:1078B000C4F20202D3684FF47054D803C4F2020435
:1078C000F8D4236923F480732361236943F400739C
:1078D000236115F0030338D1032E40F28F80A6F107
:1078E000040C05F1040828464FEA9C0C4FF470552F
:1078F00008EB8C08391AC4F202052A690B5842F0C9
:1079000001022A6140F8043BEC684FF47053E20333
:10791000C4F20203F8D41C69404524F001041C6140
:10792000EBD10CF1010C07EB8C0706F00306002EDF
:1079300033D14FF47053C4F2020300201A6942F0AD
:1079400000421A6103B0BDE8F083C3EB050902A849
:10795000D9F80020C3F1040840F8042DB04528BF31
:10796000B046184442463946FBF78AFB2269019B20
:1079700042F001022261C9F80030E1684FF470530F
:10798000C903C4F20203F8D41A6922F00102454483
:107990004744C8EB06061A619EE7D8F8003002A8F3
:1079A000394640F8043D3246FBF76AFB4FF470510C
:1079B000C4F20201019B0A6942F001020A61C8F89F
:1079C0000030CA684FF47053D503C4F20203F8D4F0
:1079D0001A6922F001021A61ABE740F2231148F65E
:1079E000AB12C4F26751CCF6EF5259605A601B6972
:1079F000002BBFF65BAF4FF0FF30A3E7A84696E73A
:107A0000704700BFAFF30080AFF30080AFF300809A
:107A1000704700BFAFF30080AFF30080AFF300808A
:107A2000704700BFAFF30080AFF30080AFF300807A
:107A300041F6E033C2F2000300221A60704700BF33
:107A400070B441F6E034C2F200042568092D16DC5A
:107A5000002DD8BFAE000EDD636898420FD0211F05
:107A6000AE003144234604E09A68904203F10403D7
:107A700005D08B42F8D1264401357060256070BC7A
:107A8000704700BFAFF30080AFF30080AFF300801A
:107A900030B441F6E035C2F200052C68002C0DDD53
:107AA0006B68984224D02A46002304E091688842FB
:107AB00002F1040204D00133A342F7D130BC704775
:107AC000002BFBDBA3420BDA05EB8301E31A043145
:107AD0009B000022486804329A4241F8040BF9D115
:107AE000013C05EB840300222C605A6030BC7047D7
:107AF0000023E9E7AFF30080AFF30080AFF300802D
:107B000010B90846FFF7C4BF0846FFF799BF00BF8A
:107B100030B441F6E034C2F200042568002D05605F
:107B200008DDAD000023E218C11852680433AB42EF
:107B30004A60F8D130BC7047AFF30080AFF30080EB
:107B400041F6E033C2F2000318680028D4BF0020D9
:107B500001207047AFF30080AFF30080AFF30080E7
:107B6000002930B4054611DD4A1E0020920003466C
:107B7000EC5C392C94BF303C573C013394408B4231
:107B80002044A2F10402F3D130BC70470020FBE78F
:107B90002DE9F0432DED028B83B008EE900AF9F742
:107BA0001BFF6A46F9F7ECFA00230022C4F25903DE
:107BB00080468946DDE90001FAF78CF8FAF700FA09
:107BC00007EE100A9FED368AF8EEC77A064667EE92
:107BD000887A17EE900AF9F7FFFEF9F729FB64237C
:107BE00003FB06F607EE106AF8EEC77A044678EE55
:107BF000E78A0D46FDEEE88AF8EEE88A68EE888AA4
:107C000018EE900AF9F7E8FEF9F712FB0023064692
:107C10000F46404649460022C4F24E03F9F730FFB2
:107C20001DA3D3E90023F9F72BFFF9F701FB8046E9
:107C3000894630463946FAF7EBF9DFED1A7A07EE56
:107C4000100A87EE278A29462046FAF7E1F94946C5
:107C500007EE900A404638EE278AFAF7D9F9DFEDA9
:107C6000127A07EE100AC7EE277A78EE277A17EE17
:107C7000900AF9F7B1FEF9F7DBFA07A3D3E900237D
:107C8000FAF728F8FAF7C4F903B0BDEC028BBDE8A7
:107C9000F08300BFAFF300800000000080842E411D
:107CA000002474490000704200006145AFF3008079
:107CB0004E2970B504461DBFD4ED007AF1EE677A07
:107CC00017EE900A0068452B1CBFD2ED007AF1EE4A
:107CD000677A15460CBF166817EE906AFFF758FFD3
:107CE00020603046FFF754FF286070BDAFF300807E
:107CF00038B504460D46FBF74BFB2378B0F5807F83
:107D0000B4BF01464FF4807100222C2B10460BD0DB
:107D1000002902DC08E0884206D0AB5414F8013F89
:107D200001302C2B0246F6D10023AB5438BD00BFE6
:107D300070B50D46C0B02C21FBF74AFA2C2101305A
:107D4000FBF746FA0446461C30466946FFF7D0FF6B
:107D500063780BB940B070BD68461DF0D1FA2C2194
:107D600028603046FBF734FA034601305B784E2B2F
:107D700004D0532B02D02C2B02D1002385F84C3099
:107D80002C21FBF725FA441C69462046FFF7B0FF7B
:107D900068461DF0B5FA2C2168602046FBF718FAFA
:107DA000034601305B78452B04D0572B02D02C2B97
:107DB00002D1002385F84D302C21FBF709FA441C31
:107DC00069462046FFF794FF68461DF001FA2C2112
:107DD00068642046FBF7FCF9441C69462046FFF71F
:107DE00087FF68461DF0F4F92C21A8642046FBF7B4
:107DF000EFF92C210130FBF7EBF969460130FFF771
:107E000077FF68461DF07CFAE86040B070BD00BFA7
:107E10002DE9F0410C46CCB02C21FBF7D9F9451CDB
:107E20000CA92846FFF764FF0CA8FBF7B1FA052858
:107E300023D99DF830109DF832209DF834309DF8FC
:107E400031709DF833609DF835003039303A303B61
:107E50004FEA41084FEA420C4FEA430E08EBC101DA
:107E60000CEBC2020EEBC3033944324403443039F5
:107E7000303A303B03910292019328462C21FBF7C4
:107E8000A7F9451C28460CA9FFF732FF9DF83030B2
:107E9000562B04BF0023636470D004236364284618
:107EA0002C21FBF795F9451C0CA92846FFF720FF6C
:107EB0000CA81DF025FA2C2120602846FBF788F934
:107EC000034601305B784E2B5CD0532B5AD02C2BC1
:107ED00057D02C21FBF77CF9451C0CA92846FFF74D
:107EE00007FF0CA81DF00CFA2C2160602846FBF758
:107EF0006FF9034601305B78452B47D0572B45D0AF
:107F00002C2B42D02C21FBF763F9451C0CA92846E9
:107F1000FFF7EEFE0CA81DF0F3F92C21A060284617
:107F2000FBF756F9451C0CA92846FFF7E1FE0CA803
:107F30001DF0E6F92C2120612846FBF749F90CA930
:107F40000130FFF7D5FE0CA8FBF722FA052820D850
:107F500001AB5A69002A11DD1E46143409AF3546BB
:107F60000FCDBD4220606160A260E3602E4604F147
:107F70001004F4D107CE20606160A2604CB0BDE86F
:107F8000F081002384F84C30A3E7002384F84D30BF
:107F9000B8E79DF830009DF832109DF834309DF818
:107FA00031709DF833609DF83550303B30383039B2
:107FB0005A004FEA40084FEA410C02EBC30208EBBB
:107FC000C0000CEBC101384431442A443038303908
:107FD000343201AB049005910692BBE7AFF3008009
:107FE00010B52A210446FBF79BFA88B10221013023
:107FF000FFF7B6FD63782A2B04F102014FF000026F
:1080000004D05A4011F8013B2A2BFAD1824201D008
:10801000802010BD002010BDAFF30080AFF30080C2
:1080200010B50446FFF7DCFF48B949F21011C0F65D
:1080300002012046FBF7FEFB18B1022010BDC0B2C2
:1080400010BD49F218112046C0F60201FBF7F2FB01
:10805000003018BF012010BDAFF30080AFF30080E7
:1080600070B5044608460D46FFF7DAFF012884F88C
:10807000400010D002280DD128462146FFF758FEB7
:108080002046221D94F84C1094F84D30BDE8704005
:10809000FFF70EBE70BD28462146BDE87040FFF7D1
:1080A000B7BE00BFAFF30080AFF30080AFF3008036
:1080B00010B5FCF785F84FF4C042C4F2020241F655
:1080C0000C43C2F2000311681C6801F03D0191608D
:1080D0000CB15868A047FCF7A3F8BDE81040FBF7C7
:1080E00057BE00BFAFF30080AFF30080AFF3008056
:1080F00010B5FCF765F84FF4C042C4F2020241F635
:108100000C431168C2F20003890901F03D019C682B
:10811000880190600CB1D868A047FCF781F8BDE8F1
:108120001040FBF735BE00BFAFF30080AFF3008017
:1081300010B5FCF745F84FF4C042C4F2020241F614
:108140000C431168C2F20003090C01F03D011C69E7
:10815000080490600CB15869A047FCF761F8BDE8CD
:108160001040FBF715BE00BFAFF30080AFF30080F7
:1081700010B5FCF725F84FF4C042C4F2020241F6F4
:108180000C431168C2F20003890D01F03D019C69A6
:10819000880590600CB1D869A047FCF741F8BDE8AC
:1081A0001040FBF7F5BD00BFAFF30080AFF30080D8
:1081B00010B5FCF705F84FF4C042C4F2020241F6D4
:1081C0000C43C2F2000351681C6A01F03D01D1600A
:1081D0000CB1586AA047FCF723F8BDE81040FBF744
:1081E000D7BD00BFAFF30080AFF30080AFF30080D6
:1081F00010B5FBF7E5FF4FF4C042C4F2020241F6AE
:108200000C435168C2F20003890901F03D019C6AE8
:108210008801D0600CB1D86AA047FCF701F8BDE82E
:108220001040FBF7B5BD00BFAFF30080AFF3008097
:1082300010B5FBF7C5FF4FF4C042C4F2020241F68D
:108240000C435168C2F20003090C01F03D011C6BA4
:108250000804D0600CB1586BA047FBF7E1FFBDE804
:108260001040FBF795BD00BFAFF30080AFF3008077
:1082700010B5FBF7A5FF4FF4C042C4F2020241F66D
:108280000C435168C2F20003890D01F03D019C6B63
:108290008805D0600CB1D86BA047FBF7C1FFBDE8E3
:1082A0001040FBF775BD00BFAFF30080AFF3008057
:1082B00010B5FBF785FF4FF4C842C4F2020241F645
:1082C0000C43C2F2000311681C6C01F03D01916087
:1082D0000CB1586CA047FBF7A3FFBDE81040FBF7BB
:1082E00057BD00BFAFF30080AFF30080AFF3008055
:1082F00010B5FBF765FF4FF4C842C4F2020241F625
:108300000C431168C2F20003890901F03D019C6C25
:10831000880190600CB1D86CA047FBF781FFBDE8E5
:108320001040FBF735BD00BFAFF30080AFF3008016
:1083300010B5FBF745FF4FF4C842C4F2020241F604
:108340000C431168C2F20003090C01F03D011C6DE1
:10835000080490600CB1586DA047FBF761FFBDE8C1
:108360001040FBF715BD00BFAFF30080AFF30080F6
:1083700010B5FBF725FF4FF4C842C4F2020241F6E4
:108380000C431168C2F20003890D01F03D019C6DA0
:10839000880590600CB1D86DA047FBF741FFBDE8A0
:1083A0001040FBF7F5BC00BFAFF30080AFF30080D7
:1083B00010B5FBF705FF4FF4C842C4F2020241F6C4
:1083C0000C43C2F2000351681C6E01F03D01D16004
:1083D0000CB1586EA047FBF723FFBDE81040FBF738
:1083E000D7BC00BFAFF30080AFF30080AFF30080D5
:1083F00010B5FBF7E5FE4FF4C842C4F2020241F6A5
:108400000C435168C2F20003890901F03D019C6EE2
:108410008801D0600CB1D86EA047FBF701FFBDE822
:108420001040FBF7B5BC00BFAFF30080AFF3008096
:1084300010B5FBF7C5FE4FF4C842C4F2020241F684
:108440000C435168C2F20003090C01F03D011C6F9E
:108450000804D0600CB1586FA047FBF7E1FEBDE8FF
:108460001040FBF795BC00BFAFF30080AFF3008076
:1084700010B5FBF7A5FE4FF4C842C4F2020241F664
:108480000C435168C2F20003890D01F03D019C6F5D
:108490008805D0600CB1D86FA047FBF7C1FEBDE8DE
:1084A0001040FBF775BC00BFAFF30080AFF3008056
:1084B00041F68C43C2F2000330B4002149F280152A
:1084C00041F60C4419600A460B46C0F60205C2F29A
:1084D0000004E8580C33C02B0160A15002F10802DF
:1084E000F7D14FF4C0414FF4C842C4F20201C4F2C4
:1084F00002024FF0FF338B6030BCCB609360D360DF
:10850000704700BFAFF30080AFF30080AFF300808F
:108510002DE9F043064683B08946904600284ED0A8
:1085200041F68C44C2F20004777A2268012505FAEC
:1085300007F1114218BF28463ED141F60C4CC2F259
:10854000000C0A430CEBC70012F0FF0F4CF8378009
:1085500043601CBF4FF46053C4F20203226018BF93
:10856000196B34681CBF41F40011196312F47F4F7A
:108570001FBF4FF46053C4F202031A6B42F480022F
:1085800018BF1A63236823F01F032360236813F0C6
:108590000105FBD1327A73683D2191402122196097
:1085A000404625606261B8F1000F05D0B07A4FEA0D
:1085B0000911FBF76DFC284603B0BDE8F08349F2D2
:1085C000201049F23811C0F60200C0F6020140F254
:1085D000CF12019319F08CF9019BA1E7AFF3008052
:1085E00010B5044638B3A07AFBF77AFC41F68C4309
:1085F000C2F20003627A1968012000FA02F221EA4D
:10860000020212F0FF0F1A6001BF4FF46053C4F270
:108610000203196B21F4001108BF196312F47F4F94
:1086200001BF4FF46053C4F202031A6B22F48002BC
:1086300008BF1A6310BD49F2681049F23811C0F63C
:108640000200C0F6020140F2FB1219F051F9CAE72C
:108650004FF46053C4F20203F0B400224FF0FF3431
:1086600019691C611A6159695C615A611E6A4EF28E
:108670001001CEF2000166F0805649F23F054EF639
:10868000F0501E62CEF200001A62C0F20205072608
:108690005F6A5C625A624D608A600E60C4684FF423
:1086A0008051CEF2000144F08074C460086840F04C
:1086B00001000860186C4FF4E041C4F2000140F082
:1086C00080501864086840F480700860196F01F4E5
:1086D0004071B1F5007F1EBF4FF4803119671A67F2
:1086E0004FF46053C4F202031A6F120407D41A6FD6
:1086F00042F400721A671A6F42F400421A674FF48C
:10870000E043C4F20003F0BC5A6822F400725A60DD
:10871000FFF7CEBEAFF30080AFF30080AFF3008071
:108720004FF460514FF4E043C4F20201C4F200037D
:108730004FF080504FF4404208641A600B6843F0D9
:1087400001030B600A684FF460539007C4F2020300
:10875000F8D59A6822F003029A609A6819469A60DE
:108760008B684FF4605213F00C03C4F20202F7D18D
:10877000116801F0F90111609360136843F48033CC
:10878000136011684FF460538903C4F20203F8D5F3
:108790005A6F42F001025A6719464A6F4FF460530C
:1087A0009207C4F20203F8D545F20842C0F24072C3
:1087B0005A6019684FF4E04241F080711960C4F2C8
:1087C000000253685B04FCD54FF46051C4F202010F
:1087D0000A684FF460539001C4F20203F8D54FF4D5
:1087E0007052C4F202024FF41441C3F6080140F281
:1087F0000570996010609A6842F002029A6019460A
:108800008A6802F00C024FF46053082AC4F2020393
:10881000F6D15A6C42F480425A645A6E42F4804255
:108820005A667047AFF30080AFF30080AFF300806B
:1088300070B541F69045C2F20005284641F6C444A1
:10884000FCF78EFFC2F20004104E4FF4005242F6C5
:108850001643C4F20102C0F202032046AA622B634F
:10886000EE62FCF77DFF4FF4045242F61643183EC9
:10887000C4F20102C0F20223E662A2622363122064
:108880006021BDE87040FBF703BB00BF10920208F7
:108890000378012B10B5044600D010BD41F690437B
:1088A000C2F20003984216D041F6C443C2F200035C
:1088B000984229D04FF40C52C4F20102A36A5468C2
:1088C00004F44004002144F48034012054605960D1
:1088D0009960986010BD48F63132C0F6000206215A
:1088E0002346C06AFFF714FEE36A42F24C0219689D
:1088F0004FF46053C4F20102C4F202038A605A6C5E
:1089000042F480725A64D5E748F63132C0F600026C
:1089100006212346C06AFFF7FBFDE36A42F24C12D0
:1089200019684FF46053C4F20102C4F202038A6072
:108930005A6C42F400725A64BCE700BFAFF3008087
:108940000369026B19782DE9F003C56829B1012D7F
:1089500094BF42F4807242F48472C16A5E880968EE
:108960008468D3F80C80CC6006FB05F44C600A6088
:10897000D1F800909F69DE691D6A5C6AD3F814C063
:108980001B69826A49F00109C1F80090590044BF8F
:1089900023F0804121F0020148F0806046BF41F49D
:1089A000407143F4407343F440734FF0000840F4C7
:1089B000807046BF41F0030143F0030343F001031D
:1089C000C2F80080C2F80CC01761D6621563546308
:1089D0005060BDE8F00348BF91609360704700BFEE
:1089E000C16A0A68136823F01F0310B41360136888
:1089F00013F00103FBD10C7A826A48683D2101FA29
:108A000004F40121046053605DF8044B93609160AD
:108A1000704700BFAFF30080AFF30080AFF300807A
:108A200010B5FBF7CDFB4FF40053C4F20103002156
:108A30001A681960940608D541F69044C2F2000401
:108A4000E36A1B685B68002B41D14FF40453C4F206
:108A5000010300211A681960900632D541F6C4441A
:108A6000C2F20004E36A1B685B6853B3236943B333
:108A70002046FFF7B5FF23699B684BB105222270A2
:108A80002046012198472378052B04BF0223237039
:108A900000232361202383F31188FBF749FB41F670
:108AA000C443C2F20003586930B14FF0FF32026292
:108AB00000225A61FBF79CFCFBF75AFB002383F36F
:108AC0001188FBF7ADFBBDE81040FBF761B92369E6
:108AD000002BBAD02046FFF783FF23699B684BB178
:108AE000052222702046012198472378052B04BFD8
:108AF0000223237000232361202383F31188FBF7D3
:108B000017FB41F69043C2F20003586930B14FF0B1
:108B1000FF32026200225A61FBF76AFCFBF728FB76
:108B2000002383F3118890E7AFF30080AFF3008058
:108B300011F00C0F38B504461ED10369DBB18A066B
:108B400011D51D78002D3DD05D68A5B1C268012A00
:108B500085BF598883688168520884BF514303EBFD
:108B60004101A84738BDCD0605D55B681BB1C26879
:108B700081685208984738BDFFF732FF23699B6828
:108B80004BB1052222702046002198472378052BFF
:108B900004BF0223237000232361202383F3118861
:108BA000FBF7C6FA63693BB100214FF0FF32616108
:108BB00018461A62FBF71CFCFBF7DAFA002383F372
:108BC000118838BDFFF70CFF23695B68D3B104221D
:108BD00022702046A168E26898472378042B02BFE0
:108BE000022325612370202383F31188FBF7A0FA69
:108BF0006369002BE0D00022626118461A62FBF71D
:108C0000F7FBD9E7022223612270ECE7AFF3008083
:108C100008B5FBF7D5FA41F66850C2F200004FF4F0
:108C200070534268C4F20103012152685961002166
:108C30009047FBF7F5FABDE80840FBF7A9B800BF7D
:108C400008B5FBF7BDFA41F66850C2F200004FF4D8
:108C500070534268C4F201030221D26859610121B4
:108C60009047FBF7DDFABDE80840FBF791B800BF7D
:108C700008B5FBF7A5FA41F66850C2F200004FF4C0
:108C800070534268C4F20103042152695961022100
:108C90009047FBF7C5FABDE80840FBF779B800BF7D
:108CA00008B5FBF78DFA41F66850C2F200004FF4A8
:108CB00070534268C4F201030821D269596103214B
:108CC0009047FBF7ADFABDE80840FBF761B800BF7D
:108CD00008B5FBF775FA41F66850C2F200004FF490
:108CE00070534268C4F201031021526A5961042191
:108CF0009047FBF795FABDE80840FBF749B800BF7D
:108D000010B5FBF75DFA4FF47053C4F201035C69D0
:108D100004F478725A61A30634D4600628D421067C
:108D20001CD4E20510D4A30508D541F66853C2F25D
:108D3000000318465B680921DB6C9847FBF770FA63
:108D4000BDE81040FBF724B841F66853C2F20003B7
:108D500018465B6808215B6C9847E4E741F6685366
:108D6000C2F2000318465B680721DB6B9847D8E71F
:108D700041F66853C2F2000318465B6806215B6B3C
:108D80009847CCE741F66853C2F2000318465B6887
:108D90000521DB6A9847C0E7AFF30080AFF300809E
:108DA00010B5FBF70DFA4FF47053C4F201035C6980
:108DB00004F47C4261055A6140D4220534D4E304B2
:108DC00028D4A0041CD4610410D4220408D541F690
:108DD0006853C2F2000318465B680F21DB6F9847A7
:108DE000FBF71EFABDE81040FAF7D2BF41F6685310
:108DF000C2F2000318465B680E215B6F9847E4E7F8
:108E000041F66853C2F2000318465B680D21DB6E21
:108E10009847D8E741F66853C2F2000318465B68EA
:108E20000C215B6E9847CCE741F66853C2F2000311
:108E300018465B680B21DB6D9847C0E741F6685325
:108E4000C2F2000318465B680A215B6D9847B4E7DD
:108E500008B5FBF7B5F941F66850C2F200004FF4CF
:108E600070534268C4F201034FF48031D2F8842079
:108E7000596110219047FBF7D3F9BDE80840FAF794
:108E800087BF00BFAFF30080AFF30080AFF3008077
:108E900008B5FBF795F941F66850C2F200004FF4AF
:108EA00070534268C4F201034FF40031D2F88C20B1
:108EB000596111219047FBF7B3F9BDE80840FAF773
:108EC00067BF00BFAFF30080AFF30080AFF3008057
:108ED00008B5FBF775F941F66850C2F200004FF48F
:108EE00070534268C4F201034FF48021D2F89420F9
:108EF000596112219047FBF793F9BDE80840FAF752
:108F000047BF00BFAFF30080AFF30080AFF3008036
:108F100008B5FBF755F941F66850C2F200004FF46E
:108F200070534268C4F201034FF40021D2F89C2030
:108F3000596113219047FBF773F9BDE80840FAF730
:108F400027BF00BFAFF30080AFF30080AFF3008016
:108F500008B5FBF735F941F66850C2F200004FF44E
:108F600070534268C4F201034FF48011D2F8A42078
:108F7000596114219047FBF753F9BDE80840FAF70F
:108F800007BF00BFAFF30080AFF30080AFF30080F6
:108F900008B5FBF715F941F66850C2F200004FF42E
:108FA00070534268C4F201034FF48001D2F8B42038
:108FB000596116219047FBF733F9BDE80840FAF7ED
:108FC000E7BE00BFAFF30080AFF30080AFF30080D7
:108FD00008B506206021FAF75BFF07206021FAF749
:108FE00057FF08206021FAF753FF09206021FAF7A4
:108FF0004FFF0A206021FAF74BFF17206021FAF794
:1090000047FF28206021FAF743FF01206021FAF78B
:109010003FFF2920F021FAF73BFF2A206021FAF7D1
:1090200037FF3E206021FAF733FF4C206021FAF72A
:109030002FFF0220F021FAF72BFF0320F021BDE8DB
:109040000840FAF725BF00BFAFF30080AFF3008000
:109050004FF46053C4F20203F0B41C6C4FF4C845E3
:10906000C4F2000544F000741C64D5F800321B0CF7
:109070001B0443F0010343EA0023C5F80032002932
:1090800065D00020C5F81C020346C5F8040204465A
:10909000C5F80C02C5F81402D80000F1804000F5B4
:1090A000C84001331C2BC0F84042C0F84442F3D101
:1090B0004FF4C843C4F20003002501271079146857
:1090C00010F0010F18BFD3F804024FEAC40607FAE4
:1090D00004F41EBF2043C3F80402107910F0020FFD
:1090E0001FBFD3F80C022043C3F80C0210794007CD
:1090F00042BFD3F814022043C3F8140206F180469D
:10910000906806F5C8460135C6F84002D068C6F832
:109110004402D3F81C028D4244EA000402F110021A
:10912000C3F81C42CAD14FF4C842C4F200024FF443
:109130006053D2F80012C4F2020321F00101C2F818
:1091400000121A6C22F000721A64F0BC7047C3005F
:10915000012203F1804303F5C84302FA00F01043F3
:10916000C5F84012C5F84412C3F84012C3F84412BF
:10917000C5F80412C5F81412C5F80C02C5F81C0293
:10918000D1E700BFAFF30080AFF30080AFF3008002
:1091900038B5426B40F20113C0F2010393600446FC
:1091A000202383F31188FAF7C3FF2369002BB8BF8C
:1091B00004F1080505DA2846FBF762FB2369002B5A
:1091C000F9DB04F124000121FBF7A2FCFAF7D0FF40
:1091D000002383F3118838BDAFF30080AFF3008024
:1091E000436B70B5DE68B207044614D1F30611D59F
:1091F000636B1022DA60202383F31188FAF798FF5B
:1092000004F128001021FBF783FCFAF7B1FF0023DB
:1092100083F3118870BD5A6922F002025A6120233B
:1092200083F31188FAF784FFE369002BB8BF04F1D8
:10923000140505DA2846FBF723FBE369002BF9DB6D
:1092400004F120000121FBF763FCFAF791FF0023F2
:1092500083F31188CAE700BFAFF30080AFF300804B
:10926000436B70B51E690446B00714D1F10611D5E1
:10927000636B10221A61202383F31188FAF758FFD9
:1092800004F128001021FBF743FCFAF771FF0023DB
:1092900083F3118870BD5A6922F010025A612023AD
:1092A00083F31188FAF744FFE369002BB8BF04F198
:1092B000140505DA2846FBF7E3FAE369002BF9DB2E
:1092C00004F120000221FBF723FCFAF751FF0023F1
:1092D00083F31188CAE700BFAFF30080AFF30080CB
:1092E000426B70B555681C232E07044653601FD48B
:1092F0006D071CD5636B9D699A6905F0070622F01E
:10930000700215F0700F9A6118BF46F0080620230E
:1093100083F31188FAF70CFF04F1280046EA0541AF
:10932000FBF7F6FBFAF724FF002383F3118870BDE7
:109330001168064621F00201032306F8303B202382
:10934000116083F31188FAF7F3FE30460021FBF732
:10935000DFFBFAF70DFF002383F31188C8E700BF96
:1093600008B5FAF72DFF41F6F840C2F20000FFF70A
:109370000FFFFAF755FFBDE80840FAF709BD00BF37
:1093800008B5FAF71DFF41F6F840C2F20000FFF7FA
:1093900027FFFAF745FFBDE80840FAF7F9BC00BF20
:1093A00008B5FAF70DFF41F6F840C2F20000FFF7EA
:1093B00057FFFAF735FFBDE80840FAF7E9BC00BFF0
:1093C00008B5FAF7FDFE41F6F840C2F20000FFF7DB
:1093D00087FFFAF725FFBDE80840FAF7D9BC00BFC0
:1093E00008B5FAF7EDFE41F63050C2F20000FFF783
:1093F000CFFEFAF715FFBDE80840FAF7C9BC00BF79
:1094000008B5FAF7DDFE41F63050C2F20000FFF772
:10941000E7FEFAF705FFBDE80840FAF7B9BC00BF60
:1094200008B5FAF7CDFE41F63050C2F20000FFF762
:1094300017FFFAF7F5FEBDE80840FAF7A9BC00BF30
:1094400008B5FAF7BDFE41F63050C2F20000FFF752
:1094500047FFFAF7E5FEBDE80840FAF799BC00BF00
:1094600038B541F6F845C2F20005284641F63054B9
:10947000FCF7DEF9C2F200044FF4C843C4F2000363
:1094800020466B63FCF7D4F94FF4D043C4F20003D9
:10949000002163630A460E20BDE83840FFF7D8BDBF
:1094A00041F6F843C2F20003984210B5044620D0BA
:1094B00041F63053C2F20003984233D0636B02216D
:1094C000012221701A605A68D10707D406200121B1
:1094D000FAF7EEFF636B5A68D207F7D5616848F672
:1094E0005B7248680968D861C0F2010219605A616C
:1094F00010BD1320B021FAF7CBFC1420B021FAF7ED
:10950000C7FC1520B021FAF7C3FC1620B021FAF7EA
:10951000BFFC4FF46053C4F202031A6C42F00072B5
:109520001A64CBE73F20B021FAF7B2FC4020B0210B
:10953000FAF7AEFC4120B021FAF7AAFC4220B02194
:10954000FAF7A6FC4FF46053C4F202031A6C42F01F
:1095500080621A64B2E700BFAFF30080AFF300800F
:1095600003291AD8DFE801F0110C0702436B986851
:10957000C0F300707047436B9868C0F3C0607047D9
:10958000436B9868C0F380607047436B9B6813F02F
:10959000E05F0CBF0020012070470020704700BF33
:1095A00010B4032925D8DFE801F02F2B2702436BE5
:1095B00003F5D073117888064CBFC1F30010C1F3D6
:1095C000001001F00F0154BF9488546859609168ED
:1095D00048BF400099604CBF40EAC4006405D168B0
:1095E0004CBF40F0040044EA400040F00102D96062
:1095F0001A605DF8044B7047436B03F5C873D9E7F5
:10960000436B03F5C073D5E7416B8B68C3F301630C
:10961000183301EB0313CDE7AFF30080AFF3008005
:10962000012911D00AD3022906D1436B186910F021
:10963000030018BF0120704700207047436BDA68B1
:109640009207F3D001207047436BD86810F00300F5
:1096500018BF0120704700BFAFF30080AFF3008058
:1096600010B4002930D1436BD968890735D0D3F8BD
:10967000B041D3F8B411D3F8B831D360436BD3F809
:10968000BC311361436B2020D860D868800743D079
:109690001079C4F3400363F30410C4F3800363F34D
:1096A00045101071002B31D09368E40864F31C035B
:1096B000936013795DF8044B080A61F30303090C06
:1096C000137110705180704701292AD0022908BFF8
:1096D000436B05D05DF8044B704719698C07F9D0CE
:1096E000D3F8C041D3F8C411D3F8C831D360436B69
:1096F000D3F8CC311361436B2020186118698007BF
:1097000002BF586940F010005861C1E71389640D29
:1097100064F30A031381CCE7586940F002005861F2
:10972000B6E7436BA3E700BFAFF30080AFF3008061
:1097300041F66850C2F20000FCF76AB9AFF300804E
:109740000F29F0B429D9436853F83100C2073DD539
:109750004FF47054C4F201040122A5688A401543F5
:10976000A560D44310F0020F4FF47050C4F2010012
:1097700003EBC101C5684B6814BF15432540C560A4
:109780007BB34FF47053C4F2010319680A431A60A3
:109790005A6814405C60F0BC704721F003024368D3
:1097A00002F1804202F59C3253F83100976801F0D3
:1097B0000304A4000F25A540C0F3031627EA0505FE
:1097C00006FA04F42C439460C207C1D44FF47055D8
:1097D000C4F201050122AE688A40D4432640AE603F
:1097E000C0E74FF47053C4F2010359680A435A604A
:1097F0001A6814401C60F0BC704700BFAFF30080D3
:109800004FF47053C4F201030122186802FA01F107
:10981000CA4310401860586810405860986810405B
:109820009860D8680240DA6059617047AFF30080F1
:1098300038B50378012B054614D0002404E0013428
:10984000FFF77EFF172C0CD06B6853F8343013F001
:10985000040F21462846F2D10134FFF7D1FF172C1F
:10986000F2D138BDFFF7B4FBE7E700BFAFF30080EC
:109870004FF46053C4F202031A6B6FEA52226FEA8C
:1098800042221A631A6D6FEA52226FEA42221A6567
:1098900000234168C4F202034FF48062596081687A
:1098A0009960C168D960016959614169196281692A
:1098B000596201681960016AC4F202024FF4006340
:1098C0005160416A9160816AD160C16A5161016BE6
:1098D0001162416B5162C1691160C4F20203C16B34
:1098E0005960016C9960416CD960816C5961C16C9F
:1098F0001962016D5962816B4FF440621960816D8C
:10990000C4F202024FF480535160C16D9160016E48
:10991000D160416E5161816E1162C16E5162416DC3
:109920001160C4F20203416F5960816F9960C16F89
:10993000D960D0F880105961D0F884101962D0F83D
:1099400088105962016F4FF4A0521960D0F890103E
:10995000C4F202024FF4C0535160D0F894109160E9
:10996000D0F89810D160D0F89C105161D0F8A010B8
:109970001162D0F8A4105162D0F88C101160D0F8A8
:10998000AC10C4F202034FF4E0525960D0F8B010AA
:109990009960D0F8B410D960D0F8B8105961D0F8F7
:1099A000BC101962D0F8C0105962D0F8A810C4F2E7
:1099B00002021960D0F8C8305360D0F8CC30936000
:1099C000D0F8D030D360D0F8D4305361D0F8D8304C
:1099D0001362D0F8DC305362D0F8C4104FF4005357
:1099E0001160D0F8E420C4F202035A60D0F8E820F5
:1099F0009A60D0F8EC20DA60D0F8F0205A61D0F804
:109A0000F4201A62D0F8F8205A62D0F8E0201A60E8
:109A1000704700BFAFF30080AFF30080AFF300806A
:109A20002DE9F00F002302F00307C2F38006C2F312
:109A3000C105C2F341144FF00F09C2F3C3124FF036
:109A4000010A04E07600AD00A400BF00013303F07A
:109A5000070C4FEA8C0C11F0010F02FA0CF809FA0E
:109A60000CFC3CD0072B95BFD0F820B0D0F824B028
:109A70002BEA0C0C2BEA0C0C95BF4CEA08084CEABC
:109A80000808C0F82080C0F82480D0F804C00AFA82
:109A900003F82CEA080C4CEA060CC0F804C04FF09E
:109AA000030B4FEA430CD0F808800BFA0CFC6FEA6A
:109AB0000C0C0CEA080848EA0508C0F80880D0F841
:109AC0000C800CEA080848EA0408C0F80C80D0F8BA
:109AD00000800CEA080C4CEA070CC0F800C04908EA
:109AE000B0D1BDE8F00F7047AFF30080AFF3008056
:109AF00070B541F67055C2F20005FAF761FB6C6B68
:109B0000238BA68AB6B246EA0343082223F07F439A
:109B1000C0F2030293425ED027D80122C0F20302B2
:109B200093424CD00222C0F20302934213D1A38885
:109B3000EA6A23F400731B0412681B0CA3801368E9
:109B400043F001031360A3889BB243F48053A380C6
:109B50005368012B65D916F00A0F18BF238BFAF74B
:109B60005FFBBDE87040FAF713B98222C0F207022A
:109B7000934217D08422C0F207029342EBD1EB6AE2
:109B80001B685B6863B323882A8C9BB243F4A06391
:109B900042F001022A842380FAF742FBBDE87040BC
:109BA000FAF7F6B8A3882A6B23F400731B04126833
:109BB0001B0CA380136843F001031360CBE72B8CCD
:109BC0001A0A0BD003F0010343F0F00302F006027F
:109BD0001A432282BFE72B8CC3F347032382BAE7E1
:109BE000A38823F400731B041B0CA38023889BB25F
:109BF00043F400732380202383F31188FAF798FA43
:109C0000E86941F67053C2F2000320B100220262FB
:109C1000DA61FAF7EDFBFAF7ABFA002383F3118868
:109C200099E7238823F480631B041B0C238092E7AD
:109C3000F8B541F67054C2F20004636B9D8AADB270
:109C4000FAF7BEFA266B616B326805F45F4383F462
:109C50007F4383F0FF038B82136823F01F0313609D
:109C60001368DF07FCD4377AE06A736802683D2620
:109C7000BE401E60136823F01F0313601368DE07E5
:109C8000FCD4067A426805F480733D20B0409BB254
:109C9000106003B10123AA05A36044BF43F002038F
:109CA000A3606F050ED58A8822F400721204120C8C
:109CB0008A80088880B243F0040240F400730B806D
:109CC0001346A2602E0544BF43F00803A360680456
:109CD00044BF43F02003A360E90444BF43F01003F2
:109CE000A3602A0444BF43F04003A36006D42BB909
:109CF000FAF796FABDE8F840FAF74AB8202383F35A
:109D00001188FAF715FAE06941F67053C2F20003C0
:109D100030B16FF0010202620022DA61FAF768FBEB
:109D2000FAF726FA002383F31188FAF779FABDE8E7
:109D3000F840FAF72DB800BFAFF30080AFF3008012
:109D400010B541F67054C2F200042046FBF708FF3C
:109D5000064B4FF4A8420020C4F2000203F10C01AC
:109D6000E0616263E362216310BD00BFBC91020841
:109D70002DE9F04F40F29851C1F2000185B08A6997
:109D8000046D029149F25023C0F6020393618146AB
:109D9000202383F31188FAF78BF9C846A14698F877
:109DA0000030012B06D0D8F85C3083B9D9F81430D4
:109DB000DA060CD40299D9F818208B6942F0100207
:109DC000C9F818200220C8F86430FAF759FBFAF7EE
:109DD0008FF9002383F311884FF0000AD9F814306B
:109DE000DB0623D5D8F850703D6A05F4F013B3F5BF
:109DF000802F34D0B3F5402FF0D105F00F0208EBDF
:109E00008202C5F30A13D26803339B08106AE5D0B7
:109E100007F580570222396812B140F8041B013A55
:109E2000013BF8D1D9F81430DB06DBD4D8F85C302C
:109E3000012101FA0AF11942019108BF0AF1010B4F
:109E400040F08780D8F854309B685FFA8BFA9A45C7
:109E5000C4D9202383F31188FAF72AF99FE705F084
:109E60000F0608EB860BC5F30A15DBF80C30986972
:109E70000378E3B9021D1CCA0332D21AEB1C9B08FB
:109E80004FEA92021CBF07F58057A64606D03968F4
:109E900012B14EF8041B013A013BF8D12C44C460C6
:109EA000DBF80C309B699A682A449A6096E7C4688C
:109EB00007F580572846AE46002D2BD0032807D93A
:109EC00063692269934242D3E36803286361F7D848
:109ED0003E68F0B16369002200E06369D10026FAB0
:109EE00001F15D1C65611970636921698B4224BFB2
:109EF000E3686361013802F101020CBF0023012312
:109F0000032A8CBF002303F00103002BE5D10028B6
:109F1000D4D17546202383F31188FAF7C9F8A368D2
:109F200020682B44A042A36009D0036823605C60D2
:109F3000FAF75EFA002202622068A042F5D1FAF731
:109F40003FFBFAF7D5F8002383F31188A8E73E68B2
:109F5000C1E7202383F31188FAF7AAF8D9F808207B
:109F6000D8F85C30019922F0010223EA0103C9F814
:109F70000820C8F85C30FAF7BBF8002383F3118897
:109F800008EB8A020092D1684C69A36862689A4221
:109F900040F2D480D8F85000098A4FEA4A17C51910
:109FA000D21AD5F818398A4234BF15460D469BB2ED
:109FB000B5EB830F0AF1010B9EBF4FEA0B32CDF8D0
:109FC0000C9091462DD82378002B43D1EB1CD4F86C
:109FD0000CE09B08484418BF724604D052F8041B9A
:109FE000013B0160FAD10EEB0503E360009AD168F2
:109FF0004C69A36862682B449A42A36040F29A803D
:10A00000D8F85000098AC519D21AD5F818398A42E9
:10A0100034BF15460D469BB2B5EB830FD3D9DDF89F
:10A020000C900024202383F31188FAF741F8D9F823
:10A03000083043F00103C9F808302CB9D9F8343896
:10A0400001990B43C9F83438FAF752F8002383F327
:10A050001188F7E600EB090AE4682A46AE4615B314
:10A0600096083DD02569A169681AC31C30EA200012
:10A0700028BF184683109E4238BF33464FEA830CF0
:10A08000CCEB02023BB1084650F8046B013BCAF826
:10A090000060F9D16144A942A16148D3E368A3619A
:10A0A000002ADDD17546202383F31188FAF700F8E2
:10A0B000A36820682B44A042A36009D003682360F2
:10A0C0005C60FAF795F9002303622068A042F5D19D
:10A0D000FAF776FAFAF70CF8002383F3118885E78C
:10A0E0001646FAB12569A1690026334600E0A16948
:10A0F000481CA06191F800C0D9000CFA01F1A842F7
:10A1000046EA010624BFE168A161013A03F10103B7
:10A110000CBF00210121032B8CBF002101F00101A4
:10A120000029E4D1CAF80060002A99D1BAE7002AD0
:10A13000DAD1B7E7DDF80C90012473E70AF1010BDF
:10A14000FAE700BFAFF30080AFF30080AFF3008009
:10A15000D1F808C000212DE9F0010D464FF08048EC
:10A160004FF0FF3713E00319C3F81059C3F808790B
:10A17000D2F8006B002EA8BFC2F8005B18DB0444C5
:10A1800001316145C4F8105BC4F8087B18D84C0154
:10A190000219D2F80039002BA8BFC2F80059E2DA40
:10A1A000C2F800891646D6F808399B07FBD5DAE7CE
:10A1B000C2F8008B1A46D2F8083BDE06FBD5DEE774
:10A1C0004FF00113C0F81C38BDE8F001704700BF24
:10A1D00010B541F6A854C2F200042046FCF788FEF0
:10A1E00049F2402300224FF0A041C0F6020321654E
:10A1F00063652266626610BDAFF30080AFF3008036
:10A2000070B50378066D012B82B0054601D002B00F
:10A2100070BD41F6A853C2F20003984251D02B6E94
:10A220000022EA65002B3DD04FF4A2520323C0F276
:10A230002023C4F2000200204FF45021F260C6F83F
:10A240000038C6F8000EB1632C6D2020FBF758FAD9
:10A25000012323612369DA07FCD40C20FBF750FAB1
:10A260002369002BFCDA0024B460286D696DFFF7C8
:10A270006FFF6B68C6F81048DB68C6F81448C6F86C
:10A280001C485BB143F20803B3614FF0FF337361C5
:10A29000B36843F00103B36002B070BD4FF44053A4
:10A2A000B361F2E749F671530095C0F6000305F17A
:10A2B00068004FF4AA610222FAF7CAF968662866B4
:10A2C000B2E74FF46053C4F202030022596B41F02D
:10A2D00080015963596941F08001596143205A61F5
:10A2E000E021F9F7D5FD9AE7AFF30080AFF30080E6
:10A2F000F8B5046D202307462361226912F020057A
:10A30000FBD10C20FBF7FCF97B6D9E682A46FF21F0
:10A310004FF0006504EB42130132B242C3F800591A
:10A32000C3F8005BC3F80819C3F8081BF2D94FF053
:10A33000FF324FF00113C4F81828C4F81C387B6DA5
:10A340001A68BA651B6863623A6D1023136113695A
:10A3500013F01005FBD10C20FBF7D2F9D4F800382C
:10A3600023F4FE63C4F80038A06949F2602240F487
:10A37000402048F24003C1F200030921C0F6020266
:10A3800040F01000A061C4F81018C4F81418FA6066
:10A39000C4F8105BC4F8003BC4F81059C4F8003985
:10A3A000BB6D03F1100243F48013BA65A362F8BDDC
:10A3B000036D90F84E10D3F8002822F4FE6242EAB2
:10A3C0000112C3F800287047AFF30080AFF300809C
:10A3D0002DE9F0410FFA81F800EB88064FF40047B1
:10A3E000F368046D1A6802F00302022A0D4608BFE2
:10A3F000C1F208070CD0032A08BFC1F20C0707D02E
:10A400003946C1F20001C1F20407012A18BF0F4604
:10A410006A0104EB020ED9684FF0000CCEF810CBA5
:10A4200000294DD0B3F812E005F15801490147EA7F
:10A430000E0E44F801E04FF0010CD4F81C1805F1A1
:10A44000100E0CFA0EFE4EEA0101C4F81C1822444C
:10A4500099684FF0000EC2F810E900294CD09A8B91
:10A46000198A012A4FEA910388BF534305F13F013E
:10A47000826D04EB810103EB020E42EA0343C0F854
:10A4800058E04B60026DAB0143F020031361136988
:10A490009806FCD40C20FBF733F9F3681A8A05F10F
:10A4A000480342EA85525B011743E7500122D4F882
:10A4B0001C3802FA05F51D43C4F81C58BDE8F081AC
:10A4C00004EB481105F1100ED1F800CB2CF4004C30
:10A4D000C1F800CBD4F81C184FF0010C0CFA0EFE9A
:10A4E00021EA0E01C4F81C18224499684FF0000EAE
:10A4F000C2F810E90029B2D105F13F0204EB820253
:10A500004FF48063C0F200235360026DAB0143F04F
:10A510002003136113699906FCD404EB48180C203E
:10A52000FBF7EEF8D8F8003923F40043C8F80039F7
:10A53000D4F81C38012202FA05F523EA0503C4F811
:10A540001C38BDE8F08100BFAFF30080AFF300809E
:10A550005831036D49015B5813F4004004D013F4E3
:10A56000001F0CBF02200120704700BFAFF3008026
:10A570004831036D49015B5813F4004004D013F4D3
:10A58000001F0CBF02200120704700BFAFF3008006
:10A5900000EB8101CB681B6A19685B68116053602E
:10A5A000704700BFAFF30080AFF30080AFF30080CF
:10A5B00000EB810330B4DC68A2695368136141B9D0
:10A5C000402B06D940252B465560C6F200033F2597
:10A5D00002E05D1E43F0C043628A006DAC18B4FB1C
:10A5E000F2F200EB411143EAC243C1F8103B30BC28
:10A5F000704700BFAFF30080AFF30080AFF300807F
:10A60000F8B5076D07EB41130546D3F8084BC3F8BF
:10A61000084B23070E4603D5D7F814381A0719D468
:10A62000E30716D5D7F81438DC0712D505EB8603F7
:10A63000DA68936959681869814211D36989D368C6
:10A64000012000FA06F221EA02026A813146284618
:10A650009847F8BD00EB8103DB685B689847DFE74C
:10A66000411A002259609A6028463146FFF7A0FF40
:10A67000202383F31188F9F75BFD2B6D03EB46165E
:10A68000D6F8003B43F08063C6F8003BF9F770FD55
:10A69000002383F31188F8BDAFF30080AFF300808F
:10A6A00000EB810330B4DC68626953681361A3B1C5
:10A6B00069B15D1E228A006DAC18B4FBF2F200EBAA
:10A6C000411143EAC243C1F8103930BC7047402BF6
:10A6D000EFD9402353603F25ECE7036D03EB4111B5
:10A6E0004FF40023C1F8103930BC7047AFF300803D
:10A6F000F8B5056D05EB41130646D3F80849E207A6
:10A700000F46C3F8084903D5D5F81038DB0708D43D
:10A71000220605D50122D5F83438BA401A422ED186
:10A72000F8BD00EB8103DA685369D3F804E0D3F88D
:10A7300010C0E64540D2CEEB0C0E0022C3F804E078
:10A740009A60FFF7ADFF202383F31188F9F7F0FC3F
:10A75000336D03EB47120120D2F8001941F0044198
:10A76000C2F80019D3F8341800FA07F20A43C3F804
:10A770003428F9F7FDFC002383F31188C8E7202370
:10A7800083F31188F9F7D4FCF36DD5F83428706E93
:10A79000012101FA07F73B4322EA0707F365C5F8F1
:10A7A000347818B1F9F724FE00237366F9F7E0FC5A
:10A7B000002383F31188F8BDB0F808E093684FF0E8
:10A7C000010C0CFA01F22EEA0202028198479FE77F
:10A7D00070B541F6A856C2F20006F9F7F1FC356DE6
:10A7E0006B69AC691C40E3046C6138D4A00448BFB9
:10A7F000D5F80838210707D57368DB6823B141F61F
:10A80000A850C2F200009847E20633D46303D5F89B
:10A81000185807D5EE0763D4A8076AD4690771D41E
:10A820002A0778D4230307D5EE0346D4AC034DD4CE
:10A83000680338D4290305D4F9F7F2FCBDE8704069
:10A84000F9F7A6BA41F6A850C2F200000321FFF7BB
:10A85000D7FEF9F7E5FCBDE87040F9F799BA304644
:10A86000FCF726FC73681B68002BBFD03046002124
:10A870009847BBE7202383F31188F9F759FCAB69AC
:10A88000706E23F0100341F6A856AB61C2F20006C9
:10A8900018B1F9F7ADFD00237366F9F769FC0023E1
:10A8A00083F31188B2E741F6A8500221C2F20000FA
:10A8B000FFF7A6FE2903BFD5C4E741F6A850C2F2B0
:10A8C00000000021FFF79CFEAC03B1D541F6A85073
:10A8D000C2F200000121FFF793FE6803AAD5E2E768
:10A8E00041F6A850C2F200000021FFF701FFA807BF
:10A8F00094D541F6A8500121C2F20000FFF7F8FEFE
:10A9000069078DD541F6A850C2F200000221FFF779
:10A91000EFFE2A0786D541F6A850C2F200000321B7
:10A92000FFF7E6FE7EE700BFAFF30080AFF30080E5
:10A93000036D03EB4111D1F8003B43F08063C1F894
:10A94000003B7047AFF30080AFF30080AFF30080AF
:10A95000036D03EB411210B4D2F8004944F00444F3
:10A96000C2F80049D3F834285DF8044B012000FAFE
:10A9700001F11143C3F83418704700BFAFF30080F2
:10A98000036D03EB4111D1F8003B43F40013C1F810
:10A99000003B7047AFF30080AFF30080AFF300805F
:10A9A000036D03EB4111D1F8003943F40013C1F8F2
:10A9B00000397047AFF30080AFF30080AFF3008041
:10A9C000036D03EB4111D1F8003B23F40013C1F8F0
:10A9D000003B7047AFF30080AFF30080AFF300801F
:10A9E000036D03EB4111D1F8003923F40013C1F8D2
:10A9F00000397047AFF30080AFF30080AFF3008001
:10AA000042F27C324FF42053C4F20003C2F200023F
:10AA10005321CA20136058625962DA68D10614D4EF
:10AA2000DA6842F08002DA601946CA684FF42053AF
:10AA30005206C4F20003F8D5F922C0F27F021A616F
:10AA40001A61DA6822F08002DA607047AFF30080A2
:10AA500042F27C3310B4C2F200031A68D3689C0639
:10AA6000FCD51369946A106852684860C3F30E03FA
:10AA7000181B4FF47A7404FB00F00133B0FBF3F3BE
:10AA8000CB600A605DF8044B704700BFAFF30080F5
:10AA90002DE9F043202385B0044683F31188F9F7AC
:10AAA00007FB20466946FFF7D3FFF9F721FB002398
:10AAB00083F311889DE80C00C3F30231C3F3032034
:10AAC00001EB8109C3F3021103F00F0500EB490903
:10AAD00001EB8108C2F30030C3F38051C2F30114CB
:10AAE00002F00F0C4FEA491905EB480804EB840407
:10AAF00086004D000CEB44073044C2F3032C49EAB6
:10AB00005808C2F303460D44C2F30352C3F3015184
:10AB10000CEB400448EA07471436AD0001EB810115
:10AB200002EB820247EA445406EB420205EB410085
:10AB3000C3F3034344EA4262184442EAC02005B02A
:10AB4000BDE8F083AFF30080AFF30080AFF3008087
:10AB5000704700BFAFF30080AFF30080AFF3008019
:10AB600038B50446406A0268136823F01F03136077
:10AB70001368D907FCD4057A216A43680A683D2026
:10AB8000A8401860136823F01F0313601368DB07E5
:10AB9000FCD46368087A4A681B683D2181401160D3
:10ABA000CBB104222270204698472378042B12D080
:10ABB000202383F31188F9F7BBFAA3682BB1002295
:10ABC000A26018461A62F9F713FCF9F7D1FA0023CC
:10ABD00083F3118838BD02232370E9E7AFF30080C7
:10ABE0002DE9F04142F2803342F28436C2F200068F
:10ABF000C2F20003254F4FF6FF72304642F2B435E1
:10AC0000C2F200051A80FBF7FBFF4FF440511622F9
:10AC1000462307F1240EC4F20101C0F20162C0F222
:10AC20000163284642F2E434C2F20004F161376263
:10AC3000C6F824E0B262F3624FF01608FBF7E0FFBB
:10AC400046264FF46053A7F13002C4F20003A7F187
:10AC50003C01C0F20108C0F201062046EB616A62C5
:10AC60002962C5F82880EE62FBF7CAFF4FF47053E3
:10AC7000A7F16002C4F200030C3FC4F82880E6622A
:10AC8000E36122626762BDE8F08100BFE0910208E3
:10AC90000378012B10B504461ED0C3696268A06A10
:10ACA0005289E16A20F4F04021F4F04112F4006F7F
:10ACB0001CBF40F4205041F42051A062E16242F4F4
:10ACC00041720020072118801A8099801A8892B258
:10ACD00042F040021A8010BD42F28433C2F20003F7
:10ACE000984215D042F2B433C2F2000398422AD0FF
:10ACF00042F2E433C2F2000398423FD0216A626A12
:10AD0000E3690868116803F10C0282608A60C5E794
:10AD10004AF66132C0F600020A212346006AFDF7B6
:10AD2000F7FB4AF65132C0F600022346606A0A2158
:10AD3000FDF7EEFB4FF46053C4F202035A6C42F489
:10AD400080525A64DAE74AF66132C0F600020A21FC
:10AD50002346006AFDF7DCFB4AF65132C0F60002DA
:10AD60002346606A0A21FDF7D3FB4FF46053C4F217
:10AD700002031A6C42F480421A64BFE74AF6613259
:10AD8000C0F600020A212346006AFDF7C1FB4AF61D
:10AD90005132C0F600022346606A0A21FDF7B8FB73
:10ADA0004FF46053C4F202031A6C42F400421A6476
:10ADB000A4E700BFAFF30080AFF30080AFF30080E3
:10ADC0000378022B10B5044600D010BDC369006A99
:10ADD00000221A809A80FDF703FC606AFDF700FCF0
:10ADE00042F28433C2F200039C4215D042F2B433E3
:10ADF000C2F200039C4218D042F2E433C2F20003D4
:10AE00009C4201BF4FF46053C4F202031A6C22F457
:10AE1000004208BF1A6410BD4FF46053C4F202032D
:10AE20005A6C22F480525A6410BD4FF46053C4F23D
:10AE300002031A6C22F480421A6410BDAFF3008042
:10AE400043681A895B68012101FA02F292B25A83BF
:10AE5000704700BFAFF30080AFF30080AFF3008016
:10AE600043681A895B68012101FA02F292B21A83DF
:10AE7000704700BFAFF30080AFF30080AFF30080F6
:10AE8000026A436A12681B6870B4866AC56A42F235
:10AE9000144442F28030C2F20004C2F20000D460D6
:10AEA00051601660D86059601D60116841F0010161
:10AEB00011601A6842F001021A6070BC704700BF4E
:10AEC000F0B4046A476A866AC56A24683868E36031
:10AED00046F4806645F4806561602660C26041602A
:10AEE0000560236843F001032360036843F0010316
:10AEF0000360F0BC704700BFAFF30080AFF3008089
:10AF0000F0B4036A476AC66A1C68806A3B6842F20A
:10AF10001445C2F2000546F48066E5606160206079
:10AF2000DA6059601E60226842F0010222601A68ED
:10AF300042F001021A60F0BC704700BFAFF300801E
:10AF400070B4436A046A866A24681B68C06AE26057
:10AF500042F2803546F48066C2F2000561602660E8
:10AF6000DD6059601860226842F0010222601A68B0
:10AF700042F001021A6070BC704700BFAFF300805E
:10AF800008B5F9F71DF942F21843C2F20003002197
:10AF90001878DA680428116107D10220187011604E
:10AFA0001161D16821F0FF01D1605B6842F2184065
:10AFB0005B68C2F200009847F9F732F9BDE8084033
:10AFC000F8F7E6BEAFF30080AFF30080AFF3008088
:10AFD00042F21843C2F200034FF44062C4F200028E
:10AFE0001846DA60FAF74CBDAFF30080AFF300808B
:10AFF0000378012B10B5044610D06368A0681A6866
:10B00000197AE368B0FBF2F00138002280B208241C
:10B010001A605C609862D9601A6110BD42F21843F0
:10B02000C2F200039842E8D14FF46053C4F2020325
:10B030000022196C41F008011964196A41F00801F5
:10B04000196232201A624021F8F722FF4FF43D4383
:10B05000C0F20153A360D0E7AFF30080AFF30080EC
:10B06000C368002201390120D96258615A621A610D
:10B07000D96805220143D9601A607047AFF3008098
:10B08000C36800221A601A61DA6822F0FF02DA60EF
:10B09000704700BFAFF30080AFF30080AFF30080D4
:10B0A000C368426870B51D69DE68117D3540ADB278
:10B0B000EEB2F64304461E6189B9AE0706D50378A1
:10B0C0000421032B017001D0D368984768071BD473
:10B0D000EB0703D5636820461B69984770BDA90735
:10B0E00006D50378032B03D0052193680170984798
:10B0F0006A07EDD523780422032B2270E8D0636819
:10B100002046DB689847E3E72378032BE0D06368A9
:10B1100005229B68227020469847D9E7AFF300804C
:10B1200008B5F9F74DF842F27040C2F20000FFF79F
:10B13000B7FFF9F775F8BDE80840F8F729BE00BF7A
:10B1400008B5F9F73DF842F27040C2F20000FFF78F
:10B15000A7FFF9F765F8BDE80840F8F719BE00BF8A
:10B1600008B5F9F72DF842F22840C2F20000FFF7C7
:10B1700097FFF9F755F8BDE80840F8F709BE00BF9A
:10B1800008B5F9F71DF842F24040C2F20000FFF79F
:10B1900087FFF9F745F8BDE80840F8F7F9BD00BFAB
:10B1A00008B5F9F70DF842F25840C2F20000FFF777
:10B1B00077FFF9F735F8BDE80840F8F7E9BD00BFBB
:10B1C00070B542F27044C2F20004204642F22846B2
:10B1D000FAF7D6FCC2F20006002342F24045C4F260
:10B1E00001033046C2F20005E360FAF7C9FC42F2FF
:10B1F00058444FF080432846F360C2F20004FAF747
:10B20000BFFC4FF48063C4F200032046EB60FAF702
:10B21000B7FC4FF48043C4F20103E36070BD00BF8C
:10B22000F8B50378012B04463BD0C36800221A60AE
:10B230005A639A635A626268A56850689169167D7C
:10B240001278B5FBF0F0013880B221F0FF01002543
:10B250004FF6FF771D61D9609862DF626EB940F2E8
:10B260000120542198619960C2B113221A6203F13E
:10B270003802343322616361F8BD4FF48170642178
:10B28000986199603AB131221A6203F1340238337D
:10B2900022616361F8BD13221A62F6E731221A6255
:10B2A000E5E742F27043C2F20003984213D042F243
:10B2B0002843C2F20003984229D042F24043C2F22E
:10B2C000000398423CD042F25843C2F20003984235
:10B2D00045D0E368AFE74FF46053C4F202030022A5
:10B2E000596C41F001015964596A41F001015962F8
:10B2F00019205A623021F8F7CBFD1B203021F8F7D6
:10B30000C7FD4FF4F443C0F60323A360E1E74FF415
:10B310006053C4F202030022196C41F00101196468
:10B32000196A41F0010119621C201A623021F8F7F4
:10B33000AFFD4FF43D43C0F20153A360E3687AE7E9
:10B340004FF46053C4F202030022196C41F0020171
:10B350001964196A41F0020119621D20E5E74FF4F2
:10B360006053C4F202030022596C41F480315964E5
:10B37000596A41F48031596218205A62BEE700BF11
:10B3800008B50378022B00D008BD42F27043C268B2
:10B39000C2F20003002198421160D16011611DD0FA
:10B3A00042F22843C2F20003984226D042F24043C0
:10B3B000C2F2000398422CD042F25843C2F200037A
:10B3C0009842E1D11820F8F78BFD4FF46053C4F296
:10B3D00002035A6C22F480325A64D5E71920F8F738
:10B3E0007FFD1B20F8F77CFD4FF46053C4F202038D
:10B3F0005A6C22F001025A6408BD1C20F8F770FD57
:10B400004FF46053C4F202031A6C22F001021A6472
:10B4100008BD1D20F8F764FD4FF46053C4F2020329
:10B420001A6C22F002021A6408BD00BFAFF300805C
:10B43000C36842685869117D10B440F001000024CF
:10B4400058611C61B1B9D16819B1D96841F00201E4
:10B45000D960916819B1D96841F00401D9601269C5
:10B460001AB1DA6842F00102DA6005221A605DF86A
:10B47000044B7047916819B1D96841F00201D96055
:10B48000D1680029E7D1EAE7AFF30080AFF300808D
:10B49000C36800221A601A61DA6822F0FF02DA60DB
:10B4A000704700BFAFF30080AFF30080AFF30080C0
:10B4B00038B542F28845C2F20005F8F781FE2B69E3
:10B4C0001A69DC681440A4B2E2B2D2431A61A3073D
:10B4D0002CD4600722D4210718D4E2060ED4E30747
:10B4E00006D56B6842F288409B68C2F2000098471C
:10B4F000F8F796FEBDE83840F8F74ABC6B6842F2B0
:10B5000088409B6AC2F200009847E8E76B6842F205
:10B5100088401B6AC2F200009847DEE76B6842F27F
:10B5200088409B69C2F200009847D4E76B682846C0
:10B530001B699847CDE700BFAFF30080AFF30080F1
:10B5400008B5F8F73DFE42F29C40C2F200004FF40D
:10B5500080634268C4F201036FF0010192681961CF
:10B560009047F8F75DFEBDE80840F8F711BC00BF52
:10B5700010B5F8F725FE4FF48063C4F201031A6991
:10B58000DC681440A4B2E2B2D2431A61A30725D406
:10B5900060071AD421070FD4E20607D542F29C4374
:10B5A000C2F2000318465B689B6A9847F8F738FEBA
:10B5B000BDE81040F8F7ECBB42F29C43C2F2000336
:10B5C00018465B681B6A9847E6E742F29C43C2F262
:10B5D000000318465B689B699847DBE742F29C438F
:10B5E000C2F2000318465B681B699847D0E700BFAA
:10B5F00038B542F28845C2F20005284642F29C4422
:10B60000FAF7E6FFC2F200044FF40063C4F200034D
:10B6100020462B61FAF7DCFF4FF48063C4F201038C
:10B62000236138BDAFF30080AFF30080AFF300803B
:10B630000378012B70B5044655D0036900221A60C7
:10B640005A639A63DA631A645A626268E668106839
:10B650002589D168D46AB6FBF0F00138013D01F0CC
:10B660000F0180B2ADB201299862DD625C6003D047
:10B6700002290CBF03210021506900F00F000128AE
:10B680002ED002282AD0D06900F00F00012822D045
:10B6900002281ED0506A00F00F00012803D00228B3
:10B6A00003D141F4005141F48051106B926819624A
:10B6B00020F0FF00002A18BF40F0010001250024FF
:10B6C0004FF4004185225D611C61D86059641A60A5
:10B6D00070BD41F4007141F48071DBE741F020015D
:10B6E00041F01001CFE742F28843C2F200039842D2
:10B6F0000BD042F29C43C2F2000398421DD0236952
:10B7000046F668029A61DA619FE74FF46053C4F22B
:10B7100002030022196C41F004011964196A41F016
:10B72000040119621E201A627021F8F7B1FB4FF470
:10B730003D43C0F20153E360E1E74FF46053C4F2CC
:10B7400002030022596C41F002015964596A41F028
:10B75000020159622C205A627021F8F799FB2E20C1
:10B760007021F8F795FB4FF4F443C0F60323E36030
:10B77000C5E700BFAFF30080AFF30080AFF30080F8
:10B780004FF48053C4F201039A8992B242F08002CE
:10B790009A817047AFF30080AFF30080AFF3008071
:10B7A0004FF48843C4F200039A8992B242F08002B7
:10B7B0009A817047AFF30080AFF30080AFF3008051
:10B7C0004FF49043C4F200039A8992B242F080028F
:10B7D0009A817047AFF30080AFF30080AFF3008031
:10B7E0002DE9F041456FB5F80C802C88A4B2E20534
:10B7F00006461FFA88F85BD4202383F31188F8F7F4
:10B8000097FC14F02F0F2DD0371D08E0A988A00653
:10B8100089B21ED42C88A4B214F02F0F22D0230793
:10B82000F4D014F0080F14BF80210021E00748BFB6
:10B8300041F02001A20748BF41F04001630748BF23
:10B8400041F480713846F9F763F9A988A00689B2F6
:10B85000E0D5C9B23046FAF7A3FF2C88A4B214F0A1
:10B860002F0FDCD1F8F784FC002383F3118818F044
:10B87000800F01D022062ED4630601D4BDE8F081EA
:10B88000202383F31188F8F753FC726CB36C9A424F
:10B8900035D04FF6BF7308EA03034FF6BF72AB8192
:10B8A0002A80F8F765FC002383F31188BDE8F08156
:10B8B000202383F31188F8F73BFC301D4FF400710F
:10B8C000F9F726F9F8F754FC002383F311884FF6B3
:10B8D000FF632B8090E7202383F31188F8F728FC7F
:10B8E00006F13000F9F7A4FA0028A4BF80B2A880BE
:10B8F0000DDBF8F73DFC002383F31188BCE7B36B45
:10B90000002BC6D0301D1021F9F702F9C1E7301D18
:10B910000821F9F7FDF828F0C00343F04003AB819C
:10B92000E7E700BFAFF30080AFF30080AFF3008024
:10B9300008B5F8F745FC42F2B040C2F20000FFF74C
:10B940004FFFF8F76DFCBDE80840F8F721BA00BFDB
:10B9500008B5F8F735FC42F22850C2F20000FFF7B4
:10B960003FFFF8F75DFCBDE80840F8F711BA00BFEB
:10B9700008B5F8F725FC42F2A050C2F20000FFF72C
:10B980002FFFF8F74DFCBDE80840F8F701BA00BFFB
:10B9900070B542F2B046C2F200064BF281723046F8
:10B9A000C0F60002002142F22855FAF7A9FEC2F2C1
:10B9B00000054FF480534BF2A172C4F201032846F4
:10B9C000C0F60002002142F2A0547367C2F20004E4
:10B9D000FAF796FE4FF488434BF2C172C4F20003AB
:10B9E0002046C0F6000200216B67FAF789FE4FF48B
:10B9F0009043C4F20003636770BD00BFAFF30080E3
:10BA000038B549F29024037AC0F60204002918BF21
:10BA10000C46012B054631D06B6F4FF4A0514FF40B
:10BA20008052C4F20102C4F20101934218BF8B425A
:10BA30000BBF216821684FF43D424DF680620CBF78
:10BA4000C0F20152C0F28022B2FBF1F292B21A812E
:10BA5000A288E188208942F4045241F0400442F077
:10BA60002C0240F0010092B2A4B280B200211C82EC
:10BA700098829A8119801A889B8838BD42F2B04317
:10BA8000C2F20003984218D042F22853C2F20003D7
:10BA900098421FD042F2A053C2F200039842BBD199
:10BAA0004FF46053C4F2020327201A6C42F4802240
:10BAB0001A64C021F8F7ECF9AEE74FF46053C4F212
:10BAC000020325205A6C42F010025A64C021F8F794
:10BAD000DFF9A1E74FF46053C4F2020326201A6C89
:10BAE00042F400321A64C021F8F7D2F994E700BF9B
:10BAF000FCF716BEAFF30080AFF30080AFF3008019
:10BB000001207047AFF30080AFF30080AFF30080F7
:10BB100000207047AFF30080AFF30080AFF30080E8
:10BB2000704700BFAFF30080AFF30080AFF3008039
:10BB300010B5022408B1204610BD48F60C23C2F20D
:10BB4000000318461C79053C18BF0124FFF7E0FFED
:10BB50000028F0D044F00404E4B2204610BD00BF39
:10BB600010B5022408B1204610BD48F60C23C2F2DD
:10BB7000000318461C79053C18BF0124FFF7C8FFD5
:10BB80000028F0D044F00404E4B2204610BD00BF09
:10BB900010B50C4682B010B1042002B010BD48F6BA
:10BBA0000C20C2F200000179052918BF0320F4D14E
:10BBB00011460193FAF7FCFA019B90B91BB912E008
:10BBC00013F0FF030FD048F60C202146C2F200000C
:10BBD0000193FAF725FB019B04F50074013B002853
:10BBE000EED00120D9E748F60C20C2F2000002B0E6
:10BBF000BDE81040FAF75CBBAFF30080AFF3008004
:10BC000030B50D4683B010B1042003B030BD48F606
:10BC10000C24C2F200042179052918BF0320F4D1B5
:10BC2000204601920093FFF773FF019A08B10220AA
:10BC3000EBE720461146FAF78BFB009B90B91BB946
:10BC400012E013F0FF030FD048F60C202946C2F291
:10BC500000000093FAF7B4FB009B05F50075013B6B
:10BC60000028EED00120D0E748F60C20C2F20000F8
:10BC700003B0BDE83040FAF7FBBB00BFAFF3008074
:10BC800008B10420704729B10229FAD14FF400739A
:10BC90001380704708467047AFF30080AFF3008011
:10BCA00042F27C30C2F20000FAF7CABCAFF3008067
:10BCB00001460020F9F79CB9AFF30080AFF3008094
:10BCC000F9F7DEB9AFF30080AFF30080AFF3008087
:10BCD0002DE9F041C56A8D4204460E4602D0037933
:10BCE00073B916B90020BDE8F081607804F1300125
:10BCF00032460123FFF74CFF20BBE662BDE8F0812E
:10BD000000F13008414640782A460123FFF778FFCA
:10BD1000C0B9E369226A20711A449542E1D2E778FA
:10BD2000012F01D8DDE7E3691D44013F2A46607811
:10BD300041460123FFB2FFF763FF012FF3D1002E2D
:10BD4000D0D0D2E70120BDE8F08100BFAFF3008082
:10BD500038B504460A46407804F130010123FFF764
:10BD600017FF08B1032038BD94F82F1294F82E2243
:10BD70004AF6552342EA012212B2CFF6FF739A42E5
:10BD800018BF022000D038BD94F8683094F869508C
:10BD900094F8661094F867201B0443EA05630B438C
:10BDA00043EA022244F2461322F07F42C0F25403D7
:10BDB0009A42E8D094F8842094F8855094F8821040
:10BDC00094F88300120442EA05620A4342EA002022
:10BDD00020F07F40C01A18BF012038BDAFF30080AB
:10BDE0002DE9F04103681C78303C092C154602D837
:10BDF0005A783A2A18D042F21C63C2F200031C6837
:10BE00000C6074B12378B3B16078FFF7A9FEC20764
:10BE100011D405B310F0040F0CBF00200A20BDE8B8
:10BE2000F0810C20BDE8F08102330360002CE2D0E9
:10BE30000B20BDE8F081002020706070FFF778FED5
:10BE4000C30702D50320BDE8F0813DB1470705D502
:10BE50000A20BDE8F0812846BDE8F0812046002197
:10BE6000FFF776FF012818BF002506D0032800F051
:10BE7000BA80C8B10D20BDE8F08194F8F231002BF2
:10BE8000F8D094F8F82194F8F91194F8F63194F870
:10BE9000F751120442EA0162134343EA0525294699
:10BEA0002046FFF755FFE1E794F83C2094F83B303B
:10BEB00043EA0223B3F5007FDCD194F8471094F8ED
:10BEC000463053EA01210DD194F8562094F85700DA
:10BED00094F8543094F85510120442EA0062134367
:10BEE00043EA012194F84000E161431EDBB2012BDB
:10BEF000E070BFD894F83D20A270002ABAD0531E3B
:10BF00001342B7D194F8426094F8413043EA0623D3
:10BF10001E072381AED194F8447094F8436056EA2A
:10BF200007260FD194F852C094F8538094F85060CB
:10BF300094F851704FEA0C4C4CEA086C4CEA060637
:10BF400046EA072694F83FC094F83E7057EA0C275B
:10BF500090D000FB01FC07EB13106044864289D3AC
:10BF6000361AB6FBF2F2002A84D040F6F576B242D9
:10BF700040F2BC8006F57046B24200F29C80022678
:10BF8000023228442F44A261A0622762002B3FF4B2
:10BF900071AF022E1CBF03235343674418BF02F046
:10BFA000010267620EBF520002EB5302012602F249
:10BFB000FF12B1EB522FFFF45DAF4FF0FF320023C1
:10BFC000032E2261E36011D042F21863C2F2000333
:10BFD00000201A882670013292B220711A80E28005
:10BFE000E062BDE8F0810120BDE8F08194F86110C5
:10BFF00094F86020637142EA01222A446261607809
:10C0000004F130010123FFF7C3FD0028DCD194F8CF
:10C010002F1294F82E224AF6552342EA012212B238
:10C02000CFF6FF739A42CFD194F8322094F83300C0
:10C0300094F8303094F83110120442EA00621A4346
:10C0400045F2522342EA0122C4F261139A42BBD163
:10C0500094F8162294F8170294F8143294F81512F2
:10C06000120442EA00621A4347F2722342EA0122B2
:10C07000C6F241139A42A7D194F81E7294F81A524C
:10C0800094F81F8294F81BC294F81C2294F818327A
:10C0900094F81D0294F819123F042D0447EA08672A
:10C0A00045EA0C653A432B4342EA002243EA012366
:10C0B000E260236188E7023228442F44A261A06233
:10C0C0002762002B7FF4D6AE94F85E6094F85F7020
:10C0D00094F85C3094F85D00360446EA0766334312
:10C0E00043EA002392006362032660E7012647E7E4
:10C0F00008B508B103780BB9092008BDC3888B4285
:10C10000FAD14078FFF72CFD10F0010F0CBF002092
:10C11000032008BDAFF30080AFF30080AFF30080D1
:10C12000F8B50378022B04460D4646D0032B28D0E1
:10C13000012B02D04FF0FF30F8BD016A05EB550628
:10C1400001EB5621FFF7C4FD0028F3D1C6F3080325
:10C15000216A2344013601EB5621204693F83070C2
:10C16000FFF7B6FD0028E5D1C6F308063444E90719
:10C1700094F8303047EA03204CBF0009C0F30B00AD
:10C18000F8BD016A01EBD511FFF7A2FD0028D1D15E
:10C19000AD0005F4FE7505F1300323442C44D87836
:10C1A00099785A7894F83030000640EA014040EA25
:10C1B0000220184320F07040F8BD016A01EB152100
:10C1C000FFF786FD0028B5D16D0005F4FF756319F2
:10C1D0001C4693F8303094F8310043EA0020F8BD53
:10C1E000836870B50446012B0D46E18003D00068DA
:10C1F0008269934201D3022070BDB3B90378032B47
:10C2000010D003890022AB42E260F4D9436A03EB09
:10C210001513236105F00F0500EB45103030606108
:10C22000002070BD436A002BEBD086783601B54202
:10C2300019D3012BDFD9AD1B9A42ADB2DBD908E08F
:10C24000012BD8D9206882699A42D4D9AE420AD843
:10C250000D461946FFF764FFA91B0346013089B25A
:10C26000EED1012070BD991E023A9142E3603BBFBE
:10C270008278836A002102FB013101EB15112161F3
:10C28000C8E700BFAFF30080AFF30080AFF30080DA
:10C29000F8B50378022B04460D4616465BD0032BF7
:10C2A0003AD0012B18BF022002D001232371F8BD20
:10C2B000216A05EB550701EB5721FFF709FD00281F
:10C2C000F3D1C7F30803234415F0010518BF93F811
:10C2D0003010F2B21EBF01F00F0141EA0212D2B2D9
:10C2E000216A83F830200137012301EB57212371A4
:10C2F0002046FFF7EDFC0028D7D1C7F30807002D33
:10C300003DD12744C6F3032697F8303023F00F03BE
:10C310001E4387F83060C8E7016A01EBD511FFF7CB
:10C32000D7FC0028C1D1AD0005F4FE7505F130033E
:10C3300023442544DA78120602F070421643C6F30D
:10C340000727310C320E85F830605F709970DA7013
:10C3500001232371F8BD016A01EB1521FFF7B8FC39
:10C360000028A2D16D0005F4FF756219C6F30723FA
:10C3700082F83130012382F830602371F8BDC6F3B2
:10C3800007162744C5E700BFAFF30080AFF3008076
:10C39000F8B506460F4669B9C5688369CDB9012568
:10C3A0002C460134A34217D8012D25D9022B52D88F
:10C3B0000120F8BD0129FBD983699942F8D2FFF722
:10C3C000AFFE0128F4D9B369834298BF3D46E7D94F
:10C3D000F8BD9D42E3D2E3E7012CE9D9304621467E
:10C3E000FFF79EFE50B1B0F1FF3F18BF0128EFD01C
:10C3F000A54201D0B369D4E70020F8BDB3699C42DF
:10C40000D6D2304621466FF07042FFF741FFD0F19F
:10C41000010338BF0023002F08BF00234BB1012FB9
:10C42000C6D9B3699F42C3D2394630462246FFF788
:10C430002FFF58B93369F4605D1C05D00122013B20
:10C44000727133612046F8BD2046C1E70128AFD1A3
:10C450004FF0FF30F8BD0224C0E700BFAFF300800B
:10C460002DE9F047C5880135ADB204460E4615B931
:10C470000420BDE8F0870369002BF9D015F00F0701
:10C4800008D0036803EB471330336361E580002075
:10C49000BDE8F087C16801330361036861B19A7830
:10C4A000013A12EA1512EDD1012902D99A69914295
:10C4B00006D30220BDE8F0871A89AA42D8D9E1E75D
:10C4C0001846FFF72DFE01288046F2D9B0F1FF3F54
:10C4D0001BD023689A6982420AD8002EC8D0184619
:10C4E000E168FFF755FF804690B90720BDE8F08767
:10C4F000861E023A9642C4F80C803BBF99789A6A2D
:10C50000002601FB06262661BCE70120BDE8F08776
:10C510000128CED0B0F1FF3FF7D020680021FFF70F
:10C52000D7FB0028F1D12268014602F1300302F561
:10C530000C7203F8011B9342FBD122689369A8F1A6
:10C540000206023B9E423BBF936A9178002301FBA7
:10C550000633D3624FF000094FF0010A0EE082F873
:10C5600004A02068FFF7B4FB09F101090028CCD131
:10C570002268D36A01335FFA89F9D362907848451B
:10C580004FF000011346EAD8D16A9269C9EB010164
:10C59000D962AEE7AFF30080AFF30080AFF3008065
:10C5A0002DE9F04FFF2785B0DFF850810546B946E9
:10C5B0004FF6FF7609E00F2942D04FF0FF092846D9
:10C5C0000021FFF74DFF002837D128682969FFF7C0
:10C5D0007FFB002831D16C692378002B75D0E27A7B
:10C5E000E52B02F03F01E8D01207E4D40F2927D051
:10C5F000B9F1000F11D19C46224604F10A09034605
:10C6000001E012F801CFD90141EA53035CFA83F348
:10C610004A45DBB2F5D1BB420FD0AB692E84DA7A42
:10C62000D20758BF04F10B0CC7D414F8011B13F840
:10C63000012B9142C1D16445F7D105B0BDE8F08F1F
:10C64000EA69002ABBD058063BD5E988677B298474
:10C6500003F0BF0994F80DA0BA45AED12378264F58
:10C6600023F04003013B03EB430C03EB8C0C4FF036
:10C67000010B03E0B04235D147452AD017F8013FFE
:10C68000E018E35C407843EA0020BBF1000FF1D0F2
:10C690000CF101030192CDF808C0039301F0B0F84A
:10C6A000DDF808C0019ABCF1FE0F83461AD832F8B3
:10C6B0001C0001F0A5F88345019A13D1DDF80CC0E8
:10C6C000DAE74B457FF479AFC4E7042005B0BDE855
:10C6D000F08F2378590609D5BBF1000F06D032F848
:10C6E0001C301BB157464FF0FF0968E709F1FF39CD
:10C6F0005FFA89F9574662E73F9402084C940208B2
:10C700002DE9F04F0B782F2B18BF5C2B89464FF08B
:10C71000000408BF01F101098460054699F8000092
:10C720001F2888BF49F2A03785B084BFA046C0F655
:10C73000020740F26D815C2818BF2F2809D109F14A
:10C7400001039946013399F800002F2818BF5C288F
:10C75000F7D02F2818BF1F28EE698CBF00240124B2
:10C7600031D95C2851D00121A6F1020BCA4601241F
:10C7700001F01EF818B37F280CD822281FD049F2E8
:10C780002042C0F6020201E0984218D012F8013FA0
:10C79000002BF9D12BF8020F1AF8010F2F2818BF20
:10C7A0001F2804F1010310D95C282FD0B3F5807F36
:10C7B00005D001211C4600F0FBFF0028DBD106203C
:10C7C00005B0BDE8F08F002401231F28994498BFCD
:10C7D0004FF0040B1BD8002CF1D004F10043013BB7
:10C7E0005A0036F813302E2B18BF202B12D1931C71
:10C7F000334407E033F8042C2E2A18BF202AA3F173
:10C80000020307D1013CF5D1D9E7012399444FF048
:10C81000000BE0E7AB6926F8148003F10B0106EB8F
:10C82000440E202203F8012B8B42FBD13388202BAE
:10C8300018BF2E2B14BF4FF0000A4FF0010A40F032
:10C84000F38032464FF0000A32F8020F202818BF5A
:10C850002E280AF1010AF7D04BF0030B734633F888
:10C86000022D2E2A01D0013CF9D100239C4608223A
:10C870000AF1010A00B3202864D0B4EB0A0E18BFF5
:10C880004FF0010E2E2814BF00210EF001010029E7
:10C8900058D1544518BF934234BF0021012162D3BF
:10C8A0000B2A00F0C380BEF1000F00F09080A2457B
:10C8B0004BF0030B40F28B80AB691978E52902BF7E
:10C8C00005211970AB69082A04BF4FEA8C0C5FFA86
:10C8D0008CFC0CF00C020C2A00F081800CF003019F
:10C8E00003297CD01BF0020F0AD10CF0030CBCF121
:10C8F000010F08BF4BF0100B042A08BF4BF0080BC8
:10C9000083F80BB028460021FFF76AFCF8B92846E7
:10C91000FFF746FEAB69DB7AD8B95C073FF550AF4D
:10C920006B69DA7AD1067BD5587D1A7DD97E9B7EDC
:10C9300042EA002243EA012343EA0243AB6099F84A
:10C940000000F8E64BF0030B36F81A0090E7AB69ED
:10C95000DB7A04287FF434AF13F0040F08BF0520FE
:10C9600005B0BDE8F08F7F2819D82B2828D049F2D0
:10C970002C4EC0F6020E01E0884221D01EF8011FA5
:10C980000029F9D1A0F1410189B219299CBF4CF0CD
:10C99000020CC0B22CD8A969C8540133D4E7019263
:10C9A0000293CDF80CC000F003FF01AA92E80C102E
:10C9B000C0B138444BF0020B10F8800C0028D4D1E1
:10C9C0004BF0030B5F20A969C8540133BCE74FEA61
:10C9D0008C0C5FFA8CFCA2460B220823B4E74BF0C8
:10C9E000020B7FE74BF0020B4BF0030B5F20EAE7F3
:10C9F000A0F1610189B2192998BF2038A9698CBFBB
:10CA0000C0B2C0B2C85498BF4CF0010C01339BE7D0
:10CA100028462146FFF7E4FB6C6105B0BDE8F08FC6
:10CA2000052005B0BDE8F08F184617E74BF0030B63
:10CA300042E700BFAFF30080AFF30080AFF30080A8
:10CA400070B401F10B0683B0044611F8015BB142EA
:10CA500004F8015BF9D1052B0CD9148800E00C46D1
:10CA6000D90341EA530332F8021F14FA83F39BB24D
:10CA70000029F4D1072203F00F0404F13001013A38
:10CA800000AD3929154488BF04F137011B096970CD
:10CA9000F1D102A911447E2401F8084CE2B10178D9
:10CAA000202908D0014603E011F8014F202C02D0C4
:10CAB00001339342F8D1072A9BBF02A9891820218C
:10CAC00011F8081CC15403F1010398BF0132072B70
:10CAD000F1D903B070BC70471346ECE7AFF30080A8
:10CAE00008B10B20704742F21C63C2F200031A68BF
:10CAF00002B1107009B100220A701960002070475D
:10CB00002DE9F04F95B014AB914643F8441D002237
:10CB100002600BA909F01E0204461846FFF760F9EF
:10CB200007464FF40070FFF7C3F805461120002DAB
:10CB300000F0E88005AB1295119309F01F06002F55
:10CB400000F08F8019F01C0F00F02B81042F40F0B3
:10CB50002881DDF844A0DDF8489052460DF11F030E
:10CB60000DF12B0012F8011B03F8011F8342F9D1CC
:10CB70009DF82B30DA072BD500238AF80B304FF0C5
:10CB8000010812930BE0FFF70BFD08F101080746BF
:10CB90001FFA88F888B9B8F1640F00F01081504688
:10CBA00008A94A464346FFF74BFF0BA80021FFF7B1
:10CBB00017FB07460BA8002FE5D0042F40F0F180AB
:10CBC0009DF82B308AF80B309DF82B30CDF848902B
:10CBD0009B0758BF4FF0010915D5B9F8003033B1A4
:10CBE000002301339BB239F81320002AF9D14EF605
:10CBF0004F421933C4F6C46282FB0302DB17C3EB56
:10CC0000A2091FFA89F90BA80021FFF7E9FA0746E4
:10CC1000002840F0C68023468246544698460BE0E2
:10CC20000CB9BDF832A094B24C4500F00781FFF773
:10CC300017FC0746002868D10F990B98FFF748F8B2
:10CC40000746621C0BA80121002F5ED1109B1B78A8
:10CC5000E52B18BF002B14BF00230123E0D01C4696
:10CC6000E5E70BA80399FFF74BFDDDF84080074689
:10CC700000287FF467AFB8F1000F00F09B8019F037
:10CC80001C0F40F07F8198F80B30DA0600F190809D
:10CC900019F0020F40F0908009F00803DBB2DDF8D4
:10CCA0002CA00BB146F02006DAF82C30C4F8208016
:10CCB0002846E361FFF704F8A67198F8155098F834
:10CCC0001A0098F8141098F81B200B9B41EA0521D4
:10CCD00040EA022242EA0142226198F81E6098F876
:10CCE0001F5098F81C0098F81D10DA882360330450
:10CCF00043EA0563034343EA01230020E360A28083
:10CD0000A060A06115B0BDE8F08F444646F008066B
:10CD1000DDF84080002F44D1370758BFDDF82CA044
:10CD2000C2D5FEF7BDFF98F81A3098F815C098F8EC
:10CD3000141098F81B20DDF82CA088F80E0043EAA8
:10CD4000022241EA0C210023C0F3072E070C4FF00A
:10CD50000109000E52EA014B88F80FE088F81070C4
:10CD600088F8110088F80B3088F81C3088F81D30DE
:10CD700088F81E3088F81F3088F81A3088F81B3081
:10CD800088F8143088F815308AF804908AD0DAF8D8
:10CD90002C30CB45009303D0DAF818309B4510D3E4
:10CDA00002272846FEF78CFF384615B0BDE8F08F05
:10CDB0000427F6E70627C5E6DF077FF56DAF0727EF
:10CDC000EFE7019627465E4621E00128E8D00130D2
:10CDD00000F0D680DAF818209642E1D2314650466B
:10CDE0000022FFF755FA002840F0D880DAF810301A
:10CDF000591C1CBF0133CAF81030DAF8183018BFBC
:10CE00008AF80590A34209D9012CC9D92646504673
:10CE10003146FFF785F904460028D6D10B980099D2
:10CE2000019E0BF1FF33C360FEF752FF3C46DDF875
:10CE30002CA0074600283FF435AFB2E7B9F1010F47
:10CE4000444671D051460BA8FFF7CAF9074600289F
:10CE5000A7D1119B024603F10B0013F8011BD70168
:10CE600047EA520251FA82F28342D2B2F5D109F175
:10CE7000FF339BB249F240498DE86000C0F60209D9
:10CE80004FF6FF784FF0FF0B16461D4602940B98A5
:10CE90000F99FEF71DFF0246002A6ED15FFA85FA50
:10CEA0000AF1FF31109CDDF848C0667301EB4100C8
:10CEB00001EB80014FF00F001346E0722273A2765F
:10CEC000E2760EE03CF8113027184FEA132E235477
:10CED000013187F801E0002B08BF434601320D2ADB
:10CEE00009D0434519F80200ECD1271804F800B026
:10CEF00087F801B0F2E7434502D03CF811300BB996
:10CF00004AF0400A84F800A00B9B4FF00101197110
:10CF10000BA80021FFF7A4FA78BB013DADB2002DAC
:10CF2000B5D19DE86000029C0B980F99FEF7D0FEEA
:10CF3000074600287FF435AFDDF840E00EF120020F
:10CF4000734603F8017B9342FBD1119B724603F1B8
:10CF50000B0013F8011B834202F8011BF9D1119A4F
:10CF60000B9BD17A012201F018018EF80C101A7176
:10CF700046F00806DDF84080CEE6009D074610E743
:10CF800001270EE798F80B3013F0110F7FF417AF5D
:10CF900019F0040F3FF4C0AE082702E7074600E788
:10CFA0002DE9F04F07469B46002383B00C46CBF893
:10CFB00000300068B9889146FFF79AF840B9BB790C
:10CFC000190648BF022003D49A0758BF072002D48D
:10CFD00003B0BDE8F08FFA68B96819EB020F07D308
:10CFE000914243F0200388BFF960BB710020EFE756
:10CFF000B9F1000FF4D007F12403019307F5097884
:10D00000C1F30805002D67D13B689D78013D05EA15
:10D01000512515F0FF050DD1002940F086803869B3
:10D02000002800F08D80012800F09D80461C76D0FD
:10D030003B687861BA79510664D479699A69A1F13B
:10D04000020C023A944580F08E8099789A6A0CFB23
:10D050000122002A00F087805FEA592605EB020AC8
:10D060002FD0AA198A4288BFC5EB010658782146FD
:10D070005246F3B2FEF7C4FD002850D1BB69CAEB9B
:10D08000030C66450CD9019D04EB4C2313F8012BCE
:10D0900005F8012B4545F9D1BB7923F04003BB715D
:10D0A0007202B968A318DBF8000011441044B9EB10
:10D0B0000209B9601C46CBF80000A1D1FA68BB791F
:10D0C0008EE7BA69B968524502D0FA68914240D3F6
:10D0D000C7F818A0C1F30805C5F500724A4528BF76
:10D0E0004A463D44243523463AB1A31814F8016B4F
:10D0F0009C4205F8016BF9D1B968B87940F040005D
:10D10000B871D0E75878BA6901990123FEF778FD24
:10D1100028B9BA793B6822F04002BA718DE7BB7931
:10D1200063F07F03BB71012052E718467969FFF76E
:10D130002FF900287FF477AFB968FA68BB794FE719
:10D1400018462946FFF724F9386100287FF46BAFB1
:10D15000F2E75878019952460123FEF719FD00289D
:10D16000DDD1B968B4E7BB7963F07F03BB710220FE
:10D170002EE700BFAFF30080AFF30080AFF3008075
:10D180002DE9F84F04460068A188FEF7B1FFD8B931
:10D19000A27902F0200303F0FF00ABB150060DD5D9
:10D1A0002146A26951F8240B01234078FEF728FD9F
:10D1B000002849D1A37923F04003A3712068E169D5
:10D1C000FEF786FD06460EB1BDE8F88F256AEB7ABC
:10D1D00043F02003EB72E3682B77A3891B0A6B777C
:10D1E000E389AB77E37BEB772369AB76238A1B0A72
:10D1F000EB76638A2B75638A1B0A6B75FEF750FD0D
:10D20000C0F30721020C030EA8752A76E9756B7628
:10D21000A179236821F020010122A1711A712568EA
:10D2200031462846FEF754FD034650B92B78032BB0
:10D230000DD0002168780A46FEF722FD031C18BFB6
:10D2400001231846BDE8F88F0120BDE8F88F6B79FF
:10D25000002BEED005F13001E8620B4605F50C72AB
:10D2600003F8010B93424FF00004F9D12A69EB68EF
:10D2700085F81822C2F3072B4FEA124A4FEA134CE3
:10D280004FEA136E52204FEA1269C3F30728612256
:10D2900085F819B285F81AA24FF0410B4FF0720AC7
:10D2A0005527AA2685F81C3285F8300085F831000C
:10D2B00085F8322085F8172285F81B9285F81D82A3
:10D2C00085F81EC285F81FE285F82E7285F82F6258
:10D2D00085F833B085F816B285F814A285F815A242
:10D2E00068786A690123FEF78BFC6C71A1E700BFC7
:10D2F00010B50446FFF744FF00B9206010BD00BF21
:10D3000070B504460D460068A188FEF7F1FE0028BE
:10D3100054D1A3791E0663D4E268AA4203D213F063
:10D32000020F08BF15460023A268A360002D59D044
:10D3300020688678760242B1013A691EB2FBF6F3A4
:10D34000B1FBF6F1994280F08A80216900294BD027
:10D350006161002933D1A3680D46C3F30802002A96
:10D3600000F08380A269AA427FD0A3795E0658BFED
:10D3700004F124060DD5236804F1240658783146BB
:10D380000123FEF73DFCA379002837D123F04003A9
:10D39000A3712368314658782A460123FEF7F8FB2B
:10D3A00058BBA368E268A5619A4206D2A279E360FD
:10D3B00042F02003A371002070BD002070BDB54273
:10D3C00088BF206856D9A3799A07C6EB05051AD4F9
:10D3D000012902D982698A423DD863F07F03A37193
:10D3E000022070BD284670BDFEF7D2FF012801461D
:10D3F0002FD0013018BF2161AAD1A37963F07F0338
:10D40000A371012070BDFEF7C3FF0146002830D094
:10D410004B1CF2D001291CD920688369994218D28B
:10D42000A36861613344AE42A360CCD32B44C5F3FF
:10D430000802A360DAB12668B0698A1E0238824207
:10D4400007D2B078B16A00FB021202EB5525002A20
:10D4500083D1A379C1E7FEF763FE0146D8E77342A3
:10D460001A40A260AD1A616973E7E2689CE715464D
:10D4700073E73546A368D9E7AFF30080AFF30080C8
:10D4800070B586B006AB044643F8141D002218465A
:10D490002146FEF7A5FC08B106B070BD4FF4007040
:10D4A000FEF706FC05461120002DF5D003ABE56123
:10D4B000A36120460199FFF723F906462846FEF7A7
:10D4C000FFFBBEB963696BB1DA7AD20617D55D7D11
:10D4D0001A7DD87E997E42EA052241EA002343EA7A
:10D4E0000243A3602368DB882046A3800021FEF767
:10D4F00077FE0646042E04D0304606B070BD0526E1
:10D50000FAE70520C8E700BFAFF30080AFF3008063
:10D510002DE9F04F044687B00E460068A188FEF75B
:10D52000E7FD0546002D76D1002E7AD04FF400702D
:10D53000FEF7BEFB80461120B8F1000F6BD003ABA5
:10D54000FF27A3610423C4F81C803D46DFF85092F6
:10D550004FF6FF7A184608E00F2820D0FF25204616
:10D560000021FEF77DFF00284AD12169002900F043
:10D5700090802068FEF7ACFB002841D163691A78DF
:10D58000002A00F0E680E52A18BF2E2AD97AE5D0D5
:10D5900001F03F000907DFD40F2840F0EA80500671
:10D5A0003CD5E1885F7B218402F0BF0593F80DE054
:10D5B000BE45D3D11978D4F81CC0784A01F03F0198
:10D5C000013901EB410001EB8000012708E0FE2852
:10D5D00013D82CF810100F4601304A4500F0BB80DC
:10D5E00012F8011F03EB010B595C9BF801B041EAF3
:10D5F0000B21002FEBD15145EFD07746FF25AEE749
:10D6000003460022042B226110D040460193FEF70E
:10D6100057FB019B184607B0BDE8F08FAA429DD189
:10D62000C4E720463146FEF7DBFDF4E706F10902C8
:10D6300000251570B76917B3F36903B32369DBB12C
:10D64000228C4FF6FF739A4216D0E369188898B17E
:10D6500099460CE0F369013BAB4205F1010507EB8C
:10D66000050309D903F8010C39F8020F28B100218C
:10D6700000F09EF80028EDD1002500237B552046C0
:10D680000021FEF7EDFE0428034604BF00232361BA
:10D69000BBE703460028B4D106F109020029C7D030
:10D6A000616991F80CC00CF0080E5FFA8EFE7346AB
:10D6B000481E8E4606F11107194610F8013F202B2F
:10D6C0000ED0052B08BFE523A3F14105EDB219B13A
:10D6D000192D9CBF2033DBB202F8013BBA42ECD1DA
:10D6E0009EF80830202B71461BD015462E230CF0D7
:10D6F000100E05F8043B5FFA8EFE0132C81D10F8CB
:10D70000013FA3F14107202BFFB20AD0BEF1000F69
:10D7100003D0192F9CBF2033DBB202F8013BAA4291
:10D72000EDD1CB7A33728D7FCF7F0B7F487F2D0475
:10D7300045EA07652B4343EA00233360487E0B7EAE
:10D7400043EA0023B380C87D8B7D43EA0023F38046
:10D750006EE7042355E71B78590606D5FE289CBFC3
:10D7600000232CF810303FF648AF013DEDB277466C
:10D77000F5E675B903F10A0001E013F8012FE9019C
:10D7800041EA550552FA85F58342EDB2F5D1BD4225
:10D7900002D04FF6FF73238421697DE73F9402088E
:10D7A0004C940208AFF30080AFF30080AFF3008029
:10D7B0007F2810B40DD979B90F4B02E0A1B28029AE
:10D7C00016D033F8022F824201F10104F6D18031E4
:10D7D00088B25DF8044B7047FF2809D849F25043DE
:10D7E0008038C0F602035DF8044B33F81000704730
:10D7F00000205DF8044B70474E940208AFF30080A0
:10D8000061280DD049F23072C0F60202002101E019
:10D81000834206D032F8023F0131002BF8D1704725
:10D82000002149F25053C0F6020333F8110070474B
:10D8300041F20073C2F2000318607047AFF300803A
:10D8400041F2047241F20073C2F20002C2F200031C
:10D850004CF6FF110120C3F69A3110701960704721
:10D8600041F6F403C2F200031B6893F8DD355B0652
:10D8700005D549F6B013C0F602031B5C0BB100F0EE
:10D8800047BF7047AFF30080AFF30080AFF3008075
:10D8900041F6F403C2F200032DE9F0411B6806468D
:10D8A0000F46C3F83803F0B942F610330022C2F233
:10D8B0000003C7F6C0729A6197F881322BB143F624
:10D8C0004850C2F2000004F08BF842F68043C2F2E6
:10D8D000000349F6101132461868C0F60201BDE88F
:10D8E000F04116F035BED3F8E00106F0F1FD07EE89
:10D8F000106AF8EEC76A07EE100ADFED0F7A66EEDF
:10D90000876A9FED0E7AC6EEA77A42F61038C2F209
:10D910000008C7EE276A16EE900AF4F7B9FEA823AE
:10D92000A0FB034503FB015520462946F4F788FC7C
:10D93000C8F81800C0E700BF000070420024744916
:10D940002DE9F041054642F66C4086B0C2F2000077
:10D9500017F01EFE00283BD042F68044C2F20004BD
:10D9600042F66C40C2F20000266817F009FE8046BD
:10D9700005F06EFD074616F073F949F63811C0F64A
:10D98000020142463B460090304616F0E1FD206819
:10D9900006F09EFC41F6E803C2F200031C68D4F8CE
:10D9A000FC3D1A6803925A6804929B6804F5217042
:10D9B000059302F02DF903AB0146D4F8002E009335
:10D9C0002846032307F034FB0023CBF68073AB63B8
:10D9D00006B0BDE8F08100BFAFF30080AFF3008078
:10D9E000086D0969F8B58318013B93FBF0F400FB5F
:10D9F000143391E81100896810F903C0E756CE5638
:10DA00008056A5568C561CF1000318BF0123003721
:10DA100018BF0127003618BF0126834204D000300A
:10DA200018BF0120FFF71CFFAF4205D0002D0CBF2F
:10DA300002200320FFF714FFA64207D0002C0CBFE2
:10DA400004200520BDE8F840FFF70ABFF8BD00BF7D
:10DA500038B541F20073C2F200030C461B688B42DA
:10DA600041F204730546C2F200030CD01B784BB19F
:10DA70000CF0E6FB41F6F403C2F200031B68B3F9B5
:10DA800050301BB938BD00221A7038BD42F67040C4
:10DA900029462246C2F20000BDE83840FFF7A0BF89
:10DAA000F0B541F6F402C2F2000242F68043126879
:10DAB000C2F200030C4689B01860D2F83803FFF7B1
:10DAC000E7FED4F8FC3D1A6805925A6806929B68F6
:10DAD00004F52170079302F09BF84DF641164DF6C0
:10DAE00051254FF0030E0246C0F60006C0F60005B1
:10DAF00005AF42F6103049F66811D4F8003ECDF873
:10DB000000E0029603950197C2F20000C0F6020100
:10DB100007F0BEFA49F678104DF691012246C0F69C
:10DB20000200C0F6000116F02BFF49F67C104DF6FE
:10DB300031012246C0F60200C0F6000116F020FFB7
:10DB400049F698104DF641012246C0F60200C0F693
:10DB5000000116F0B5FE09B0F0BD00BFAFF30080C4
:10DB6000002303600268036003684260002BC1BFAA
:10DB7000D0ED007AF8EEE77A9FED157AC7EE277AB6
:10DB8000F0B4D8BF002310A5D5E900450146D8BFA1
:10DB9000C7F6C0734FF00007D8BF83604FF0000690
:10DBA000C7F6C0774FF000024FF00003C8BFC0EDCA
:10DBB000027AC0E90445CE618E61C1E904238F6019
:10DBC000F0BC7047AFF30080003CDD9BFFFFFFFF20
:10DBD000ABC22248AFF30080AFF30080AFF3008008
:10DBE000F8B5044616F034F841F6E803C2F2000333
:10DBF0001B68D3E90C2352EA030509D00EA7D7E925
:10DC00000067821A61EB03039F4208BF96420ED25F
:10DC1000D4E904450AA3D3E90023001B61EB050105
:10DC20008B4208BF824234BF00200120F8BD002093
:10DC3000F8BD00BFAFF30080FF6D0A1E00000000BA
:10DC4000FF79030A00000000AFF30080AFF300800B
:10DC500041F6E803C2F2000310B51C682046FFF746
:10DC6000BFFF08B9E061206042F68C502168C2F223
:10DC7000000017F0E5FA43F648504FF2943142F6AF
:10DC80008C52C2F20000C0F60201C2F20002BDE8EE
:10DC9000104003F06DBF00BFAFF30080AFF3008012
:10DCA00070B582B041B941F6F403C2F200031B68BB
:10DCB00093F8D0359B0601D402B070BD41F6E8055B
:10DCC000C2F200052C682046A669FFF789FF08B953
:10DCD000E0612060226847F22E53013A9A42EBD865
:10DCE00015492A6846F25043C1F20003D1ED006A9B
:10DCF000D3ED6F7A92ED027A76EEA77A06F00106FE
:10DD000067EE877A7300FDEEE77A42F698511E447B
:10DD10000024C2F2000149F6C0104DF6514317EE3F
:10DD2000902A01EBC6010094C0F60200C0F6000381
:10DD300007F0FEFBC0E700BF043D0120AFF3008009
:10DD400080697047AFF30080AFF30080AFF30080CD
:10DD5000C0697047AFF30080AFF30080AFF300807D
:10DD6000D0ED007A90ED017AF8EEE77AB8EEC77A56
:10DD7000C7EE276A16EE900A704700BFAFF3008027
:10DD800010B50446FFF72CFF08B9E0612060206859
:10DD900010BD00BFAFF30080AFF30080AFF3008091
:10DDA00010B50446FFF71CFF08B9E0612060226847
:10DDB000002A0BDD41F6F403C2F200031B68B3F93D
:10DDC00068009042D4BF0020012010BD002010BD8B
:10DDD00041F6E803C2F200031868FFF7E1BF00BF95
:10DDE00041F6E803C2F200031B689869704700BF60
:10DDF00041F6E803C2F200032DE9F041D3F80080B8
:10DE0000064640460F46D8E90445FFF7E9FE18B933
:10DE1000C8F81C00C8F80000D8F80080B8F1000F5E
:10DE200016D030463946001B61EB0501F4F708FABD
:10DE300007EE108AF8EEC77A9FED087AC7EE277AC8
:10DE400007EE100AC7EE277A17EE900ABDE8F081B8
:10DE5000DFED037A17EE900ABDE8F081809FD54B85
:10DE60000000C07FAFF30080AFF30080AFF300800D
:10DE70002DE9F84341F6E806C2F2000681468846DD
:10DE8000376815F0E5FE4FF480533268CEF2000398
:10DE900002F50E525B6804460D461362B8F1000F9E
:10DEA0000AD041F6EC03C2F200031B68D3F810332A
:10DEB000012B3DD0BDE8F8833846FFF791FEC8B18D
:10DEC000D7E90423A21A65EB030352EA03013FD109
:10DED0004FF0FF323B683A603A687B60002A62DDAF
:10DEE000D7ED007A9FED367AF8EEE77AC7EE277A1B
:10DEF000C7ED027A41F6EC03BA69C2F200030132BF
:10DF00001B68BA61FA69D3F810330132012BFA6148
:10DF1000C7E904454CD033684FF4805203F50E53E3
:10DF2000CEF20002196A5268511A5962BDE8F883AC
:10DF3000FFF75EFF4FF47A7101FB098107EE901A3B
:10DF4000F8EE677ABDE8F84317EE901A03F048BC84
:10DF500041F6F401C2F2000146F2B7000968096E09
:10DF6000CBF20B6080FB01E00844C917C1EB202015
:10DF70004FF418414FEAE0794FEA400EC5F6D00160
:10DF800001FB09EEA0FB01017144F4F769FB47F2C4
:10DF900030539842C8BF4FF0FF303B6838603A6852
:10DFA0007B60002A9CDC0023C7F6C073BB60A1E73E
:10DFB00029462046FFF71CFF002103F011FCAAE7C9
:10DFC000ABC22248AFF30080AFF30080AFF3008014
:10DFD00010B549F6CC1104464DF6A1402246C0F6D4
:10DFE0000000C0F6020100F073FA4DF6716049F6C8
:10DFF000DC112246C0F60000C0F60201BDE8104068
:10E0000000F066BAAFF30080AFF30080AFF300809A
:10E01000019807EE102AD0ED027A67EE877A49F66A
:10E02000C010FDEEE77AC0F6020017EE902A07F066
:10E030007FBA00BFAFF30080AFF30080AFF3008082
:10E040002DE9F04F41F6F408C2F2000843F6B0564D
:10E05000D8F80030C2F2000687B007461868356865
:10E0600012F0F6FBD8F800308246D3F80402D3F859
:10E0700000B004F02DFBD8F8004042F62071C2F247
:10E080000101D4F80422034691F8E80D04920593A7
:10E0900016F0E6FFD8F80010044691F8DD05C0F34D
:10E0A000801016F0DDFF059B049A009342F6D059CC
:10E0B00049F6F011039001925B4628465246C0F69D
:10E0C0000201C2F20009029416F042FA49F6302128
:10E0D000D9F840313068D9F83C21C0F6020116F079
:10E0E00037FA97F88532002B40F08D81D7F8F44D40
:10E0F000D7F8EC2DD7F8F03D3068009449F6802130
:10E10000C0F6020116F024FAD8F8003097F885021C
:10E11000D3F80442356816F0A3FF49F6A021034660
:10E1200022462846C0F6020116F012FAD7F89002ED
:10E13000D6F800A0F3F750FC0446D7F894020D4639
:10E14000F3F74AFCCDE9000149F6C42122462B46EB
:10E15000C0F60201504616F0FBF997F884023568C4
:10E1600016F07EFF049002F05BFB16F079FF044688
:10E1700042F6D050C2F20000D9F83CB0D9F844A021
:10E1800001F066FED8F800308146B3F95000003047
:10E1900018BF012016F064FF49F6E0210390049AAD
:10E1A000CDF800B02346CDF804A0CDF8089028465D
:10E1B000C0F6020116F0CCF997F8842243F6B0536A
:10E1C000C2F20003002A40F0048141F6EC04C2F2DE
:10E1D000000435682368D3F8280109F019FE49F6D0
:10E1E00050310246C0F60201284616F0B1F9236804
:10E1F0003568D3F8600109F00BFE23688146D3F837
:10E200006C0104F055FB2268D2F8D02049F66C313D
:10E210000346009228464A46C0F6020116F098F9D5
:10E2200097F8853243F6B055C2F2000553B3236820
:10E23000D5F80080D3F82C0109F0EAFD49F69831B1
:10E240000246C0F60201404616F082F92368D5F86E
:10E250000080D3F8640109F0DBFD236842F6103535
:10E260008146C2F20005D3F8700104F021FBAD6CC9
:10E2700049F6B43103464A4640460095C0F60201CD
:10E2800016F066F92368D6F80080D3F8580209F032
:10E29000BFFD23680546D3F85C0204F009FB49F68C
:10E2A000E0312A460346C0F60201404616F050F916
:10E2B00023683568D3F8840109F0AAFD49F60041C6
:10E2C0000246C0F60201284616F042F92368346877
:10E2D000D3F8880109F09CFD49F618410246C0F6C2
:10E2E0000201204616F034F946F6502307F50D5486
:10E2F000C2F2000349F6344107F50E571B68E26B82
:10E300003068C0F6020116F023F949F654417A68E4
:10E310003068C0F6020116F01BF9616B626AE36AAD
:10E32000009149F66C413068C0F6020116F010F910
:10E33000796A7A69FB69009149F6A0413068C0F6B4
:10E34000020116F005F941F2DC2242F6C853C2F28E
:10E350000102C2F2000349F6C441306812681B682A
:10E36000C0F6020116F0F4F846F65823C2F2000394
:10E3700049F6F0411A683068C0F6020116F0E8F874
:10E3800049F24053C2F2000349F608511A68306856
:10E39000C0F6020116F0DCF846F6B843C2F20003FC
:10E3A00049F6245143F6B4541A683068C2F20004A6
:10E3B000C0F6020116F0CCF849F6385130682268F0
:10E3C000C0F6020116F0C4F80023236007B0BDE8D0
:10E3D000F08F07F6DC52D3F800801068F3F7FCFAF0
:10E3E00007F55E63044618680D46F3F7F5FACDE9C4
:10E3F000000149F63C31404622462B46C0F6020158
:10E4000016F0A6F8E1E649F65821C0F60201306898
:10E41000D9F84421D9F8483116F09AF866E600BFD9
:10E420002DE9F04343F6B057C2F2000783B0064629
:10E4300090F8E80D3C6816F013FE49F65851024674
:10E44000C0F60201204616F083F806F6DC53D7F832
:10E4500000901868F3F7C0FA06F55E630446186882
:10E460000D46F3F7B9FACDE9000149F63C312246F1
:10E470002B464846C0F6020106F5217816F068F8EA
:10E4800006F5616500240FE055F8040B3E68F3F7CC
:10E49000A3FACDE9000149F6645122463046C0F6A0
:10E4A000020116F055F80134404601F0B1FB8442F8
:10E4B000EADB03B0BDE8F083AFF30080AFF3008088
:10E4C00042F6D050C2F2000001F0B2BCAFF30080BF
:10E4D00038B5044649F670501546C0F602000FF0F4
:10E4E0007FFD21462A460248BDE8384016F068B94B
:10E4F000902E0020AFF30080AFF30080AFF30080D8
:10E5000038B500F1C005044601F0EAFC284616F0D3
:10E510003FF900230022C4E92E230021182204F52C
:10E520009E70F4F705FE284616F06AF9204638BDBD
:10E5300010B500210446182200F59E70F4F7F8FD8E
:10E540002046BDE8104001F06BBC00BFAFF3008077
:10E5500008B542F6D050C2F20000FFF7E9FF41F6DD
:10E56000E803C2F200031868BDE80840FFF768BD81
:10E570002DE9F04706460F4615F06AFB0B4641F6BB
:10E58000E801C2F200010246C6E92E23086806F03F
:10E590003FF806EB870341F2087ED3F83C210132B5
:10E5A000C3F83C21C2F2000ED6E92E45DEE9002375
:10E5B00053A1D1E90001A21A65EB0303994208BFF8
:10E5C00090423CBF0023337122462B4630463946E9
:10E5D000CEE9004502F074F93379002B4CD041F6B6
:10E5E000F405C2F2000530462B68D3F8E031012B68
:10E5F00044D001F00DFCDFF81091804643F69854AA
:10E60000C2F20004A01C414616F01AFE49F600634F
:10E61000C0F60203DB5D002B4CD049F6E053C0F698
:10E62000020343F6485053F827A0C2F200007523B6
:10E6300051462246237003F09BFA2B6893F8DD3590
:10E640005B065AD4D9F81030F26C9A4226D2D6F82A
:10E65000C030002BC4BF3546002429DDD5F8C430B6
:10E66000384641469847D6F8C0300134A34205F1F8
:10E670000405F3DCBDE8F087BDE8F08701F0E8FBB6
:10E68000DFF884900446304601F0C2FBE10754BF36
:10E69000D9F81030002300EB0308AFE749F68C519E
:10E6A000C0F6020140F25E20BDE8F04713F060B909
:10E6B000BDE8F08749F6E053C0F6020343F6485040
:10E6C00053F827A022466423C2F20000514623706B
:10E6D00003F04EFA2B6893F8DD355A06B2D5752350
:10E6E00043F6485043F698525146C2F20000C2F237
:10E6F0000002237003F03CFAA4E76423F0E700BFB4
:10E70000007A030A0000000000460120AFF30080F9
:10E71000F8B54FF4805243F6A85442F6C853C2F2FB
:10E720000004C2F20003CEF20002014657681868E6
:10E73000226842F6CC5641F2D8258242C2F2000647
:10E74000C2F2010542F6D050C8BF1A604FF0010E68
:10E750000132C2F200003760226085F800E0FFF766
:10E7600007FF4FF48052CEF2000243F6B453C2F2D8
:10E770000003576831681868266843F6AC52791A66
:10E78000C2F20002013E00278142116026602F7014
:10E7900088BF1960F8BD00BFAFF30080AFF3008001
:10E7A00043F6B053C2F2000342F628711868C2F271
:10E7B000000116F095BE00BFAFF30080AFF30080FC
:10E7C000014642F6D050C2F2000002F059B800BF34
:10E7D00038B549F6A85243F6B053C2F20003C0F66A
:10E7E00002021860126843F69853C2F20003150C37
:10E7F00043F648501A809D70C2F200000C4603F0A8
:10E8000037FA49F6AC504EF241012246C0F60200FA
:10E81000C0F6000116F054F849F6B8504EF2214106
:10E820002246C0F60200C0F6000116F049F849F68B
:10E83000CC504EF25151C0F60200C0F60001BDE8C6
:10E84000384016F06DB800BFAFF30080AFF3008022
:10E85000436AD3F8A031002B70B506460CDD074D96
:10E860000024284606F00CFA736AD3F8A03101346C
:10E87000A34205F11405F4DC70BD00BFBC6A0020A2
:10E88000436AD3F8A031002B70B506460CDD074D66
:10E890000024284606F0BCF9736AD3F8A03101348D
:10E8A000A34205F11405F4DC70BD00BFBC6A002072
:10E8B0002DE9F04F49F60043C2F201032DED048B20
:10E8C0001B7889B00C4623B109B0BDEC048BBDE8C0
:10E8D000F08F41F6E805C2F200052868FFF750FA0C
:10E8E00006460028F0D0471C00F0E68241F6F40707
:10E8F000C2F200073B68D3F8A831984200F3718157
:10E900002868FFF71DFA00F001000790002C00F0C6
:10E9100098823B6893F8DD25D3F8F01541F6F408AA
:10E920005006C2F2000802D5CA0700F1C5818C4228
:10E9300000F093822B68002C40F08A804FF48059BD
:10E94000CEF2000903F50E53D9F8042030469A6040
:10E9500004F04EFA2B68D9F80480396803F50E5C90
:10E96000D1ED8A7ADCF80820D1F8DCB1D1F860A0CA
:10E97000C2EB080806EE900ACCF80C80D9F8040027
:10E9800066EEA77A42F6207803F50D52C2F201082E
:10E99000C8ED9C7A9062BBF1000F00F080810AEB19
:10E9A000DA7A4FEA6A0A07EE10AAB8EEC78AD3ED00
:10E9B0009D7AF5EE407AF1EE10FA00F09A82B4EE0C
:10E9C000E78AF1EE10FA00F184820022D3F878127F
:10E9D000C7F6C07291423FF477AF07999A6AD3F8AD
:10E9E000780241F6086E0EFB01FED3F874120EF6A3
:10E9F000C8631A4418F0DCFB2B684FF4805203F50F
:10EA00000D53CEF20002996A5068411AD9625268D9
:10EA1000002E1A633B6804DDB3F968209642C0F209
:10EA2000A982D8F82800D3F8B0214DF6E02100F2F1
:10EA30004470C1F2000118F0ABFC2B684FF4805118
:10EA400003F50D52CEF20001106B4968081A5063AD
:10EA5000586A18F0BDFE002800F0D280002E40F366
:10EA600036813B68B3F968309E4280F2308142F6CD
:10EA70002073C2F201032868D3F828B00BEB04031B
:10EA800093F84436002B00F0BC8000F5AE7004F023
:10EA90001FFC2868483004F02BFC304604F0A8F92D
:10EAA0003B68DBF80020D3ED8A7A06EE900A41F647
:10EAB000E80342F6207866EEA77AC2F20003C2F2BB
:10EAC0000108002AC8ED9C7AD8BF186840F39980E5
:10EAD0009FEDD09AD9464FF0000A039606E00AF15E
:10EAE000010A924509F1140980F28980D9F80430AD
:10EAF0009C42F4D198ED9C8A002318EE101AC7F6B8
:10EB0000C073994200F07582B5EEC08AF1EE10FA3A
:10EB100000F17A822B6803F5F4531B7E002BDED1C3
:10EB200042F62072C2F2010292ED027AD9ED037A26
:10EB300099F8143067EE278A002B00F07682B5EE44
:10EB4000C08AF1EE10FA00F19482D9F810C0CDF825
:10EB500010C0FFF745F900EBD07303F00103A3EBFE
:10EB6000D07041F6E803C2F2000300EB40001A68DF
:10EB7000DDF810C000924FEAC00EFDEEE88A0EF1FB
:10EB8000080149F6F8600EF1380E4EF68103614433
:10EB9000C0F60200F444C0F6000318EE902ACDF847
:10EBA00010C006F0C5FCF8EEE87A41F6E806E8EE9B
:10EBB000097AC2F20006DDF810C03668FDEEE77A89
:10EBC00049F600704EF6510317EE902A6146009602
:10EBD000C0F60200C0F6000306F0AAFCDBF8002035
:10EBE0007DE749F620610246C0F6020140F25E2050
:10EBF00009B0BDEC048BBDE8F04F12F0B9BE039E26
:10EC00002868721E47F22E539A42D0F828803FF6A9
:10EC10005BAE3B6893F8DC359B077FF555AE43F65A
:10EC2000B85BC2F2000BDBF80010002957D08B6CE8
:10EC3000069542F62077C2F201079C42BA46D946B1
:10EC40004F6D06D0002F49D039468B6C4F6D9C42DA
:10EC5000F8D1DBF80020914208BFC9F8007003D159
:10EC600005E0994238D01A46536D002BF9D1D1ED09
:10EC7000147A9AED027A67EE277A0D68FDEEE77A4C
:10EC800049F60C7044F6814317EE902A0095203126
:10EC9000C0F60200C0F6010306F04AFCD2E7D1F844
:10ECA000A0219AFBF2FA07EE90AAB8EEE77ADFED20
:10ECB0005A7A87EE278A7AE649F64060C0F6020063
:10ECC00019F076F8D8F80030D3F8F0152FE6286858
:10ECD000836A03F2447BD1E65765C8E7069D07992E
:10ECE00041F6086303FB01F303F6C86308EB030A6C
:10ECF00058F80330002B7FF7E7AD44F6E83CC2F24A
:10ED0000000CCDF818B00AF108090AF150074FF0CD
:10ED10000008E3460AE0DAF8003008F101089845F7
:10ED200009F1600907F16007BFF6CEAD57F80C3C5A
:10ED30009C42F0D12A6802F5F35318680023C7F605
:10ED4000C073984271D006EE900AF5EEC06AF1EEFB
:10ED500010FA6AD492ED027ADBF80031DBF8082170
:10ED6000013357ED017ACBF80031DBF8001144F69E
:10ED7000E8339142C2F2000367EE277A04BF002213
:10ED8000C3F80021F5EEC07ADBF80021F1EE10FAAD
:10ED900054BF002301234BF82230DBF80421013259
:10EDA000CBF80421002B40F0D18057F8482CFDEE21
:10EDB000E77A49F6307044F61143C0F60103009239
:10EDC000C0F60200A7F1400117EE902A06F0B0FB52
:10EDD000384657F8101C18F07BF9D9F848309C4297
:10EDE00000F0EC80069A1168002900F051818945F5
:10EDF0001CBF0B464FF47A7206D1D6E0013A00F000
:10EE00002681994500F0D1805B6D002BF6D1FB6027
:10EE10000A4604E000007A44CDCC8C3F1A46536D7C
:10EE2000002BFBD1C2F8549075E7F2F7D5FD0246EE
:10EE300049F664600B460096C0F6020018F0B8FF71
:10EE400069E743F6C050C2F2000016F0A1FB0028AB
:10EE50003FF45FAD18F0ACFB5BE5D3F85406B0F5BA
:10EE60005E7F52D12B684FF48052DFF82CC2CEF275
:10EE70000002DCF80000D2F804E0002103F50D5296
:10EE8000C7F6C0718842C2F820E07ED007EE100AB3
:10EE9000B5EEC07AF1EE10FA77D4DCED017AF1EE3E
:10EEA000677AC3ED9E7A70464FF48051CEF200012E
:10EEB0004968091A51623EE549F61061C0F602013F
:10EEC00040F2551009B0BDEC048BBDE8F04F12F0D4
:10EED0004FBD17EE900AF2F77FFD0B4649F68C61A5
:10EEE0000246C0F6020140F25E2012F041FD2B689E
:10EEF0006BE549F67C61C0F6020140F25E2012F03B
:10EF000037FD2B68D3ED9D7A59E50AF071FC06EECA
:10EF1000900ADFED607A3A682B68B8EEE67A93F8EB
:10EF2000801227EE277AD2ED6E7A27EE277AF0EE5E
:10EF3000047AB4EEE77AF1EE10FAD4BF002201228F
:10EF4000114383F87F2283F880128CE743F6C45381
:10EF5000C2F2000317EE900A1B680793F2F73CFD1C
:10EF60000B4649F618710246C0F60201079815F0E3
:10EF7000EFFAD0E64CF69001D8F82800D3F8AC218F
:10EF8000C1F2000118F004FA57E5F2F725FD024638
:10EF900049F664600B46C0F60200009618F008FFC0
:10EFA0002B6803F50D52106A7EE749F65871C0F6DA
:10EFB000020140F25E2012F0DBFCACE62B6857F851
:10EFC000481C93ED027AD7ED027A67EE277A49F66C
:10EFD0003C70FDEEE77A44F68143009117EE902AEB
:10EFE000C0F60200C0F60103A7F1280106F0A0FA5E
:10EFF00091E649F6A861C0F6020140F25E2012F0E7
:10F00000B7FCDBF800206AE518EE100AF2F7E4FC22
:10F010000B4649F6BC610246C0F6020140F25E2092
:10F0200012F0A6FCDBF8002059E5D9F8106014F0C6
:10F03000FFFD28EE098A02460B4630468DED018A17
:10F04000CDED008A05F06CFEDBF8002047E549F6BF
:10F050004870C0F60200049218F0AAFE0699049ABD
:10F060000B68FA60002B7FF4D9AE069AC2F80090C4
:10F0700051E618EE100AF2F7AFFC024649F6D860E6
:10F080000B46C0F6020018F093FEDBF8002026E5E0
:10F09000F960EAE7010C403A804D0120AFF30080AF
:10F0A000F0B583B00746FEF76BFE054617F050FF3C
:10F0B000F2F792FC43F6C454CDE90001C2F2000419
:10F0C00049F67C712A462068C0F6020115F040FA24
:10F0D0002846266803F08CFEF2F77EFC07F5F3570E
:10F0E000044678680D46F2F777FCCDE9000149F651
:10F0F0009471304622462B46C0F6020115F028FADC
:10F1000003B0F0BDAFF30080AFF30080AFF3008039
:10F1100008B5FFF745FB43F6C453C2F2000343F6BC
:10F12000C8511868C2F2000116F0DAF9BDE80840CB
:10F1300002F096BDAFF30080AFF30080AFF3008024
:10F14000F8B543F6C454C2F2000443F6BC550E466B
:10F150002060C2F2000549F6A8704FF21111C0F606
:10F160000200C0F600012E6015F0DAFB49F6B87017
:10F170004FF2A1013246C0F60001C0F6020015F0C0
:10F180009FFB276814F06CFD49F6C4710246C0F677
:10F190000201384615F0B4F92B68586A18F018FBCC
:10F1A00030B949F6D8712068C0F6020115F0A8F907
:10F1B0004EF6B1004AF200013246C0F60000C0F639
:10F1C0000201BDE8F840FFF783B900BFAFF300804C
:10F1D00070B444F6E835C2F20005D5F80431052BC9
:10F1E0001EDCD5F80461D5F80011002ED8BF002030
:10F1F00014DD0024D5F80821204600290B4601DA49
:10F200009B18FDD455F823300130B0421C4401F165
:10F21000FF31F2DB042CD4BF0020012070BC70470A
:10F22000D5F800110626E4E7AFF30080AFF30080C5
:10F2300038B502212DED048B0122044600F018FDA3
:10F2400046F6C9112046C3F6BE710122002300F024
:10F2500087FFDFED548A9FED549A1725012213464C
:10F2600018EE901A204600F07BFF78EE898A20463F
:10F2700018EE901A0122002300F072FF013DDFED2D
:10F280004A9A78EE898AE9D19FED488A78EE888A91
:10F29000012218EE901A1346204600F061FF38EE66
:10F2A000888A2B4618EE101A2046012200F058FFDB
:10F2B00038EE298AF0EE698A24250122134618EED9
:10F2C000101A204600F04CFF38EE288A204618EE2F
:10F2D000101A0122002300F043FF013D38EE288A76
:10F2E000EBD100212A462046C4F2BC31012300F0B4
:10F2F00037FFDFED2D8A15250122134618EE101A6F
:10F30000204600F02DFF38EE288A204618EE101A0D
:10F310000122002300F024FF013D9FED239A38EEE7
:10F32000288AE9D1DFED218A38EE288A012218EEF9
:10F33000101A1346204600F013FF38EE288A2B4699
:10F3400018EE101A2046012200F00AFF38EE098A52
:10F35000F0EE498A21250122134618EE101A2046A4
:10F3600000F0FEFE38EE288A204618EE101A012220
:10F37000002300F0F5FE013D38EE288AEBD1012292
:10F38000134618EE101A204600F0EAFE002120462F
:10F39000C4F234412A462B4600F0E2FEBDEC048B59
:10F3A000257038BD57CF8E40C9693E4057CF0E41BA
:10F3B00070B501220221044600F05AFC4FF4D551E9
:10F3C0002046C3F6BF710125002601F081F84DF2F9
:10F3D000747120462A462B4684F8646B2570C4F26B
:10F3E000532100F0BDFE44F29C5120462A4633468C
:10F3F000C4F2F52100F0B4FE4EF2A451204632468C
:10F400002B46C4F2583100F0ABFE4AF2DB31204605
:10F410002A462B46C4F2683100F0A2FE46F6EC0103
:10F42000204632463346C4F2903100F099FE45F250
:10F43000BB2120462A463346C4F2973100F090FEA5
:10F4400043F65A1120462A462B46C4F2CE3100F02C
:10F4500087FE46F68A0120462A463346C4F2F13139
:10F4600000F07EFE44F24621204632462B46C4F28E
:10F47000104100F075FE43F6330120462A462B4624
:10F48000C4F2144100F06CFE4BF6951120462A465A
:10F490003346C4F2254100F063FE00212046324687
:10F4A0003346C4F23441BDE8704000F059BE00BF9D
:10F4B00070B544F2AE7104460025C3F6E15101F087
:10F4C00007F8204684F8645B0221012200F0D0FB9B
:10F4D000002120462A46C4F2A011012300F040FE7C
:10F4E000002120462B46C4F28421012200F038FE80
:10F4F0000122002120461346C4F28C2100F030FE88
:10F50000002120462B46C4F20831012200F028FEDB
:10F510000122002120461346C4F20C3100F020FEE7
:10F52000002120462B46C4F27631012200F018FE5D
:10F530000122002120461346C4F27A3100F010FE69
:10F54000002120462B46C4F29E31012200F008FE25
:10F550000122002120461346C4F2A03100F000FE33
:10F56000002120462A462B46C4F2AA3100F0F8FDBD
:10F57000002120462A46C4F2B431012300F0F0FDF8
:10F58000002120462A462B46C4F2BE3100F0E8FD99
:10F59000002120462A46C4F2C831012300F0E0FDD4
:10F5A000002120462B46C4F2D531012200F0D8FDBF
:10F5B0000122002120461346C4F2D73100F0D0FDCD
:10F5C000002120462B46C4F2F831012200F0C8FD8C
:10F5D0000122002120461346C4F2FA3100F0C0FD9A
:10F5E0004FF4004120462B46C4F21741012200F09F
:10F5F000B7FD01224FF4004120461346C4F21841E2
:10F6000000F0AEFD002120462B46C4F22941012224
:10F6100000F0A6FD0122002120461346C4F22A4133
:10F6200000F09EFD002120462A462B46C4F23441BC
:10F63000BDE8704000F094BDAFF30080AFF30080F0
:10F6400010B502210022044600F012FB41F27B417A
:10F650002046C4F2E2210022012300F081FD0022B5
:10F66000002113462046C4F2343100F079FD48F2FF
:10F670001F512046C4F292310022012300F070FD98
:10F680000022002113462046C4F2B43100F068FD88
:10F6900048F21F512046C4F2EC310022012300F051
:10F6A0005FFD0022002113462046C4F2074100F00E
:10F6B00057FD44F28F212046C4F22341002201234A
:10F6C00000F04EFD0022002113462046C4F23441D2
:10F6D00000F046FD0023237010BD00BFAFF3008093
:10F6E00010B502210122044600F0C2FA4AF6940144
:10F6F0002046C4F2BE210022012300F031FD012288
:10F7000046F6721113462046C4F2DC2100F028FDB3
:10F7100040F2D7512046C4F232310122002300F0DA
:10F720001FFD002247F2CB2113462046C4F2683168
:10F7300000F016FD01224DF6922113462046C4F238
:10F740008F3100F00DFD47F25E112046C4F2B23158
:10F750000122002300F004FD012243F2E7111346C9
:10F760002046C4F2EA3100F0FBFC4BF24651204641
:10F77000C4F206410122002300F0F2FC01224AF605
:10F78000763113462046C4F2224100F0E9FC002104
:10F79000C4F2344101220023204600F0E1FC41F68E
:10F7A000816104F53662C4F20931002311602370CF
:10F7B00010BD00BFAFF30080AFF30080AFF3008057
:10F7C00070B502210446002200F052FA0025012300
:10F7D000002184F8643B20462A462570C4F2074184
:10F7E00000F0BEFC002120462A462B46C4F23441DC
:10F7F000BDE8704000F0B4BCAFF30080AFF3008010
:10F8000070B5022104460022012500F031FA41F2D0
:10F81000CB0144F69842204684F8645B84F8655B2B
:10F82000C3F6FF71C4F2BF0200F042FE41F23D2177
:10F8300020462B46C4F20F31002200F091FC00223A
:10F840004AF64E7120461346C4F2363100F088FC69
:10F8500046F6964120462B46C4F25731002200F06E
:10F860007FFC002241F6AB7120461346C4F2803182
:10F8700000F076FC45F27B4120462B46C4F29031E5
:10F88000002200F06DFC002246F29D312046134616
:10F89000C4F2A33100F064FC4CF2D42120462B4684
:10F8A000C4F2B431002200F05BFC002247F6EF21E5
:10F8B00020461346C4F2FE3100F052FC46F6A40185
:10F8C00020462B46C4F20841002200F049FC0022E9
:10F8D0004BF6467120461346C4F2114100F040FC3D
:10F8E00044F6B76120462B46C4F21A41002200F0CC
:10F8F00037FC002245F6B80120461346C4F22341E6
:10F9000000F02EFC40F2E96120462B46C4F22B4168
:10F91000002200F025FC0022002120461346C4F2FC
:10F920003441BDE8704000F01BBC00BFAFF3008065
:10F9300070B501220221054600F09AF945F2EC115A
:10F940002846C3F638710124002600F0C1FD0021CD
:10F9500028462246234685F8646BC5F8804BC4F2DE
:10F96000202100F0FDFB0021284622463346C4F248
:10F97000302100F0F5FB0021284622462346C4F240
:10F98000602100F0EDFB0021284622463346C4F2F8
:10F99000702100F0E5FB0021284622462346C4F2F0
:10F9A000A62100F0DDFB0021284622463346C4F2A2
:10F9B000B02100F0D5FB0021284622462346C4F2A0
:10F9C000DE2100F0CDFB0021284622463346C4F25A
:10F9D000E82100F0C5FB0021284632463346C4F238
:10F9E000203100F0BDFB0021284622462346C4F208
:10F9F000343100F0B5FB0021284622463346C4F2DC
:10FA00005C3100F0ADFB0021284622462346C4F2BB
:10FA10006B3100F0A5FB0021284622463346C4F294
:10FA20006F3100F09DFB4FF40041284622462346EB
:10FA3000C4F2823100F094FB00212846224633466E
:10FA4000C4F2853100F08CFB002128462246234673
:10FA5000C4F2913100F084FB4FF400412846224665
:10FA60003346C4F2933100F07BFB00212846324636
:10FA70002346C4F2B43100F073FB0021284622462D
:10FA80002346C4F2C63100F06BFB4FF40041284618
:10FA900022463346C4F2C73100F062FB00212846FB
:10FAA00022462346C4F2CD3100F05AFB4FF4004108
:10FAB000284622463346C4F2CF3100F051FB4FF4C2
:10FAC0000041284622462346C4F2DA3100F048FBC2
:10FAD0000021284622463346C4F2DD3100F040FBC7
:10FAE0004FF40041284622462346C4F2E83100F094
:10FAF00037FB0021284622463346C4F2EB3100F0A2
:10FB00002FFB4FF40041284622462346C4F205410C
:10FB100000F026FB4FF44041284632463346C4F2FB
:10FB20000A4100F01DFB4FF40041284622463346AF
:10FB3000C4F2104100F014FB00212846224623465F
:10FB4000C4F2154100F00CFB4FF4804128462246D8
:10FB50003346C4F2164100F003FB4FF440412846FF
:10FB600022462346C4F21B4100F0FAFA002128463F
:10FB700022463346C4F21D4100F0F2FA0021284625
:10FB800022462346C4F2234100F0EAFA4FF48041B2
:10FB9000284622463346C4F2244100F0E1FA00210F
:10FBA000284632462346C4F23441BDE8704000F096
:10FBB000D7BA00BFAFF30080AFF30080AFF300808F
:10FBC000F8B5044600F53D7704F53E76384615F065
:10FBD000EFFC04F53F75304615F0EAFC284615F0B9
:10FBE000E7FC3846214615F0F3FC304604F1FC01F1
:10FBF00015F0EEFC284604F5FC7115F0E9FC2046F2
:10FC0000F8BD00BFAFF30080AFF30080AFF300801A
:10FC100000F5A350C0687047AFF30080AFF30080D9
:10FC20002DE9F00100F5A35100F5366600F65835D0
:10FC300000F65C3400274FF000080122C4F22007D0
:10FC400000234FF07F5CC6F800800270C5F800C04A
:10FC5000276080F8642BBDE8F0010B7280F8653BEB
:10FC6000704700BFAFF30080AFF30080AFF30080B8
:10FC7000F8B5044600F5BB5300F5DB5600F5A35775
:10FC80000025B16003F11400FD60294662701D611A
:10FC90004FF47C7284F8805B84F8815B84F8825B2B
:10FCA00084F8835B84F8845B84F8855B84F8865BE6
:10FCB00084F8875B84F8885B84F8895B84F88A5BC6
:10FCC00084F88B5BF3F734FA84F8685B84F8695B3B
:10FCD00084F86A5B84F86B5B84F86C5B84F86D5B1A
:10FCE00084F86E5B84F86F5B84F8705B84F8715BFA
:10FCF00084F8725B84F8735B04F6743015F088FC4A
:10FD000000237360F8BD00BFAFF30080AFF3008045
:10FD1000F8B5044600F5BB5505F11401002204F5C1
:10FD2000A35600F6743015F063FC06F11000FFF7DF
:10FD300047FF002120460A46FFF79AFF04F65C3C85
:10FD400004F6583E04F536620023291D4FF47C77F3
:10FD50000025C4F8781B84F8645B84F8655B257023
:10FD60002946357204F68C3013606560A5603A460A
:10FD7000CCF80030CEF80030F3F7DAF904F5835010
:10FD80003A4629461830F3F7D3F9294604F67C7031
:10FD9000FC22F3F7CDF9294604F118004FF4346240
:10FDA000F3F7C6F92046F8BDAFF30080AFF300804B
:10FDB000436853F821309856704700BFAFF3008076
:10FDC000F8B5171E06460D46C8BF002403DC0DE03B
:10FDD0000134BC420AD0B36803EB84032946186897
:10FDE00015F03EFA0028F3D02046F8BD4FF0FF3062
:10FDF000F8BD00BFAFF30080AFF30080AFF3008029
:10FE0000836803EB81010A60704700BFAFF3008095
:10FE1000C06C7047AFF30080AFF30080AFF3008099
:10FE20000023036503648364704700BFAFF3008061
:10FE300030B4D0E92623C06C141843F100052046E5
:10FE4000294630BC704700BFAFF30080AFF300809D
:10FE5000D0F8A000704700BFAFF30080AFF3008080
:10FE600070B500251826044680F8545080F8555087
:10FE700080F8565080F8575080F8585080F8595004
:10FE800080F85A5080F85B5080F85C5080F85D50E4
:10FE900080F85E5080F85F50294632466430F3F7B0
:10FEA00047F9324604F180002946F3F741F92576F7
:10FEB0006576A576E57625776577A577E57784F885
:10FEC000205084F8215084F8225084F82350E564AF
:10FED00070BD00BFAFF30080AFF30080AFF30080D0
:10FEE000F8B50027064600240025076007718760E3
:10FEF000C0F8A070C7634764C76080F8607080F87E
:10FF00006170076507648764C0E90445C0E92A4554
:10FF1000C0E92C45FFF7A4FF012386F8307086F86E
:10FF2000317086F8327086F8337086F8347086F84F
:10FF3000357086F8367086F8377086F8387086F82F
:10FF4000397086F83A7086F83B70C6E9264586F81F
:10FF5000A4303046F8BD00BFAFF30080AFF300809F
:10FF600000F5DB5300F5A3509B68C068022B18BF57
:10FF700040007047AFF30080AFF30080AFF3008024
:10FF800000F5DB5208B59268022A1DD000F5A35295
:10FF900000F67430D26891420BDB891A15F040FBF1
:10FFA000DFED107A07EE100AE7EE277A17EE900AD7
:10FFB00008BD15F035FBDFED0B7A07EE100A67EE92
:10FFC000277A17EE900A08BD00F6743015F028FB6A
:10FFD000DFED057A07EE100A67EE277A17EE900A32
:10FFE00008BD00BF0000B44300003444AFF30080FC
:10FFF0002DE9F04F41F6F408C2F200082DED028B16
:020000040801F1
:10000000D8F8001085B001F50171064601F0C0F87E
:1000100041F6E80706F5DB52C2F20007014606F595
:10002000A35390683A6801930228D86802F5F45205
:1000300006F5BB5A18BF4000CAF81010D061304610
:10004000FFF79EFF3A6802F5F45208EE900AD06975
:10005000002823DD06F68C3346F2504BC1F2000B2C
:10006000029300241D469FED398A06F58353D94635
:1000700022460393C346B4B9029B83ED008A039BD7
:1000800006F5396181ED008A9C61396801F5F4510A
:100090000134C869A04205F10405ECDC05B0BDECF3
:1000A000028BBDE8F08FDAF81010DDF804E021448F
:1000B000DEF80C30009291FBF0FE00FB1E1199421D
:1000C0003046ACBFC3EB01088846FFF759FF06EE88
:1000D000900A76EEE87AD9ED1A6AF5EEC07AF1EE7A
:1000E00010FA009AB8EEE67A0DD577EE877AF5EE3B
:1000F000C07AF1EE10FAF8D4B4EEE77AF1EE10FA25
:1001000006D877EEC77AB4EEE77AF1EE10FAF8D9AE
:10011000DBF8001091F8DD154B0658BFC5ED007AED
:1001200010D5B04498F97C1F61B102F5397002F224
:10013000E52106EB800006EB8101C0ED017AC1EDFF
:10014000017A0232C5F8EC249FE700BF00000000EE
:1001500000F5DB5080687047AFF30080AFF300809C
:100160002DE9F04F00F5A3562DED028B9046327A23
:1001700089B005461F4608EE101A002A00F0E180FB
:10018000D3F1010338BF0023039305F5DB54A068C6
:1001900000F08EFD41F6F403C2F2000307EE900A70
:1001A0001B6893F8DD355B0688EE278A40F1958061
:1001B000012F00F09280F268002A40F39980D4ED7C
:1001C000018AB4EEE88AF1EE10FA88BF84ED018A64
:1001D00040F2C48005F67433184618EE101A0293E4
:1001E000FFF7EEFD411C029B40F0AD80F168B1F1DC
:1001F000010A00F1E880D5F87C0B4FEA8A0C6044D4
:10020000D0ED007AB4EEE78AF1EE10FAD8BF52468C
:1002100008DDBCE070ED017AB4EEE78AF1EE10FA89
:1002200000F3B68012F1FF32F4D20020059006925E
:10023000834604900CF10409049C07965E46CB4665
:1002400099460AF101000023D5F8782BD2580433DF
:10025000915D0C2B1154F7D15146484615F0E0F949
:10026000D5F87C3B0AF1FF3A5B44A2451860ABF13C
:10027000040BE6DAB346079EF168049B7A1E2B4412
:100280005742574183F87C7F049B8B4206D04AF249
:100290007400C0F6020017F08BFDF168013106987A
:1002A000F1600023D5F8782BD2580433115C0C2B65
:1002B00002F80B10F6D1D5F8783BD5F87C1B059ADF
:1002C00053F828300398114481ED008A03F80B009D
:1002D00009B0BDEC028BBDE8F08F05EB8803D3F8C5
:1002E000682B0132C3F8682BF268002A3FF767AF2A
:1002F00084ED018A7FF46EAF0123F360D5F8783B7B
:100300009918A818002954D09B580432002B55D0B6
:10031000D0F8801B0C2A1970F0D1781E4742D5F80E
:10032000783BD5F87C2B474185F87C7F53F8283003
:10033000039882ED008A187009B0BDEC028BBDE80D
:10034000F08F039321E74AF25800C0F6020009B08B
:10035000BDEC028BBDE8F04F17F02ABD18EE100A75
:10036000F1F73AFB044618EE900A0D46F1F734FB1C
:10037000CDE900014AF2100022462B46C0F60200E9
:1003800017F016FD09B0BDEC028BBDE8F08F5246A8
:10039000501C82450692B8BF82000490BCBF8346C1
:1003A0000592FFF66AAFDDF810B04FEA8B020592B6
:1003B00040E74AF23000C0F60200C8E74AF24000C7
:1003C000C0F60200C3E7002205920690934604920D
:1003D00053E700BFAFF30080AFF30080AFF30080BE
:1003E00007EE901A9DED007AF4EEC77AF1EE10FA5E
:1003F000DDED016A04DDF4EEE67AF1EE10FA00D4E8
:100400007047FFF7ADBE00BFAFF30080AFF30080D1
:1004100010B52DED028BB1EE0E8A70EE088A022225
:1004200018EE901A01230446FFF79AFE38EE888AE8
:10043000204618EE101A02220023FFF791FEB2EEBA
:100440000E0A38EE000ABDEC028B10BDAFF300803F
:1004500010B501222DED028B10EE101AF0EE408A3D
:100460001346B2EE0E8A0446FFF77AFE78EE888ACB
:10047000204618EE901A01220023FFF771FE38EE95
:10048000880ABDEC028B10BDAFF30080AFF3008093
:1004900083680846194615F0CBB800BFAFF300805B
:1004A00010B4012480F8644B5DF8044B00F088BC64
:1004B00030B400F65C3300F6583401250570216035
:1004C0001A6030BC704700BFAFF30080AFF300800C
:1004D00007EE901AB6EE087AF7EE046A27EE877AEE
:1004E00067EEA67A012100F6583200F65C330170FF
:1004F00082ED007AC3ED007A704700BFAFF3008051
:1005000070B50122044615460221FFF7B1FB2046D3
:10051000C4F8845B9FED590AFFF77AFF0026204656
:10052000FFF776FFC4F2B4262046FFF771FF31468D
:100530002A4600232046FFF713FE204600EE106AED
:10054000FFF766FF00262046FFF762FFC4F234364D
:100550002046FFF75DFF31462A462B462046FFF72F
:10056000FFFD204600EE106AFFF752FF00262046EE
:10057000FFF74EFFC4F287362046FFF749FF3146AA
:100580002A4600232046FFF7EBFD204600EE106AC6
:10059000FFF73EFF2046FFF73BFF2046FFF738FFFF
:1005A00000264FF48041C4F2B43620462B46C4F2F4
:1005B000B0310022FFF7D4FD31462A462B462046B3
:1005C000FFF7CEFD204600EE106AFFF721FF002660
:1005D0002046FFF71DFFC4F2E1362046FFF718FF63
:1005E00031462A4600232046FFF7BAFD204600EE9A
:1005F000106AFFF70DFF00262046FFF709FFC4F23F
:1006000007462046FFF704FF31462A462B46204680
:10061000FFF7A6FD204600EE106AFFF7F9FE4FF443
:1006200000462046FFF7F4FEC4F21D462046FFF7C1
:10063000EFFE2A46314600232046FFF791FD204673
:1006400000EE106AFFF7E4FE2046FFF7E1FE2046C9
:10065000FFF7DEFE00224FF4005113462046C4F29D
:100660003241FFF77DFD00212B4620462A46C4F289
:100670003441FFF775FD0023237070BD00000000BA
:1006800070B504462DED048B01220E460025022193
:10069000FFF7EEFA25702046B1EE040AFFF7D8FE08
:1006A000B0EE408A002E40F090802046FFF7D0FE4A
:1006B0002046FFF7CDFEB0EE408AB0EE480A204655
:1006C000FFF7C6FE2046FFF7C3FE4AF2C501B0EEB3
:1006D000408AC4F21231002201232046FFF740FD78
:1006E0002046B0EE480AFFF7B3FE00220021134671
:1006F000C4F23431B0EE408A2046FFF731FD204687
:10070000B0EE480AFFF7A4FE2046FFF7A1FE204600
:10071000FFF79EFE2046FFF79BFE2046FFF798FE60
:1007200045F26201C4F2A33100220123B0EE408AF7
:100730002046FFF715FD2046B0EE480AFFF788FE79
:100740000022002120461346C4F2B431F0EE408A64
:10075000FFF706FDDFED2C9A9FED2C9A0325B0EEF6
:10076000680A2046FFF774FE2046FFF771FE204618
:10077000FFF76EFE2046FFF76BFE2046FFF768FE90
:1007800007EE905AB8EEE78AF0EE408A28EE298A02
:10079000002278EE497A012317EE901A2046FFF7DF
:1007A000DFFC2046B0EE680AFFF752FE002220462A
:1007B00018EE101A01351346F0EE408AFFF7D0FC10
:1007C000052DCCD1BDEC048B70BDF1EE0E8A70EE20
:1007D000687A022217EE901A01232046FFF7C0FC28
:1007E0002046B0EE480AFFF733FE2046FFF730FE02
:1007F00070EE688A20462B4618EE901A0222B0EE60
:10080000408AFFF7ADFC58E700003443ED7C054219
:1008100000F118010EC9016342638363704700BF92
:1008200070B444F60855C2F20005D5F80431052B22
:100830001EDCD5F80461D5F80011002ED8BF0020C9
:1008400014DD0024D5F80821204600290B4601DAE2
:100850009B18FDD455F823300130B0421C4401F1FF
:10086000FF31F2DB042CD4BF0020012070BC7047A4
:10087000D5F800110626E4E7AFF30080AFF300805F
:1008800008B500EB81012DED028B91ED098ADFEDBA
:10089000097AB8EE488AD0E92A0128EE278AF1F7CA
:1008A000CFFC07EE100A88EE077ABDEC028B17EE3C
:1008B000100A08BD0000C842AFF30080AFF300800B
:1008C0002DE9F04F41F6F408C2F200084AF2900711
:1008D000D8F800C09CF8DD95C0F602078BB019F07F
:1008E000400FCDE90623064617F801A090F86030C6
:1008F00006D190F861209A4202BF426C01324264F4
:1009000006EB8A0986F8613086F86010D9F8542021
:1009100006EB81030132C9F854205A6E01325A663F
:1009200096F8A430002000247BB9D6E90423DDE941
:100930000645A41A65EB0305CAA3D3E90023AB421D
:1009400008BFA24238BF1446204642F62077C2F2C2
:100950000107F06097F8E80D002849D1002949D136
:1009600097F884124FF0000B86F8A4B000296FD0DE
:1009700096ED026ABA4BF8EE467AD3ED006A06EEBF
:10098000104A67EEA66AB8EEC67AB4EEE67AF1EEE1
:1009900010FA0CDDD3ED016A67EEA66AB4EEE67AD2
:1009A000F1EE10FA54BF4FF0000B4FF0010B9CF822
:1009B000DD35180700F10681BBF1000F40F03281F0
:1009C00006EBCA0ADAE9202352EA030140F0EE807E
:1009D000DDE90601CAE92001D8F8003093F8DD35D9
:1009E00013F0400FF36C18BF01330133F364CCE014
:1009F0000129B5D006EBCA0ADAE9202352EA03043A
:100A00001AD1DDE90623CAE920239CF8DD35F26C12
:100A10005C0648BF013297F8E93D0132F26443B108
:100A2000DDE90601F368C6E904010022B36086F837
:100A3000A4200BB0BDE8F08FD9F818300698034415
:100A40009A1A00200021C9F81820CAE92001DCE721
:100A50009CF8DD253379DFF814B212F0400F0CBF9B
:100A600001220222002B40F09980716DD7F8EC2D05
:100A700042F620739142C2F2010300F0BE8044F6B8
:100A8000F440C2F20000012104F05AFC13F0E0F837
:100A9000F36BD8F800200133F36392F8DD2541F2BF
:100AA0001073C2F20003C3E90001130700F1E080F4
:100AB000012044F60853C2F20003D3F80011D3F822
:100AC00008210131C3F80011D3F80011914204BF8D
:100AD0000022C3F80021D3F8002143F82200D3F804
:100AE00004210132C3F80421FFF79AFE002840F0E8
:100AF000A180012306EBCA0A3371DAE9202352EA06
:100B0000030000F09280D9F8183006990B449A1A25
:100B100000200021C9F81820CAE92001D8F80030C7
:100B2000F26C93F8DD35590648BF01323368013263
:100B3000F2640BB130469847334606F1240053F86F
:100B4000187F59689A68776241608260D6E92C23E1
:100B5000DDE90601821A61EB0303C6E92C01C6E94F
:100B60002A233046FFF77CF9D6E92623DBF81070FC
:100B7000D6F8A000316DD21943EBE773C6E92623FE
:100B800001300131C6F8A0003165DDE90601F368E6
:100B9000C6E90401B3600BB0BDE8F08FDBF81010BC
:100BA000F36C8A1A9342BFF460AF09E7D9F81830A2
:100BB000069C23449A1A00200021C9F81820CAE98B
:100BC000200109E7C7EE276A44F60453C2F2000386
:100BD0001C6816EE900AF0F7FFFEF56C0B464AF221
:100BE000A001024600952046C0F6020113F0B0FCB9
:100BF000BBF1000F3FF4E4AE14E0B16DD3F8F02D7B
:100C000091427FF43CAFD3F8F42DF36D93427FF41F
:100C100036AF44F6F440C2F20000002104F090FB2D
:100C2000002046E7DFF844B01FE7DDE90623CAE904
:100C3000202373E7D7F8F41DD7F8EC2DD7F8F03D53
:100C4000706DB76DF56D00914AF2F4010190029755
:100C50000395C0F6020140F25E2010F089FE48E7DD
:100C6000FC3C012000C4226400000000004601207A
:100C700044F60453D7F8F05D716DF26CC2F20003D4
:100C80001868D7F8EC3D0095D7F8F44DD6F858E041
:100C90000194F56D02914AF2AC01CDF80CE0049597
:100CA000C0F6020113F054FC02E700BFAFF300806E
:100CB0009FED057ADFED057A03280CBF17EE900A49
:100CC00017EE100A704700BF000034440000B44320
:100CD0002DE9F0432DED068BD31A83B003F1FF39D4
:100CE000B9F1000F05460E46DDED108A9DED11AA03
:100CF000129FDDF84C8058DD07EE102AF8EEC7AAE7
:100D00009FED2C8A8AEE2A9A0024F6EE009A38EE9D
:100D1000298AF0EE687AE8EE097A013417EE901A23
:100D200030462A4601230097CDF80480FFF758FB90
:100D300006EE904AB8EEE68AB0EE687AA8EE097A36
:100D40000097CDF8048017EE101A30462A4600238B
:100D5000FFF746FB4C45DAD1CAEE2A7A30462A46DE
:100D600001230097CDF8048007EE109AF8EEC76AC9
:100D7000B6EE007A36EE877AF0EE686AE7EE276A1A
:100D800016EE901AFFF72CFB38EE8AAA30461AEEC0
:100D9000101A2A4600231097CDF8448003B0BDEC0A
:100DA000068BBDE8F043FFF71BBB06EE902AF8EE7A
:100DB000E6AAD1E700000000AFF30080AFF30080A7
:100DC000F0B50F46511C07EE901A0446F8EEE77A8C
:100DD00085B0154617EE901A4760A2601E46FFF7D1
:100DE00077FB2B1C18BF01232370204631460022BD
:100DF000FEF73EFF9FED0F7ADFED0F7A032E4FF0E7
:100E000000004FF000064FF0000E18BFF0EE477ADA
:100E1000C4F27A46CBF68070029021463A462B46C1
:100E2000CDED017ACDF800E003960020FFF750FFEA
:100E300005B0F0BD000034440000B443AFF30080BF
:100E40002DE9F0430E464AF22C11C0F6020102F5DC
:100E5000217485B0154613F07BFB2046FEF7E0FEBB
:100E6000D6F80412132900F2EE80DFE811F0E20058
:100E7000DE00DA00D600D200CE00CA00C600BE00F6
:100E8000B600B100AD00A800A400A0009C00730053
:100E90002A00220014002046FEF792FC2046FEF7AE
:100EA000B7FE014605F6F85005B0BDE8F043FFF780
:100EB000EFBAD6F8E031204601210022FFF7F0FA20
:100EC000ECE7204602210122FEF7D2FE0026204652
:100ED0004FF08041002201230027FFF741F9C4F2BF
:100EE000B436C4F2A0174FF000094FF080430293CC
:100EF000012021463C220223CDF800900196039761
:100F0000FFF7E6FE4FF00008002213462046394660
:100F1000C4F27A48FFF724F9012021463C2202233B
:100F2000CDF8009001960297CDF80C80FFF7D0FE27
:100F30000023CBF680730293009602230196CDF82E
:100F40000C80012021463C22FFF7C2FE002385F8D9
:100F50008432A3E7204602210122FEF789FE002108
:100F60002046C4F2343100220123FFF7F9F80022B1
:100F7000002113462046C4F2B431FFF7F1F80122F4
:100F8000002113462046C4F20741FFF7E9F800218B
:100F900000232046C4F234410122FFF7E1F8002388
:100FA00085F884327AE72046FEF79AFB76E72046FA
:100FB000FEF726FC72E72046FFF7A2FA6EE720460E
:100FC0000021FFF75DFB69E7204600F0E9F965E7DE
:100FD00020460121FFF754FB60E7D6F8E0312046B8
:100FE00024210122FFF75CFA58E7D6F8E0312046C9
:100FF0003C210222FFF754FA50E72046FEF720FB7F
:101000004CE72046FEF714F948E7204600F040FA86
:1010100044E72046FEF74CFA40E72046FEF7C8F9C1
:101020003CE72046FEF784FC38E7204600F050F904
:1010300034E72046D6F80C12D6F81022D6F8E03164
:10104000FFF7BEFE2AE74AF24810C0F6020005B0DC
:10105000BDE8F04316F0ACBEAFF30080AFF3008004
:101060002DE9F04F104681B0164698468946FEF7A6
:10107000CFFD98FBF0F505FB10853046FEF7C8FD67
:1010800007463046FEF7C4FD2F44013F97FBF0F3BF
:1010900003FB10773046FEF7BBFD06F67434294695
:1010A0000646204614F0BCFA98FBF6F807EE908A44
:1010B00006EE900AF8EEE77A9FED337A77EEA67A9D
:1010C0003A4667EE877A2046FDEEE77A002117EE72
:1010D000906AFEF76DFE2A46834600212046FEF701
:1010E00067FE3A4610F1000A4FF00101204618BF92
:1010F0004FF0010AFEF75CFE2A4610F100084FF09F
:101100000101204618BF4FF00108FEF751FE3A4694
:101110000221071C204618BF0127FEF749FE2A4678
:101120000221051C204618BF0125FEF741FE1BF1D8
:10113000000B18BF4FF0010B041C18BF0124D3454E
:1011400005D0514648463246F317FFF7B9FBB8457C
:1011500008D0002F0CBF0221032148463246F31766
:10116000FFF7AEFBA5420BD04846002C0CBF042174
:1011700005213246F31701B0BDE8F04FFFF7A0BBE1
:1011800001B0BDE8F08F00BF0050C347AFF300804F
:101190002DE9F04144F60855B2B0C2F2000506460A
:1011A00004A80F46FEF79CFE284600214FF48072EB
:1011B000F1F7BEFF0023C5F804311C46C5F8043121
:1011C00003E00134B4F57C7F4ED02346009703A89A
:1011D00004A93246FFF744FF9DF81430002BF0D0ED
:1011E00041F6F408C2F2000840F61103D8F80020D6
:1011F00092F8DD25C0F601035206049348BFA51CF2
:101200000CD4651C0AE00097FFF72AFFD8F80030DD
:1012100093F8DD355B0648BF013501353046FEF7F2
:10122000F7FC04EB400E75452B4604A9324603A893
:10123000E9D99FED137A002304A91944D1ED0C7A62
:10124000F8EEE77AF218C7EE877A04330C2BC2ED7A
:10125000037AF1D13046FEF7DBFCB4FBF0F303FB7D
:10126000104032B0BDE8F0814AF27810C0F60200BA
:1012700016F09EFD4FF0FF3032B0BDE8F08100BFA8
:101280000050C347AFF30080AFF30080AFF300809E
:1012900044F60453C2F2000318607047AFF30080B5
:1012A00041F6EC03C2F200034AF29C101B6844F6BC
:1012B000F441D3F85822C0F6020003F51773C2F2C6
:1012C00000010AF095B800BFAFF30080AFF30080D3
:1012D00070B500250570022101220446FEF7C8FC06
:1012E00001224FF4246120461346C4F25321FEF735
:1012F00037FF4CF6CD4120462B46C4F2F3210122A4
:10130000FEF72EFF01224CF2902120461346C4F234
:101310006831FEF725FF4FF2333120462B46C4F2E9
:1013200096310122FEF71CFF002120462A46C4F216
:10133000B4310123FEF714FF012246F24811204682
:101340001346C4F2CE31FEF70BFF4FF23331204685
:101350002B46C4F2F0310122FEF702FF012243F2D4
:10136000A40120461346C4F21441FEF7F9FE47F6E5
:101370009A1120462B46C4F225410122FEF7F0FEC9
:10138000002120462A462B46C4F23441BDE8704075
:10139000FEF7E6BEAFF30080AFF30080AFF300804E
:1013A00070B50122044602210025FEF761FC45F2DA
:1013B0002631204684F8645BC3F6D571FFF788F8C0
:1013C000002120462A46C4F258210123FEF7C8FE18
:1013D0000122002120461346C4F2DC21FEF7C0FEA4
:1013E000002120462B46C4F234310122FEF7B8FE1C
:1013F000002120462A462B46C4F26A31FEF7B0FE91
:101400000122002120461346C4F29131FEF7A8FEC6
:10141000002120462B46C4F2B4310122FEF7A0FE83
:10142000002120462A46C4F2CF310123FEF798FE60
:101430000122002120461346C4F2EB31FEF790FE54
:10144000002120462A462B46C4F2FC31FEF788FED6
:10145000002120462B46C4F207410122FEF780FE00
:1014600001224FF4004120461346C4F22241FEF708
:1014700077FE002120462B46C4F234410122BDE80C
:101480007040FEF76DBE00BFAFF30080AFF3008089
:1014900010B5022100220446FEF7EAFB0021204697
:1014A000C4F2DC2100220123FEF75AFE00220021B3
:1014B00020461346C4F2F021FEF752FE00212046DA
:1014C000C4F2663100220123FEF74AFE0022002109
:1014D00020461346C4F27031FEF742FE002120463A
:1014E000C4F2AF3100220123FEF73AFE00220021B0
:1014F00020461346C4F2B431FEF732FE00212046E6
:10150000C4F2EB3100220123FEF72AFE0022002163
:1015100020461346C4F2F031FEF722FE4FF400419C
:101520002046C4F2134100220123FEF719FE0022D7
:10153000002120461346C4F21641FEF711FE4FF477
:1015400000412046C4F22C4100220123FEF708FE90
:101550000022002120461346C4F22F41FEF700FE70
:101560004FF400412046C4F2314100220123FEF72E
:10157000F7FD0022002120461346C4F23441BDE8A5
:101580001040FEF7EDBD00BFAFF30080AFF3008069
:101590002DE9F0414C6A804620680F460FF058F95B
:1015A00042F61035014644F614664AF2B010C2F213
:1015B0000005C2F20006C0F602000CF011FD06F1B3
:1015C00010034AF2C01006F1200E3146D4F8C823A9
:1015D0006B60C0F6020004F57573C5F808E02E6074
:1015E00009F006FF4AF2D0106968D4F8CC2304F55C
:1015F0007673C0F6020009F0FBFE4AF2E010A9681B
:10160000D4F8D02304F57773C0F6020009F0F0FE99
:1016100040463946BDE8F041FCF742BAAFF30080DE
:1016200070B5044682B0002016460D4606F048FF0D
:101630002146113551F8040BF5F7EAFA2068F5F761
:1016400037FB02AA06EB052642F8046D012120684B
:10165000F5F7D6FB2068F5F74BFB2068F5F700FBA4
:1016600006F036FF02B070BDAFF30080AFF300802C
:10167000024644F64460C2F200000121FFF7D0BFE9
:10168000F0B5A2F1340348F6AD3544F684641B028C
:10169000C2F20004C6F6DB0585FB0365DB1727688D
:1016A00083B0A3EB253303F580740D464AF2F011A5
:1016B000009206462A4638462346C0F6020112F03A
:1016C00047FF30462946224603B0BDE8F040FFF709
:1016D000A7BF00BFAFF30080AFF30080AFF300807F
:1016E00030B4C40F051944F6446368100A46C2F2C8
:1016F000000305F00101091B03EB001030BCFFF7EC
:10170000BFBF00BFAFF30080AFF30080AFF3008036
:101710002DE9F84344F68463C2F20003D1F8D420E3
:1017200018600F46002A46D010460AF029F8264DC8
:101730003C4607F110084FF40369D4F8D860502EE6
:1017400004F104040BD0D7F8D40006F0C9FE3146EA
:1017500045F8040C2846A5F80A900AF059F84445C3
:1017600005F11005E9D14AF2302041F2E161C0F6FD
:101770000200C0F6010113F01BF94AF2342041F2D5
:101780007161C0F60200C0F6010113F0E1F844F601
:101790004460C2F20000002140F6B832FFF770FF4B
:1017A00044F64460C2F20000012141F65832BDE81F
:1017B000F843FFF765BF4AF21821C0F60201BDE801
:1017C000F84312F0C5BE00BF484E0020AFF30080C2
:1017D00041F6F403C2F200031B68C3F8000270472D
:1017E00070B546F25023C2F2000382B01B68054672
:1017F0000E46002B37D041F6F404C2F200042368F1
:10180000D3F80032012B2EDDFCF7EAFA2368D3F877
:10181000003290FBF3F202FB130030BB46F24C2384
:10182000C2F200031A68002A36D044F68860C2F279
:10183000000012F0C5FE642815D92846F0F7CCF850
:10184000044630460D46F0F7C7F8CDE9000144F6EE
:1018500088604AF2542122462B46C2F20000C0F6AC
:10186000020112F025FD02B070BD46F24C24C2F216
:1018700000042368002BF6D044F688604AF2402129
:10188000C2F20000C0F6020112F012FD0CF008F8DE
:10189000C8B900232360E6E744F688600122C2F25B
:1018A00000001A6012F024FE44F688604AF24421D7
:1018B0004AF24022C2F20000C0F60201C0F6020263
:1018C00012F0F6FCB1E744F68860C2F2000012F0B4
:1018D000D7FEDEE7AFF30080AFF30080AFF3008008
:1018E00008B54AF25C2041F2D171C0F60200C0F6A0
:1018F000010113F02DF846F25023C2F20003012239
:101900001A6008BDAFF30080AFF30080AFF3008032
:1019100038B549F60043C2F201030C461B78054670
:1019200003B138BD496A01F51A71FFF7F1FE284687
:101930002146BDE83840FFF72BBE00BFAFF3008063
:1019400038B541F6F405C2F2000546F264242B686E
:1019500093F8D005C0F3401013F082FBC2F20004EC
:101960004AF290210246C0F60201204612F0F0FD34
:101970002B684AF2A421D3F8E0252046C0F60201E4
:10198000BDE8384012F0E4BDAFF30080AFF3008053
:10199000042800DC704741F6F403C2F200031B6820
:1019A000C3F8E005FFF7CCBFAFF30080AFF30080D2
:1019B00008B541F6F403C2F2000300301B6893F847
:1019C000D02518BF012060F3451283F8D025FFF71A
:1019D000B7FF41F2DC23C2F2010300221A6008BD06
:1019E00070B50646002412F083FD002500234AF25C
:1019F000B4214AF24022F363C6E910453046C0F6EE
:101A00000201C0F60202BDE8704012F051BC00BFF6
:101A100008B541F6E803C2F200031868FCF790F934
:101A200046F26833C2F20003C21C43F648501A6003
:101A3000C2F20000BDE80840FFF7D2BFAFF300805C
:101A400010B5044612F004F9D4E9102352EA030455
:101A500022D0801A61EB0301A8220023F0F700FED8
:101A600041F6F403C2F2000344F240221B68D3F8AB
:101A7000E045C0F20F024CF6CD4302FB04F2CCF677
:101A8000CC43A3FB0242120900238B4208BF8242CF
:101A90002CBF0020012010BD002010BDAFF300803E
:101AA00010B5044612F0ACFD204610BDAFF3008027
:101AB00010B54AF2C42140F2F052044641F2883394
:101AC000C0F60201C1F2000212F002FC0123A3647D
:101AD0002046BDE81040FFF783BF00BFAFF3008092
:101AE00010B54AF240210446C0F6020112F0E0FBB4
:101AF000216BE26A46F25423C2F200038A1A1A608A
:101B00000BF0CEFE41F6F403C2F200031B6893F81B
:101B1000D0359B0600D500B910BD2046BDE8104069
:101B200012F0AEBDAFF30080AFF30080AFF30080E2
:101B300041F6F403C2F2000310B51A68C36BD2F881
:101B4000E0259342044607D32046FFF7C9FF20460D
:101B5000BDE81040FFF744BFFFF772FF0028F3D144
:101B600010BD00BFAFF30080AFF30080AFF3008083
:101B70002DE9F84341F6E803C2F200030446186871
:101B80000E461546FCF7DCF846F26833C2F2000355
:101B90001B6898420DD341F6F403C2F200031B68A0
:101BA00093F8D005820604D5D3F8E025E36B934281
:101BB00001D3BDE8F88312F04BF8804689460CF05B
:101BC000CFF8E36B0746CBB1216C44F60562C1EB5D
:101BD00008084FEA1818C0F2E042A2FB08124FEAC8
:101BE00052080133E363204612F0EAFC23280BD8A5
:101BF000002FDED1BDE8F8430CF0D2B8C4F8408025
:101C0000C4F844909846ECE73146204612F0F8FAC2
